:020000040800F2
:1000000000C00020ED2C0008A1260008A32600084F
:10001000A5260008A7260008A92600080000000061
:10002000000000000000000000000000315A00083D
:10003000AB26000800000000D15A0008155B00083C
:10004000352D0008352D0008352D0008352D000808
:10005000352D0008352D0008352D0008352D0008F8
:10006000352D0008352D0008352D0008352D0008E8
:10007000352D0008352D0008352D0008352D0008D8
:10008000352D0008352D0008352D0008352D0008C8
:10009000352D0008352D0008352D0008352D0008B8
:1000A000352D0008AD260008352D0008352D000837
:1000B000BD260008352D0008352D0008352D000817
:1000C000352D0008352D0008352D0008352D000888
:1000D000352D0008352D0008CD260008DD26000846
:1000E000352D0008352D0008352D0008352D000868
:1000F000352D0008352D0008352D0008352D000858
:10010000352D0008352D0008352D0008352D000847
:1001100015270008352D0008352D0008352D00085D
:10012000352D0008352D0008352D0008352D000827
:1001300000000000000000000000000000000000BF
:1001400000000000000000000000000000000000AF
:10015000000000000000000000000000000000009F
:10016000000000000000000000000000000000008F
:10017000000000000000000000000000000000007F
:10018000000000000000000000000000000000006F
:10019000000000000000000000000000000000005F
:1001A000000000000000000000000000000000004F
:1001B000000000000000000000000000000000003F
:1001C000000000000000000000000000000000002F
:1001D000000000000000000000000000000000001F
:0401E0005FF8E0F1F3
:1001F000844641EA000313F0030349D1403A23D374
:100200000B6803604B6843608B688360CB68C36096
:100210000B6903614B6943618B698361CB69C3617E
:100220000B6A03624B6A43628B6A8362CB6AC36266
:100230000B6B03634B6B43638B6B8363CB6BC3634E
:1002400040304031403ADBD230320BD30B68036090
:100250004B6843608B688360CB68C360103010319B
:10026000103AF3D20C3205D351F8043B40F8043B6A
:10027000043AF9D2043208D0D2071CBF11F8013B6E
:1002800000F8013B01D30B8803806046704700BF34
:10029000082A13D38B07B1D010F00303AED0C3F1FB
:1002A0000403D21ADB071CBF11F8013B00F8013B25
:1002B000A4D331F8023B20F8023B9FE7043AD9D39C
:1002C000013A11F8013B00F8013BF9D20B780370B9
:1002D0004B7843708B7883706046704781F00041A3
:1002E00002E000BF83F0004330B54FEA41044FEA1B
:1002F000430594EA050F08BF90EA020F1FBF54EAB6
:10030000000C55EA020C7FEA645C7FEA655C00F051
:10031000E2804FEA5454D4EB5555B8BF6D420CDD22
:100320002C4480EA020281EA030382EA000083EAA5
:10033000010180EA020281EA0303362D88BF30BD45
:1003400011F0004F4FEA01314FF4801C4CEA11319B
:1003500002D0404261EB410113F0004F4FEA0333FA
:100360004CEA133302D0524263EB430394EA050F85
:1003700000F0A780A4F10104D5F1200E0DDB02FAF4
:100380000EFC22FA05F2801841F1000103FA0EF288
:10039000801843FA05F359410EE0A5F120050EF14E
:1003A000200E012A03FA0EFC28BF4CF0020C43FA7F
:1003B00005F3C01851EBE37101F0004507D54FF08C
:1003C000000EDCF1000C7EEB00006EEB0101B1F5DC
:1003D000801F1BD3B1F5001F0CD349085FEA300022
:1003E0004FEA3C0C04F101044FEA445212F5800F2D
:1003F00080F09A80BCF1004F08BF5FEA500C50F1CA
:10040000000041EB045141EA050130BD5FEA4C0CAC
:10041000404141EB0101013C28BFB1F5801FE9D209
:1004200091F0000F04BF01460020B1FA81F308BF2C
:100430002033A3F10B03B3F120020CDA0C3208DDF8
:1004400002F1140CC2F10C0201FA0CF021FA02F1D3
:100450000CE002F11402D8BFC2F1200C01FA02F143
:1004600020FA0CFCDCBF41EA0C019040E41AA2BF68
:1004700001EB0451294330BD6FEA04041F3C1CDA30
:100480000C340EDC04F11404C4F1200220FA04F050
:1004900001FA02F340EA030021FA04F345EA0301FA
:1004A00030BDC4F10C04C4F1200220FA02F001FABC
:1004B00004F340EA0300294630BD21FA04F029463E
:1004C00030BD94F0000F83F4801306BF81F48011D7
:1004D0000134013D4EE77FEA645C18BF7FEA655C4A
:1004E00029D094EA050F08BF90EA020F05D054EA1C
:1004F000000C04BF1946104630BD91EA030F1EBF21
:100500000021002030BD5FEA545C05D14000494124
:1005100028BF41F0004130BD14F580043CBF01F517
:10052000801130BD01F0004545F0FE4141F47001FD
:100530004FF0000030BD7FEA645C1ABF19461046D8
:100540007FEA655C1CBF0B46024650EA013406BFD9
:1005500052EA033591EA030F41F4002130BD00BF98
:1005600090F0000F04BF0021704730B54FF4806455
:1005700004F132044FF000054FF0000150E700BFD6
:1005800090F0000F04BF0021704730B54FF4806435
:1005900004F1320410F0004548BF40424FF0000122
:1005A0003EE700BF42004FEAE2014FEA31014FEA65
:1005B00002701FBF12F07F4393F07F4F81F06051B4
:1005C000704732F07F4208BF704793F07F4F04BFFF
:1005D00041F40021704730B54FF4607401F00045DC
:1005E00021F000411CE700BF50EA010208BF70473C
:1005F00030B54FF000050AE050EA010208BF70472D
:1006000030B511F0004502D5404261EB41014FF495
:10061000806404F132045FEA915C3FF4D8AE4FF09D
:1006200003025FEADC0C18BF03325FEADC0C18BF80
:10063000033202EBDC02C2F1200300FA03FC20FAD1
:1006400002F001FA03FE40EA0E0021FA02F114441E
:10065000BDE600BF70B54FF0FF0C4CF4E06C1CEA37
:1006600011541DBF1CEA135594EA0C0F95EA0C0FA8
:1006700000F0DEF82C4481EA030621EA4C5123EA1B
:100680004C5350EA013518BF52EA033541F480114A
:1006900043F4801338D0A0FB02CE4FF00005E1FBFD
:1006A00002E506F00042E0FB03E54FF00006E1FB47
:1006B00003569CF0000F18BF4EF0010EA4F1FF048A
:1006C000B6F5007F64F5407404D25FEA4E0E6D41CA
:1006D00046EB060642EAC62141EA55514FEAC520DB
:1006E00040EA5E504FEACE2EB4F1FD0C88BFBCF557
:1006F000E06F1ED8BEF1004F08BF5FEA500E50F108
:10070000000041EB045170BD06F0004646EA0101CD
:1007100040EA020081EA0301B4EB5C04C2BFD4EBFF
:100720000C0541EA045170BD41F480114FF0000EF8
:10073000013C00F3AB8014F1360FDEBF002001F066
:10074000004170BDC4F10004203C35DA0C341BDCE0
:1007500004F11404C4F1200500FA05F320FA04F0B2
:1007600001FA05F240EA020001F0004221F00041E6
:1007700010EBD37021FA04F642EB06015EEA430E59
:1007800008BF20EAD37070BDC4F10C04C4F1200589
:1007900000FA04F320FA05F001FA04F240EA02003C
:1007A00001F0004110EBD37041F100015EEA430E0D
:1007B00008BF20EAD37070BDC4F1200500FA05F22D
:1007C0004EEA020E20FA04F301FA05F243EA0203AC
:1007D00021FA04F001F0004121FA04F220EA0200BB
:1007E00000EBD3705EEA430E08BF20EAD37070BD01
:1007F00094F0000F0FD101F00046400041EB0101E1
:1008000011F4801F08BF013CF7D041EA060195F0C2
:10081000000F18BF704703F00046520043EB03037C
:1008200013F4801F08BF013DF7D043EA0603704769
:1008300094EA0C0F0CEA135518BF95EA0C0F0CD074
:1008400050EA410618BF52EA4306D1D181EA0301BA
:1008500001F000414FF0000070BD50EA410606BFB4
:100860001046194652EA430619D094EA0C0F02D1F9
:1008700050EA013613D195EA0C0F05D152EA03363E
:100880001CBF104619460AD181EA030101F000415C
:1008900041F0FE4141F470014FF0000070BD41F0A5
:1008A000FE4141F4780170BD70B54FF0FF0C4CF47F
:1008B000E06C1CEA11541DBF1CEA135594EA0C0F9E
:1008C00095EA0C0F00F0A7F8A4EB050481EA030EEB
:1008D00052EA03354FEA013100F088804FEA0333D2
:1008E0004FF0805545EA131343EA12634FEA0222A0
:1008F00045EA111545EA10654FEA00260EF0004161
:100900009D4208BF964244F1FD0404F5407402D2B2
:100910005B084FEA3202B61A65EB03055B084FEA43
:1009200032024FF480104FF4002CB6EB020E75EB40
:10093000030E22BFB61A754640EA0C005B084FEA68
:100940003202B6EB020E75EB030E22BFB61A7546E5
:1009500040EA5C005B084FEA3202B6EB020E75EB30
:10096000030E22BFB61A754640EA9C005B084FEAA8
:100970003202B6EB020E75EB030E22BFB61A7546B5
:1009800040EADC0055EA060E18D04FEA051545EAA4
:1009900016754FEA06164FEAC30343EA52734FEA4D
:1009A000C2025FEA1C1CC0D111F4801F0BD141EAC6
:1009B00000014FF000004FF0004CB6E711F4801F2B
:1009C00004BF01430020B4F1FD0C88BFBCF5E06F0B
:1009D0003FF6AFAEB5EB030C04BFB6EB020C5FEA1B
:1009E000500C50F1000041EB045170BD0EF0004E70
:1009F0004EEA113114EB5C04C2BFD4EB0C0541EAA2
:100A0000045170BD41F480114FF0000E013C90E69E
:100A100045EA060E8DE60CEA135594EA0C0F08BF62
:100A200095EA0C0F3FF43BAF94EA0C0F0AD150EA61
:100A300001347FF434AF95EA0C0F7FF425AF1046F4
:100A400019462CE795EA0C0F06D152EA03353FF41C
:100A5000FDAE1046194622E750EA410618BF52EA99
:100A600043067FF4C5AE50EA41047FF40DAF52EA6D
:100A700043057FF4EBAE12E74FF0FF3C06E000BF0A
:100A80004FF0010C02E000BF4FF0010C4DF804CD17
:100A90004FEA410C7FEA6C5C4FEA430C18BF7FEAD7
:100AA0006C5C1BD001B050EA410C0CBF52EA430C05
:100AB00091EA030F02BF90EA020F0020704710F185
:100AC000000F91EA030F58BF994208BF90422CBF14
:100AD000D8176FEAE37040F0010070474FEA410C0D
:100AE0007FEA6C5C02D150EA013C07D14FEA430C2B
:100AF0007FEA6C5CD6D152EA033CD3D05DF8040B9C
:100B0000704700BF8446104662468C4619466346CD
:100B100000E000BF01B5FFF7B7FF002848BF10F1A4
:100B2000000F01BD4DF808EDFFF7F4FF0CBF0120E9
:100B300000205DF808FB00BF4DF808EDFFF7EAFF65
:100B400034BF012000205DF808FB00BF4DF808ED20
:100B5000FFF7E0FF94BF012000205DF808FB00BF15
:100B60004DF808EDFFF7CEFF94BF012000205DF89F
:100B700008FB00BF4DF808EDFFF7C4FF34BF0120AC
:100B800000205DF808FB00BF4FEA410C7FEA6C5C77
:100B900002D150EA013C0AD14FEA430C7FEA6C5C77
:100BA00002D152EA033C02D14FF0000070474FF0EF
:100BB000010070474FEA410212F5001215D211D51B
:100BC0006FF47873B3EB625212D94FEAC12343F04A
:100BD000004343EA505311F0004F23FA02F018BFCC
:100BE000404270474FF00000704750EA013005D195
:100BF00011F0004008BF6FF0004070474FF0000058
:100C0000704700BF53B94AB9002908BF00281CBF6C
:100C10004FF0FF314FF0FF3000F076B9ADF1080C26
:100C20006DE904CE00F006F8DDF804E0DDE902230A
:100C300004B070472DE9F047089E0D4604468846EB
:100C4000002B4DD18A42944668D9B2FA82F252B151
:100C500001FA02F3C2F1200120FA01F10CFA02FCC0
:100C600041EA030894404FEA1C41B8FBF1F71FFA30
:100C70008CFE01FB178807FB0EF0230C43EA0843A8
:100C800098420AD91CEB030307F1FF3580F01E815F
:100C9000984240F21B81023F63441B1AB3FBF1F000
:100CA00001FB103300FB0EFEA4B244EA0344A64548
:100CB0000AD91CEB040400F1FF3380F00981A6453A
:100CC00040F20681644402380021A4EB0E0440EA9D
:100CD00007401EB10023D440C6E90043BDE8F087B9
:100CE0008B4208D9002E00F0EE800021C6E90005F5
:100CF0000846BDE8F087B3FA83F100294AD1AB4238
:100D000002D3824200F2FC80841A65EB03030120C7
:100D10009846002EE2D0C6E90048DFE702B9FFDEC0
:100D2000B2FA82F2002A40F09180A1EB0C0001217E
:100D30004FEA1C471FFA8CFEB0FBF7F307FB1300CA
:100D4000250C45EA00450EFB03F0A84208D91CEB30
:100D5000050503F1FF3802D2A84200F2CE804346D7
:100D60002D1AB5FBF7F007FB10550EFB00FEA4B2E1
:100D700044EA0544A64508D91CEB040400F1FF35FC
:100D800002D2A64500F2B6802846A4EB0E0440EA43
:100D900003409EE7C1F120078B4022FA07FC4CEA92
:100DA000030C25FA07FA4FEA1C49BAFBF9F820FAB6
:100DB00007F309FB18AA8D401FFA8CFE1D4300FAA9
:100DC00001F308FB0EF02C0C44EA0A44A04202FA9C
:100DD00001F20BD91CEB040408F1FF3A80F0888083
:100DE000A04240F28580A8F102086444241AB4FBB2
:100DF000F9F009FB104400FB0EFEADB245EA0444D5
:100E0000A64508D91CEB040400F1FF356CD2A645B9
:100E10006AD90238644440EA0840A0FB0295A4EB7A
:100E20000E04AC42C846AE4656D353D0002E69D00D
:100E3000B3EB080264EB0E0422FA01F304FA07F79D
:100E40001F43CC40C6E90074002147E70CFA02FCBE
:100E5000C2F1200125FA01F34FEA1C4720FA01F103
:100E600095400D43B3FBF7F107FB11331FFA8CFEDE
:100E7000280C40EA034001FB0EF3834204FA02F41B
:100E800008D91CEB000001F1FF382FD283422DD985
:100E900002396044C01AB0FBF7F307FB1300ADB290
:100EA00045EA004503FB0EF0A84208D91CEB0505F6
:100EB00003F1FF3816D2A84214D9023B6544281A20
:100EC00043EA014138E73146304607E72F46E4E67A
:100ED0001846F9E64B45A9D2B9EB020865EB0C0EB2
:100EE0000138A3E74346EAE7284694E74146D1E7BD
:100EF000D0467BE76444023847E7023B65442FE76E
:100F0000084606E73146E9E6704700BF38B5104DA0
:100F10001021284602F00AFBC4002021284602F0D6
:100F200005FB44EA800464B24FF48071284602F065
:100F3000FDFA44EA400464B24FF40071284602F01E
:100F4000F5FA40B22043C04300F00F0038BD00BFA7
:100F5000000C0140F8B505460C461646094F012223
:100F60000421384602F0E9FA33462246294606486B
:100F700003F0BBF900220421384602F0DEFA2046D5
:100F8000F8BD00BF000C01401810002010B50C4641
:100F900013460A460146044803F00DFA08B92046F4
:100FA00010BD0020FCE700BF1810002030B583B052
:100FB00004460020ADF8040001F0ACFA8DF80400FE
:100FC00001AB012211460E4801F022FA9DF80430CF
:100FD000237010B1002003B030BD01AB01222021ED
:100FE000074801F00AFA05469DF8041021721720FF
:100FF00001F0CEFA0DB90120EDE70020EBE700BFCC
:10100000440A002030B583B00446002000900190CF
:1010100001F080FAADF80000022001F07BFAA07028
:10102000042001F077FAE070A378022B0AD0042B99
:101030000CD0E378013B042B0FD8DFE803F00B1E44
:1010400022262A000123ADF80230F2E70023ADF892
:101050000230EEE70123ADF804303C23ADF8063052
:101060006B4604221421164801F0D2F9BDF8003075
:10107000237090B1002003B030BD0123ADF80430DF
:10108000EBE70223ADF80430E7E70223ADF80430C4
:10109000E3E70323ADF80430DFE76B4601220721C5
:1010A000074801F0AAF905469DF8001021721720A3
:1010B00001F06EFA0DB90120DDE70020DBE700BF8B
:1010C000440A002000B587B06DE03C4801F05CF9AF
:1010D000002001F01FFA03A8FFF794FF68B19DF804
:1010E0000C30012B09D1364B195D132001F050FA59
:1010F00003E04FF4FA6004F023F90134072C4AD8D6
:101100002F4B195D1429E0D00029F6D02B4801F0AF
:101110003BF9002001F0FEF96846FFF747FF002881
:10112000E7D09DF80030012BE3D1254B195D13204A
:1011300001F02EFA002303930493ADF8143001203C
:1011400001F0E8F9ADF80C00022001F0E3F9ADF888
:101150000E00042001F0DEF9ADF81000112001F0BE
:10116000D9F9ADF81200122001F0D4F9ADF814004D
:10117000124D0DF10E0302221146284601F048F9E6
:10118000C82004F0DDF80DF1120302220B212846DD
:1011900001F03EF9ADE70B4B186804F053FA4FF439
:1011A0007A7004F0CDF84FF0FF31064B186804F068
:1011B00007FA0028F7D10446A0E700BF440A002040
:1011C000AC0B0020400A002010B582B00146094C4B
:1011D000204601F0D9F80A2004F0B2F80DF1060318
:1011E00001221146204601F008F9B0FA80F04009CA
:1011F00002B010BD440A002070B507240FE0E31FC1
:10120000274AD5540021152001F0C2F910E0012130
:10121000152001F0BDF90A2004F092F801340A2CDF
:1012200018DCE5B22846FFF7CFFF06460028E6D1D6
:101230000A2004F085F8002EEDD12846FFF7C4FF00
:101240000028E4D0E31F164AD5540021152001F0F0
:101250009FF9E0E71420FFF7B7FF044638B90A20EA
:1012600004F06EF85CB1642004F06AF870BD0C4BB9
:1012700014221A710021152001F08AF9EFE71420D9
:10128000FFF7A2FF38B1064B14221A710021152076
:1012900001F07EF9E7E70121152001F079F9E2E795
:1012A000AC0B002008B509E0FFF7A6FF084B186853
:1012B00004F0C8F94EF6602004F042F84FF0FF3118
:1012C000034B186804F07CF90028EDD0F2E700BF6A
:1012D000400A002010B586B0002004F013F9134B2B
:1012E0001860684601F040F801238DF80030104B7B
:1012F0000193104B0293104C6946204601F06EF8A2
:101300004FF4C871204601F029F84FF4C871204607
:1013100001F027F800221146084803F099FF002247
:101320001146074803F094FF06B010BD400A0020A4
:101330008D0F0008550F0008440A0020A512000870
:10134000C5100008F8B505460C461646094F01229F
:101350000221384602F0F1F8334622462946064873
:1013600002F0C3FF00220221384602F0E6F82046D0
:10137000F8BD00BF00080140D00F002010B50C469A
:1013800013460A460146044803F015F808B92046FA
:1013900010BD0020FCE700BFD00F002010B584B0C6
:1013A0000446002101910291ADF80C1001AB052219
:1013B0001C4801F022F810B1002004B010BDBDF8A7
:1013C00004302370BDF806306370BDF80830A37098
:1013D000BDF80C30E370002300936B4601220E2110
:1013E000104801F00AF810B9BDF8003023716B46BF
:1013F000022211210B4801F000F828B9BDF8003095
:10140000A371BDF80230E3716B46012259210548F2
:1014100000F0F3FF20B9BDF8003063710120CCE784
:101420000120CAE7B80B002000B585B000256FE0A9
:101430000221084601F0ACF85BE00135EDB2092D60
:1014400059D801A800F026FC00238DF80430AA2208
:101450008DF809208DF805308DF807304FF47A703B
:1014600003F06EFF132001F055F8ADF800001720CF
:1014700001F050F8ADF802006B4602226A212948BB
:1014800000F0C6FF4FF47A7003F05AFF0134092CC4
:1014900036D8254B195D0029F8D0224800F074FF9A
:1014A00001A8FFF77BFF0028C7D09DF80430012B6F
:1014B000C3D19DF80A10112001F06AF89DF80B10B5
:1014C000122001F065F80021152001F061F801AB50
:1014D00001220A21134800F09BFF4FF4967003F09D
:1014E0002FFF9DF80630022BA2D00421022001F02C
:1014F0004FF80025A5E70121152001F049F8A0E7E4
:101500000A4B186804F09EF84FF47A7003F018FF45
:101510004FF0FF31054B186804F052F804460028DC
:10152000B5D0F1E7B80B0020200D0020B40B00204F
:1015300010B582B00146094C204600F025FF64201A
:1015400003F0FEFE0DF1060301221146204600F0D5
:1015500054FFB0FA80F0400902B010BDB80B002073
:1015600070B5012407E0C82003F0EAFE9EB1C82050
:1015700003F0E6FE0134082C1DDCE5B22846FFF737
:10158000D7FF06460028EED00B4B1D550021152035
:1015900000F0FEFFE7E72846FFF7CAFF30B1064B31
:1015A0001D550021152000F0F3FFE0E70121152073
:1015B00000F0EEFFDBE770BD200D002008B509E06C
:1015C000FFF7CEFF084B186804F03CF84EF6602099
:1015D00003F0B6FE4FF0FF31034B186803F0F0FF45
:1015E0000028EDD0F2E700BFB40B002010B586B0A4
:1015F000002003F087FF134B1860684600F0B4FE2C
:1016000001238DF80030104B0193104B0293104CC6
:101610006946204600F0E2FE4FF4C871204600F013
:101620009DFE4FF4C871204600F09BFE002211463B
:10163000084803F00DFE00221146074803F008FE9B
:1016400006B010BDB40B00207D1300084513000840
:10165000B80B0020BD1500082914000830B583B070
:101660000023019388421AD805460C4601F020FD5C
:101670000C48002303608560641B04F2FF34A40A55
:10168000C46001A901F0E0FD044620B901F02AFD83
:10169000204603B030BD01F025FD0724F8E7022401
:1016A000F6E700BF2C0D0020002950D02DE9F843AB
:1016B00005460C4612B90120BDE8F8834FEA9208AE
:1016C000C2F3400902F0010701F0F2FC0026464592
:1016D00013D22378627803EB0223A27803EB024350
:1016E000E27803EB026200232946022001F038FD74
:1016F00078BB043504340136E9E70026B1450ED93C
:101700002278637802EB032292B20023294601205B
:1017100001F026FDF8B9023502340136EEE7002665
:1017200002E0023502340136B7420CD92278A2F524
:10173000807292B200232946012001F011FD002899
:10174000EFD00520B8E701F0CDFC0020B4E7012080
:1017500070470320B0E70420AEE7000010B50A4848
:1017600006F0E6F9002405E00134E4B24FF4167007
:1017700003F0E6FD4FF40051044801F0E4FE092CAB
:10178000F2D90024F0E700BF80DA00080010014021
:1017900008B5044A0021044803F05AFD034B1860C1
:1017A00008BD00BFB0DA00085D1700083C0D00203E
:1017B0002DE9F04389B0002404940594069407941D
:1017C000334B9A6942F010029A619A6902F0100252
:1017D0000092009A9A6942F020029A619A6902F096
:1017E00020020192019A9A6942F004029A619A6970
:1017F00002F004020292029A9A6942F008029A6187
:101800009B6903F008030393039BDFF8889022464B
:101810004FF40051484601F090FEDFF87C802246EC
:1018200048F20201404601F088FE1C4D224643F278
:101830000401284601F081FE4FF400530493012770
:10184000059706940226079604A9484601F04EFD26
:1018500048F20203049305970694079604A94046AC
:1018600001F044FD43F204030493059706940796A0
:1018700004A9284601F03AFD4FF44C7304930594F3
:10188000069404A9284601F031FD09B0BDE8F083B3
:10189000001002400010014000080140000C01400F
:1018A00010B504460268074B9A4204D02368B3F18E
:1018B000804F03D010BD01F051FAF7E703F018FC98
:1018C000F8E700BF002C014072B6FEE700B591B00A
:1018D0002822002106A806F077F80023019302933E
:1018E000039304930593092306934FF480330793DE
:1018F00001220A920C9202220D920E934FF4E013F1
:101900000F9306A801F03EFE80B90F230193022138
:101910000291002303934FF480620492059301A87F
:1019200002F062F820B911B05DF804FBFFF7CCFFBC
:10193000FFF7CAFF08B501F0FFF9FFF7C7FFFFF790
:1019400037FF00F0A5FF00F0D7FF00F0EFFF00F039
:101950002BFF00F0B7FFFFF749FE00F0F1F9FFF7AA
:10196000D5FA082809D0102000F01AFE03F0C8FBB1
:10197000FFF70EFF03F0E6FBFEE7FFF7ABFCF5E732
:1019800000B583B00DF1060301226621044800F082
:1019900034FDB0FA80F0400903B05DF804FB00BFED
:1019A0004C0D002000B58BB00023089309930593DC
:1019B00006938DF81C30C4E001238DF81430BDF877
:1019C0000630023B8DF81730BDF804305E4AA2FBAA
:1019D0000323DB088DF818308CE000238DF81530D8
:1019E0008DF819509DF81450012D5BD1002E59D15E
:1019F000642003F0A5FC2946002000F0C9FD9DF8F5
:101A00001510012000F0C4FD9DF81710042000F00F
:101A1000BFFD9DF818100E2000F0BAFD0021142023
:101A200000F0B6FD494B00221A7001263AE001236E
:101A30008DF81530D4E702238DF81530D0E7032355
:101A40008DF81530CCE7414A13780133137004F157
:101A500028030DEB030212F8083C0133DBB202F855
:101A6000083C9DF81450ADB90A2B01D8012619E0A5
:101A70000121142000F08CFD2946002000F088FD93
:101A80000023324A137004F128026A4402F8083C29
:101A9000012607E0012605E001224FF400512C4801
:101AA00001F04BFD4FF47A7003F04AFC0134072C2F
:101AB00034D8284B1B5D002BEED04FF40051244846
:101AC00001F041FDE3B20133DDB204EB840101EB2F
:101AD000810166316B46042289B21F4800F08DFCFB
:101AE0000028B0D1BDF80030AA2B3FF465AF002329
:101AF0008DF81430002000F00DFDBDF80230013BE0
:101B0000032B3FF66DAF01A252F823F0DB1900085A
:101B1000371A00083F1A00082F1A00089DF81440D1
:101B20005CB956B90021142000F032FD2146002096
:101B300000F02EFD054B00221A704FF47A7003F06E
:101B4000FFFB00242646B2E7CDCCCCCC480D0020CC
:101B5000000C0140400D00204C0D002000B5C1B02C
:101B600031E040F2DC5003F0EBFB2F4805F0E0FFE2
:101B700029E02E4B00225A5401310829F9DD01AB2E
:101B8000082278212A4800F02DFC48BB9DF804105B
:101B90000A2000F0FDFC0021142000F0F9FC0022D6
:101BA000244B1A7009E09DF80430C2F107018B4004
:101BB000C3F3C0131D498B540132082AF3DD4EF6DE
:101BC000602003F0BDFBFFF7DBFE0028C9D0002436
:101BD0000194F622214602A805F0F6FE2146CCE744
:101BE00001AB08227821124800F0FCFB04464FF4B8
:101BF000967003F0A5FB002CE1D1002209E09DF8CE
:101C00000430C2F107018B40C3F3C01307498B5462
:101C10000132082AF3DD074B00221A709DF80410E8
:101C20000A2000F0B5FCCAE7D4DA0008400D002015
:101C30004C0D0020480D0020F8B505460C46164610
:101C40000A4F01224FF40041384601F076FC33463A
:101C500022462946064802F048FB00224FF4004184
:101C6000384601F06AFC2046F8BD00BF000801407C
:101C70006010002010B50C4613460A460146044881
:101C800002F099FB08B9204610BD0020FCE700BF18
:101C90006010002030B585B00278012A0ED00021F6
:101CA0000B464FF0550E42781FFA82FC541C013A45
:101CB000032A09D8DFE802F00A0E0E33C178013199
:101CC00003794FF0AA0EEEE7A44603E00CF1030CF3
:101CD0001FFA8CFCADF804E0ADF806C003EB8303FB
:101CE0005B00ADF80830ADF80A100023ADF80C30F9
:101CF0004179013901EB810101EB8101663101ABD1
:101D0000052289B20C4800F083FB58B90021142049
:101D100000F03EFC094B00221A7005B030BD4FF0B8
:101D2000030CD7E70121142000F032FC034A13789A
:101D300001331370F1E700BF4C0D0020480D002067
:101D400030B587B0684600F00FFB01258DF80050D4
:101D5000114B0193114B0293114C6946204600F040
:101D60003DFB4FF49671204600F0F8FA4FF496715F
:101D7000204600F0F6FA2946204600F005FB002236
:101D80001146084803F064FA00221146064803F0A1
:101D90005FFA07B030BD00BF751C0008391C000891
:101DA0004C0D00205D1B0008A51900080346B0F883
:101DB0000421805C0132A3F804217047B0F804319B
:101DC000C1540133A0F804317047B0F80431013335
:101DD000A0F804317047B0F80431C15C5A1C825C31
:101DE0000233A0F8043142EA01207047B0F8043110
:101DF0000A0AC2545A1C81540233A0F804317047B5
:101E00000023A0F80431704710B50446FFF7F8FF2F
:101E1000002384F8063184F80731A4F8083184F8E7
:101E20000A3184F80B3110BD38B504460D46B0F8C0
:101E300066314FF6FF7293421ED00133A0F866312F
:101E4000D4F85C3100224FF482712046D4F850C19E
:101E5000E0472046FFF7D8FF94F8653184F8063153
:101E600084F80751B4F86621A4F808211BB994F846
:101E70004C31012B04D038BD0123A0F86631DFE7D7
:101E800084F80A31F7E700B54FF0000E4FF6FF7304
:101E90000CE05B08013A3AB113F0010FF9D04AF2B5
:101EA000010C8CEA5303F5E70EF1010E8E4504D2C6
:101EB00010F80E2053400822EDE75BBA98B25DF8A7
:101EC00004FB38B50C46D0F85051B0F804C1D0F836
:101ED0005C31D0F844216044A847844208D009DD31
:101EE000002802DB6FF0020038BD6FF00300FBE753
:101EF0000020F9E76FF00300F6E738B50C46D0F89C
:101F00005451D0F85C31D0F84421A847844208D01D
:101F100009DD002802DB6FF0020038BD6FF003001E
:101F2000FBE70020F9E76FF00300F6E770B590F8E3
:101F30004C31012B02D00025284670BD0446D0F854
:101F40005831D0F85C21B0F80411984706460221B8
:101F50002046FFF7B6FF05460028EDD12046FFF7E3
:101F60003AFF8642E8D06FF00405E5E7F8B504468D
:101F70000D46D0F84461D0F84831C0F84431FFF73D
:101F800043FF00232B7094F84C31012B04D0022B1B
:101F90001FD000263046F8BD01212046FFF791FFF3
:101FA000C4F8446106460028F4D101262E7020466C
:101FB000FFF7FCFE84F8060131462046FFF781FF5B
:101FC00006460028E6D12046FFF7F0FE84F8070118
:101FD000E0E701212046FFF774FFC4F8446106469C
:101FE0000028D7D101232B702046FFF7EEFE0721F2
:101FF0002046FFF766FF06460028CBD12046FFF7B4
:10200000FFFE2046FFF7E7FEA4F808012046FFF791
:10201000E2FE07462046FFF7DEFE05462046FFF7B4
:10202000C5FE84F806012046FFF7C0FE84F80701CC
:1020300027B9FF2DAED96FF00506ABE76FF00506A7
:10204000A8E738B504460D46FFF7DAFE94F84C31A0
:10205000012B07D0022B0BD094F807112046FFF775
:10206000ADFE38BD94F806112046FFF7A7FEF3E752
:10207000B4F808112046FFF7B9FE00212046FFF70B
:10208000B5FEA91C89B22046FFF7B0FE94F80611F0
:102090002046FFF793FEDFE710B5044690F84C3179
:1020A000012B05D0B4F804112046FFF726FF10BD20
:1020B000D0F85831D0F85C21B0F8041198470146A7
:1020C0002046FFF793FEEDE7F0B583B00446B0F885
:1020D000086190F8067190F8075100238DF80730D9
:1020E0000DF10701FFF742FF88B994F84C31022B3C
:1020F0000FD0012B14D094F80731AB4207D0803BAE
:10210000AB4223D101212046FFF7DBFE78B103B0BB
:10211000F0BDB4F80821B242EBD06FF00500F6E74D
:1021200094F80631BB42E6D06FF00600EFE7204698
:10213000FFF73CFE05462046FFF7F8FE0028E6D1F3
:102140006B1EDBB2032B04D868B2E0E76FF001002E
:10215000DDE76FF00100DAE708B5FFF772FF08BDB1
:10216000F8B504460D46FFF7AFFF034608B1184621
:10217000F8BD01212046FFF7A4FE03460028F6D152
:102180002046FFF713FE0746FA2817D881B22046EB
:10219000FFF797FE03460028E9D1002601E0A85585
:1021A0000136B74205DD2046FFF700FE002DF6D1CF
:1021B000F6E72046FFF7BAFE0346D8E76FF00103C3
:1021C000D5E72DE9F04104460F461546FFF77CFFA1
:1021D00008B1BDE8F08101212046FFF772FE00281A
:1021E000F7D12046FFF7E2FD8046FA281FD881B2DA
:1021F0002046FFF766FE0028EBD1002602E025F816
:1022000016000136C8F34703B34205DD2046FFF749
:10221000E2FD002DF3D1F4E72046FFF787FE00280A
:10222000D7D1B8EB470FD4D06FF00100D1E76FF0F2
:102230000100CEE770B51D46013B9BB2B3F5FA6FC6
:102240001DD2044616465319B3F5803F1AD8FFF73E
:10225000EBFD04212046FFF77FFF31462046FFF7C4
:10226000C5FD29462046FFF7C1FD2046FFF714FFB4
:1022700000B170BD04992046FFF772FFF9E74FF0F7
:10228000FF30F6E74FF0FF30F3E770B51D46013B36
:102290009BB27C2B1ED8044616465319B3F5803FDB
:1022A0001BD8FFF7C1FD04212046FFF755FF31463B
:1022B0002046FFF79BFD29462046FFF797FD204665
:1022C000FFF7EAFE00B170BD049A29462046FFF7E9
:1022D00078FFF8E74FF0FF30F5E74FF0FF30F2E717
:1022E00040B338B50C4605464FF4B472002105F0F2
:1022F0006BFB4FF0FF33C5F84431C5F84831E4B10A
:102300006269154B9A421BD12378013BDBB2012B4A
:1023100019D86368D3B1A368DBB105F5A67EA446DE
:10232000BCE80F00AEE80F009CE803008EE8030055
:10233000002038BD4FF0FF3070474FF0FF30F8E716
:102340004FF0FF30F5E74FF0FF30F2E74FF0FF308E
:10235000EFE74FF0FF30ECE7BEDEFFFFC0F84811BB
:102360007047C0F8441170470023036043608360E6
:10237000C36003614361024BC360024B436170471A
:10238000871E0008BEDEFFFF80F8651170472DE94B
:10239000F04104460E461546FFF796FE08B1BDE82B
:1023A000F08104212046FFF78CFD0028F7D120465C
:1023B000FFF711FD07462046FFF70DFD804620463A
:1023C000FFF7B4FD0028EAD1B74204D1A845E6D012
:1023D0006FF00100E3E76FF00100E0E708B5FFF7F9
:1023E0007FFF08BD00B583B0009313460A46012164
:1023F000FFF720FF03B05DF804FB00B583B0009346
:1024000013460A460321FFF740FF03B05DF804FBC3
:102410002DE9F0411F46531E9BB27A2B34D8054656
:10242000884616468B18B3F5803F30D85400E4B286
:102430001021FFF7F9FC611D2846FFF78DFE41468C
:102440002846FFF7D3FC31462846FFF7CFFC21464C
:102450002846FFF7B3FC002405E037F8141028469F
:10246000FFF7C4FC0134A642F7DC2846FFF714FE50
:1024700010B995F80A310BB1BDE8F08132464146FA
:102480002846FFF784FFF7E74FF0FF30F4E74FF0FF
:10249000FF30F1E710B51D4CB4F800C0013989B226
:1024A0008C181E2C2FDCA1EB0C0189B29BB1012BE7
:1024B00025D0002028E0164C34F811E04FEA1E2EFB
:1024C00084460CF802EB14F811404470013189B2D3
:1024D000013A92B26046002AEDD1184614E08446D3
:1024E0001CF8023B0A4C1B0224F8113040780343CD
:1024F00024F81130013189B2013A92B26046002AC3
:10250000EDD1002000E0012010BD00BFF00E002042
:10251000B40E00201D2803D8024B33F8100070477A
:1025200000207047B40E002000B583B00025009550
:102530004FF416530322C1B2284602F063FA02F0A8
:10254000C3FA2C460BE001224FF480510F4800F0F3
:10255000F4FF00250134E4B2052002F0F1FE02F0A0
:10256000C5FA0A2CEFD91520FFF7D4FF20B91420A3
:10257000FFF7D0FF0028E6D00135ADB2142DE9D920
:102580004FF48051014800F0DEFFE3E7000C01400A
:102590001D2802D8014B23F810107047B40E0020FC
:1025A00008B50146024A034802F052FE08BD00BFCA
:1025B0000CDB00082925000800B583B0114B9A698F
:1025C00042F001029A619A6902F001020092009AB7
:1025D000DA6942F08052DA61DB6903F080530193DB
:1025E000019B00220F216FF0010000F0DBFB064A87
:1025F000536823F0E06343F00073536003B05DF869
:1026000004FB00BF001002400000014030B589B05B
:1026100004461E4B9A6942F400629A619B6903F476
:1026200000630193019B02A903A801F0B9FA01F02C
:10263000A7FA03461648A0FB03239B0C013B154851
:10264000154A026040F2E732C26043600023036132
:102650008360836101F034FC054610B1284609B05F
:1026600030BD0C4801F0E8FA05460028F6D11920E3
:1026700000F0D0FB0F2C01D90125EFE70022214605
:10268000192000F08FFB054B1C60E7E700100240AB
:1026900083DE1B43F40E0020002C014008000020C4
:1026A000FEE7FEE7FEE7FEE7FEE7704708B50248F3
:1026B00001F002FB08BD00BFF40E002008B502487F
:1026C00001F0FAFA08BD00BF400F002008B502482B
:1026D00001F066FF08BD00BFD00F002008B50C4B0D
:1026E0001B68DB6813F0200F0CD1094B1B68DB68FB
:1026F00013F0800F09D1272000F0ACFB044801F053
:102700004FFF08BD02F0BAFCEFE702F0AFFCF2E7C2
:102710001810002008B5024801F042FF08BD00BFB4
:10272000601000200120704708B505F023F916233A
:1027300003604FF0FF3008BD08B54FF0FF31FFF7E1
:10274000F3FFFEE74FF0FF3070474FF400534B604C
:1027500000207047012070470020704710B50346E5
:102760000C4A0D490D48006840B10C48006803440C
:10277000521A934206D8094A136010BD0748084C04
:102780000460F2E705F0F6F80C2303604FF0FF3029
:10279000F3E700BF00C00020000400003C0F002051
:1027A00028A000207047000000B587B000230293E6
:1027B0000393049305930093019315484FF08042CF
:1027C000026047224260836040F61F52C26003618C
:1027D000836101F075FB90B94FF48053029302A915
:1027E0000B4801F0A5FB68B90023009301936946EB
:1027F000074801F01DFC40B907B05DF804FBFFF786
:1028000063F8E9E7FFF760F8EEE7FFF75DF8F3E755
:10281000400F00200368B3F1804F00D0704700B52F
:1028200083B003F50433DA6942F00102DA61DB694F
:1028300003F001030193019B002205211C2000F0FD
:10284000B1FA1C2000F0E6FA03B05DF804FB0000CA
:1028500010B514464FF47A7392B2024801F0ABFD02
:10286000204610BD880F002008B50A464FF47A7341
:102870000146024801F039FD08BD00BF880F002065
:1028800010B50846144691B2FFF7EEFF204610BD82
:1028900008B50A480A4B03604FF4165343600023FF
:1028A0008360C36003610C2242618361C36101F0F4
:1028B000ECFC00B908BDFFF707F8FBE7601000204B
:1028C000004C004008B50A480A4B03604FF4E1335E
:1028D000436000238360C36003610C224261836113
:1028E000C36101F0D2FC00B908BDFEF7EDFFFBE7C4
:1028F000880F00200038014008B50A480A4B0360E1
:102900004FF41653436000238360C36003610C22BD
:1029100042618361C36101F0B8FC00B908BDFEF7F4
:10292000D3FFFBE7D00F00200044004008B50A4861
:102930000A4B03604FF41653436000238360C36067
:1029400003610C2242618361C36101F09EFC00B906
:1029500008BDFEF7B9FFFBE7181000200048004053
:1029600030B58DB00023089309930A930B93036845
:10297000664A93420BD0664A93423AD0654A9342E4
:1029800061D0654A934200F08E800DB030BD634B3C
:10299000DA6942F40022DA61DA6902F40022009274
:1029A000009A9A6942F010029A619B6903F0100341
:1029B0000193019B4FF4806308930223099303233F
:1029C0000B93574D08A9284600F090FC4FF4006384
:1029D0000893002409940A9408A9284600F086FC6C
:1029E00022460521342000F0DDF9342000F012FAEF
:1029F000CBE74A4B9A6942F480429A619A6902F4A1
:102A000080420292029A9A6942F004029A619B699A
:102A100003F004030393039B4FF400730893022312
:102A2000099303230B933F4C08A9204600F05EFC5A
:102A30004FF480630893002309930A9308A9204662
:102A400000F054FCA1E7354BDA6942F40032DA6158
:102A5000DA6902F400320492049A9A6942F004029C
:102A60009A619B6903F004030593059B0423089373
:102A70000223099303230B932A4D08A9284600F04B
:102A800035FC08230893002409940A9408A92846D1
:102A900000F02CFC22460521262000F083F9262098
:102AA00000F0B8F971E71D4BDA6942F48022DA616F
:102AB000DA6902F480220692069A9A6942F00802C4
:102AC0009A619B6903F008030793079B4FF48063A7
:102AD00008930223099303230B93134D08A9284657
:102AE00000F004FC4FF400630893002409940A9456
:102AF00008A9284600F0FAFB22460521272000F00D
:102B000051F9272000F086F93FE700BF004C004054
:102B100000380140004400400048004000100240DE
:102B20000010014000080140000C0140844610469E
:102B30000EE0400080B20133072B08DC10F4004F98
:102B4000F7D041F2210282EA400080B2F3E7013976
:102B5000002905DD1CF8013B80EA03200023EBE798
:102B6000704710B50446002205390330FFF7DEFF39
:102B700094F8832094F8843043EA0223984201D0E9
:102B8000002010BD0120FCE700B583B04FF0AA3350
:102B9000019304220DEB02010248FEF785FD03B00C
:102BA0005DF804FBFC8F010838B50C460378012B57
:102BB00003D0042B75D0002038BD11880139204680
:102BC000FFF7CFFF002864D03F4B1B78012B2AD0A2
:102BD000052B42D0022BEED163783C4A1278934207
:102BE000E9D1A278DB43DBB29A42E4D1384D2888A0
:102BF0000138C0018022E11C00F1006000F548406E
:102C0000FEF752FD2B8801332B80304A1378591C74
:102C10001170FF2B39D0062323702C4B19782D48C7
:102C200004F024FFC7E76278002AD1D1A178D2430B
:102C3000D2B29142CCD1244B02221A700123234AF2
:102C40001370234A13800623237023492348FEF779
:102C500005FD234804F06CFFADE76278002AB9D186
:102C6000A178D243D2B29142B4D1FFF78DFF1D4873
:102C700004F05EFF144B01221A7006232370144BDC
:102C800000221A8000F0D4F895E7134601221A704A
:102C9000C1E7152323700D4B1978134804F0E6FEA5
:102CA00089E7094B1B78022B07D0042B83D1064BF5
:102CB00005221A7006230B707DE7034B04221A705D
:102CC00015230B7077E700BF04000020A810002038
:102CD000AA10002078DB00086400020000C8000889
:102CE00048DB00085CDB000890DB0008FFF75AFDBA
:102CF0000B480C490C4A002302E0D458C45004335A
:102D0000C4188C42F9D3094A094C002301E013602E
:102D10000432A242FBD304F033FEFEF70BFE7047F1
:102D2000000000203C0A0020D8E10008400A0020F2
:102D300028A00020FEE7000008B5074A136843F00A
:102D400010031360032000F01BF80F20FFF75EFC58
:102D5000FFF732FC002008BD00200240034A116842
:102D6000034B1B780B441360704700BFAC1000206E
:102D700005000020014B1868704700BFAC10002010
:102D8000074AD36823F4E0631B041B0C000200F421
:102D9000E060034343F0BF6343F40033D360704704
:102DA00000ED00E000B5194BDB68C3F30223C3F16B
:102DB000070CBCF1040F28BF4FF0040C03F1040E04
:102DC000BEF1060F18D9033B4FF0FF3E0EFA0CFC84
:102DD00021EA0C0199400EFA03F322EA0303194396
:102DE00000280BDB0901C9B200F1604000F5614029
:102DF00080F800135DF804FB0023E5E700F00F0006
:102E00000901C9B2024B1954F4E700BF00ED00E01C
:102E100014ED00E0002807DB00F01F024009012349
:102E20009340024A42F82030704700BF00E100E0C2
:102E3000BFF34F8F0549CA6802F4E062044B1343A5
:102E4000CB60BFF34F8F00BFFDE700BF00ED00E098
:102E50000400FA05002808DB00F01F0240090123E6
:102E600093406030014A42F82030704700E100E0B2
:102E700090F82130DBB2022B06D0042383630023B9
:102E800080F82030012070470268136823F00E0399
:102E900013600268136823F001031360036CC16BB5
:102EA000012202FA03F34B6080F82120002380F80E
:102EB000203018467047000008B590F82130DBB28A
:102EC000022B03D004238363012008BD026813682A
:102ED00023F00E0313600268136823F001031360EC
:102EE00003684C4A93424ED9783A934224D0143224
:102EF000934230D0143293422FD0143293422FD0C9
:102F0000143293422FD0143293422FD01432934272
:102F10002FD002F5627293422ED0143293422DD0FC
:102F2000143293422CD01432934202D04FF48032A8
:102F300003E04FF4805200E00122374B5A60012336
:102F400080F82130002380F82030436B002B5ED0C6
:102F500098470020B9E71022EFE74FF48072ECE7C2
:102F60004FF48052E9E74FF48032E6E74FF48012E5
:102F7000E3E74FF08072E0E70122DEE71022DCE7B2
:102F80004FF48072D9E7254A934224D014329342F9
:102F900025D01432934224D01432934224D01432D8
:102FA000934224D01432934224D01432934224D03A
:102FB00002F56272934223D01432934222D014322B
:102FC000934221D01432934202D04FF4803203E076
:102FD0004FF4805200E00122114B5A60AFE71022FB
:102FE000FAE74FF48072F7E74FF48052F4E74FF4BA
:102FF0008032F1E74FF48012EEE74FF08072EBE79A
:103000000122E9E71022E7E74FF48072E4E70020AD
:103010005BE700BF8000024000040240080002405D
:1030200000000240044B0022DA61044A136943F0B5
:103030000103136101807047B0100020002002409E
:10304000194BDB6813F0100305D0184AD36943F01D
:103050000203D3611023144AD26812F0040F06D081
:103060001249CA6942F00102CA6143F004030E4AE0
:10307000D26912F0010F09D00C49CA6942F004026A
:10308000CA610949CA6922F00102CA6140F201120B
:10309000934202D0044AD3607047034AD36923F0B5
:1030A0000103D361704700BF00200240B010002030
:1030B0000A4B1B6913F0800F0BD0084B084A5A606B
:1030C00002F188325A601B6913F0800F03D100208F
:1030D0007047002070470120704700BF0020024069
:1030E00023016745034A136943F0800313610020FD
:1030F000704700BF0020024038B50446FFF73AFE93
:103100000546164BDB6813F0010F0AD0B4F1FF3F00
:10311000F7D024B1FFF72EFE401BA042F1D90320C7
:103120001BE00E4BDB6813F0200F02D00B4B20226C
:10313000DA600A4BDB6813F0100F0BD1074BDB6929
:1031400013F0010F06D1054BDB6813F0040F01D11A
:10315000002002E0FFF774FF012038BD002002408C
:103160002DE9F8431E46244B1B7E012B41D004461B
:103170000F469046204B01221A764CF25030FFF752
:10318000BBFF034678BB012C08D0022C03D04FF0C4
:1031900004091C4607E04FF00209FAE74FF0010965
:1031A000F7E70134E4B24C451DD22101C1F1200200
:1031B000A1F1200328FA01F106FA02F2114326FADE
:1031C00003F3194389B207EB4400FFF72BFF4CF2DE
:1031D0005030FFF791FF094B1D6925F001051D6176
:1031E00003460028DDD0044A002111761846BDE8C8
:1031F000F8830223FAE700BFB0100020002002404D
:10320000064B0022DA61064B1A6942F004021A6189
:103210001A6942F040021A61704700BFB0100020E6
:1032200000200240064B0022DA61064B1A6942F088
:1032300002021A6158611A6942F040021A6170472D
:10324000B010002000200240264B1B7E012B46D0F0
:1032500070B505460E46234B01221A760368022BF1
:1032600020D04CF25030FFF747FF90BB4FF0FF33B8
:103270003360AC680121EA68AB6803EBC223A34268
:1032800028D92046FFF7CEFF4CF25030FFF734FF2D
:10329000154A136923F0020313610146B8B904F516
:1032A0000064E8E74CF25030FFF726FF08B1012137
:1032B00010E00120FFF7A4FF4CF25030FFF71CFF95
:1032C0000146094A136923F00403136102E03460E4
:1032D00000E00121034B00221A76084670BD02214E
:1032E00008467047B01000200020024070B582B040
:1032F0000024A446B0E0874DAA4210D007D9864DDD
:10330000AA420CD005F58035AA4208D013E0A5F5F5
:103310008015AA4203D005F57025AA4207D18A6814
:10332000002A62D0012A5BD04361082403E0A5F59E
:103330008015AA42F3D0BEF1FF0F58D80646BEF161
:10334000FF0F56D84FEA8C0233680F25954023EAC9
:10335000050304FA02F2134333604B6813F0805FF5
:1033600078D06E4B9A6942F001029A619B6903F032
:1033700001030193019B4FEA9C02951C684B53F893
:1033800025600CF003039D000F23AB4026EA0306E3
:10339000644B984233D003F58063984200F09880E4
:1033A00003F58063984200F0958003F580639842AE
:1033B00000F0928003F58063984200F08F8003F55F
:1033C0008063984219D006231AE0CC68B3E7CC6832
:1033D0000434B0E7CC680834ADE7CC680C34AAE715
:1033E00003610824A7E70024A5E70424A3E7061D3A
:1033F000A5E7ACF108029200A6E7052300E0002350
:10340000AB4033430232464D45F822304B6813F44B
:10341000801F65D0444A936843EA0E0393604B686B
:1034200013F4001F62D0404AD36843EA0E03D3600E
:103430004B6813F4003F5FD03B4A536843EA0E03E6
:1034400053604B6813F4803F5CD0374A136843EAFB
:103450000E0313600CF1010C0A6832FA0CF357D01A
:10346000012303FA0CF302EA030E33EA0202F1D15C
:103470004A68122A3FF63FAF122A3FF65CAF01A519
:1034800055F822F01F330008CB330008D53300086D
:10349000E7330008373300083733000837330008B4
:1034A0003733000837330008373300083733000854
:1034B0003733000837330008373300083733000844
:1034C0003733000837330008CF330008DB330008F8
:1034D000012395E7022393E7032391E704238FE772
:1034E000114A936823EA0E03936098E70E4AD36863
:1034F00023EA0E03D3609BE70B4A536823EA0E03CB
:1035000053609EE7084A136823EA0E031360A1E79D
:1035100002B070BD00002210000031100010024007
:103520000000014000080140000401408368194286
:1035300001D001207047002070470AB10161704737
:10354000090401617047C36801EA030221EA03012B
:1035500041EA02410161704782B0084B1B68084A8A
:10356000A2FB03235B0A00FB03F3019300BF019B53
:103570005A1E0192002BF9D102B0704700000020C2
:10358000D34D6210002800F0F18170B582B004467E
:10359000036813F0010F2CD0994B5B6803F00C0308
:1035A000042B1DD0964B5B6803F00C03082B12D044
:1035B0006368B3F5803F41D0002B55D103F18043C0
:1035C00003F504331A6822F480321A601A6822F470
:1035D00080221A6037E08A4B5B6813F4803FE7D0A3
:1035E000874B1B6813F4003F03D06368002B00F087
:1035F000BF81236813F0020F75D0814B5B6813F015
:103600000C0F5FD07E4B5B6803F00C03082B54D08B
:103610002369002B00F08A807A4B01221A60FFF7A1
:10362000A9FB0546764B1B6813F0020F75D1FFF717
:10363000A1FB401B0228F5D903209EE1704A1368C4
:1036400043F480331360636843B3FFF793FB05468D
:103650006B4B1B6813F4003FCBD1FFF78BFB401B78
:103660006428F5D9032088E1B3F5A02F09D0644B75
:103670001A6822F480321A601A6822F480221A60D2
:10368000E1E703F18043A3F53C331A6842F480225A
:103690001A601A6842F480321A60D4E7FFF76AFBB6
:1036A0000546574B1B6813F4003FA2D0FFF762FB9F
:1036B000401B6428F5D903205FE1514B5B6813F48C
:1036C000803FA5D14E4B1B6813F0020F03D0236936
:1036D000012B40F04F814A4A136823F0F8036169D7
:1036E00043EAC1031360236813F0080F33D0A369C2
:1036F000002B5CD0434B0122C3F88024FFF73AFB38
:1037000005463F4B5B6A13F0020F21D1FFF732FBF6
:10371000401B0228F5D903202FE1394A136823F012
:10372000F803616943EAC1031360DCE7354B00220B
:103730001A60FFF71FFB0546314B1B6813F0020FA1
:10374000D1D0FFF717FB401B0228F5D9032014E165
:103750000120FFF701FF236813F0040F00F09680AB
:10376000274BDB6913F0805F34D1254BDA6942F0D7
:103770008052DA61DB6903F080530193019B0125DC
:10378000214B1B6813F4807F26D0E368012B3DD0CA
:10379000002B53D103F1804303F504331A6A22F05E
:1037A00001021A621A6A22F004021A6233E0154B0F
:1037B0000022C3F88024FFF7DDFA0546104B5B6A50
:1037C00013F0020FC7D0FFF7D5FA401B0228F5D936
:1037D0000320D2E00025D3E70B4A136843F480733B
:1037E0001360FFF7C7FA0646074B1B6813F4807F88
:1037F000CBD1FFF7BFFA801B6428F5D90320BCE0CA
:103800000010024000004242007000405F4A136A0C
:1038100043F001031362E36833B3FFF7ABFA0646E4
:103820005A4B1B6A13F0020F2FD1FFF7A3FA801B2C
:1038300041F288339842F3D903209EE0052B09D04A
:10384000524B1A6A22F001021A621A6A22F004022A
:103850001A62E0E74D4B1A6A42F004021A621A6AD1
:1038600042F001021A62D6E7FFF784FA0646474B98
:103870001B6A13F0020F08D0FFF77CFA801B41F29D
:1038800088339842F3D9032077E0E5B9E369002B48
:1038900072D03E4A526802F00C02082A56D0022B1F
:1038A00017D03B4B00221A66FFF764FA0446374BE9
:1038B0001B6813F0007F47D0FFF75CFA001B02285B
:1038C000F5D9032059E0314AD36923F08053D361FD
:1038D000DCE72F4B00221A66FFF74CFA05462B4B0C
:1038E0001B6813F0007F06D0FFF744FA401B022844
:1038F000F5D9032041E0236AB3F5803F1AD023496C
:103900004B6823F47413226A606A024313434B60CA
:103910001F4B01221A66FFF72DFA04461B4B1B684A
:1039200013F0007F0ED1FFF725FA001B0228F5D90E
:10393000032022E0154A536823F40033A1680B43A7
:103940005360DCE7002018E0002016E0012B16D0C1
:103950000E4B5B6803F48031226A914211D103F46B
:103960007013626A93420ED1002006E00120704776
:10397000012002E0012000E0002002B070BD012023
:10398000FBE70120F9E70120F7E700BF0010024044
:10399000000042420F4B5B6803F00C02082A01D082
:1039A0000D487047C3F383420C49885C13F4803F91
:1039B0000BD0084B5B68C3F34043094AD35C064A0B
:1039C00002FB00F0B0FBF3F07047064B03FB00F086
:1039D000704700BF0010024000127A00A8DB000808
:1039E000B8DB000800093D00002800F0A08070B599
:1039F0000D460446524B1B6803F007038B420BD263
:103A00004F4A136823F007030B431360136803F056
:103A100007038B4240F08D80236813F0020F17D00C
:103A200013F0040F04D0474A536843F4E063536033
:103A3000236813F0080F04D0424A536843F46053DC
:103A40005360404A536823F0F003A1680B4353606E
:103A5000236813F0010F31D06368012B20D0022BB3
:103A600025D0384A126812F0020F64D035494A68EE
:103A700022F0030213434B60FFF77CF90646314BFB
:103A80005B6803F00C036268B3EB820F16D0FFF79C
:103A900071F9801B41F288339842F0D9032045E048
:103AA000284A126812F4003FE0D101203EE0254A86
:103AB000126812F0007FD9D1012037E0204B1B683B
:103AC00003F00703AB420AD91D4A136823F007032A
:103AD0002B431360136803F00703AB422DD1236817
:103AE00013F0040F06D0174A536823F4E063E1682B
:103AF0000B435360236813F0080F07D0114A536833
:103B000023F46053216943EAC1035360FFF742FF86
:103B10000C4B5B68C3F303130B4AD35CD8400B4BCD
:103B200018600B4B1868FEF771FD002070BD012076
:103B300070470120FAE70120F8E70120F6E700BF0F
:103B4000002002400010024030DB0008000000208E
:103B500008000020014B1868704700BF00000020DB
:103B600008B5FFF7F7FF044B5B68C3F30223034A72
:103B7000D35CD84008BD00BF0010024040DB000805
:103B800008B5FFF7E7FF044B5B68C3F3C223034AA2
:103B9000D35CD84008BD00BF0010024040DB0008E5
:103BA0000F2303600B4B5A6802F0030242605A680D
:103BB00002F0F00282605A6802F4E062C2605B6860
:103BC000DB0803F4E0630361034B1B6803F00703A6
:103BD0000B607047001002400020024010B4036ADE
:103BE000046A24F001040462846924F0F00C4CEAB5
:103BF000021223F00A030B438261036210BC704778
:103C000010B4036A046A24F010040462846924F482
:103C1000704C4CEA023223F0A00343EA01138261A4
:103C2000036210BC7047836823F070030B4343F0BA
:103C3000070383607047000090F83D30DBB2012B32
:103C40002FD1022380F83D300268D36843F001038E
:103C5000D3600368154A934218D002F5006293427C
:103C600014D0B3F1804F11D0A2F5983293420DD009
:103C700002F58062934209D002F58062934205D03A
:103C80001A6842F001021A60002070479A6802F038
:103C90000702062A07D01A6842F001021A600020C3
:103CA0007047012070470020704700BF002C014082
:103CB000704770477047704770B504460368DE6808
:103CC0001D6915F0020F10D016F0020F0DD06FF025
:103CD00002021A610123037703689B6913F0030F43
:103CE0005ED0FFF7E6FF0023237715F0040F12D014
:103CF00016F0040F0FD023686FF004021A6102233C
:103D0000237723689B6913F4407F4FD02046FFF749
:103D1000D0FF0023237715F0080F12D016F0080FFC
:103D20000FD023686FF008021A61042323772368F9
:103D3000DB6913F0030F40D02046FFF7BAFF0023E2
:103D4000237715F0100F12D016F0100F0FD0236844
:103D50006FF010021A61082323772368DB6913F4DC
:103D6000407F31D02046FFF7A4FF0023237715F0D2
:103D7000010F02D016F0010F2DD115F0800F02D0E7
:103D800016F0800F2FD115F0400F02D016F0400F23
:103D900031D115F0200F02D016F0200F33D170BDB5
:103DA000FFF786FF2046FFF785FF9CE72046FFF7D9
:103DB0007FFF2046FFF77EFFABE72046FFF778FF47
:103DC0002046FFF777FFBAE72046FFF771FF20464E
:103DD000FFF770FFC9E723686FF001021A61204600
:103DE000FDF75EFDC9E723686FF080021A61204687
:103DF00000F05DF9C7E723686FF040021A612046C2
:103E0000FFF759FFC5E723686FF020021A612046CB
:103E100000F04CF9C3E700000368284A904212D032
:103E200002F5006290420ED0B0F1804F0BD0A2F5A7
:103E30009832904207D002F58062904203D002F59A
:103E40008062904203D123F070034A6813431B4AF7
:103E5000904212D002F5006290420ED0B0F1804F35
:103E60000BD0A2F59832904207D002F580629042C2
:103E700003D002F58062904203D123F44073CA68F4
:103E8000134323F080034A69134303608B68C362C2
:103E90000B688362094B984203D003F50063984294
:103EA00001D10B69036301234361036913F0010F1F
:103EB00003D0036923F0010303617047002C014024
:103EC00040B310B5044690F83D30F3B1022384F8B6
:103ED0003D30214651F8040BFFF79EFF012384F883
:103EE000463084F83E3084F83F3084F8403084F81F
:103EF000413084F8423084F8433084F8443084F808
:103F0000453084F83D30002010BD80F83C30FEF78D
:103F100081FCDBE70120704710B4846824F47F4CF7
:103F200042EA03220A4342EA0C02826010BC704754
:103F300090F83C30012B78D010B50446012380F86E
:103F40003C30022380F83D300268936823F47F43BD
:103F500023F0770393600B68602B4CD029D8402B5B
:103F600054D00CD9502B22D1CA6849680068FFF799
:103F700035FE50212068FFF756FE002005E0202B7B
:103F80000DD009D9302B0AD00120012384F83D300F
:103F9000002384F83C3010BD0BB1102B05D119461D
:103FA0002068FFF740FE0020EFE70120EDE7012049
:103FB000EBE7B3F5805F34D0B3F5005F0CD1CB688D
:103FC0004A6889680068FFF7A7FF2268936843F48E
:103FD000804393600020D8E7702B24D1CB684A68D7
:103FE00089680068FFF798FF2268936843F07703B9
:103FF00093600020C9E7CA6849680068FFF700FEBF
:1040000060212068FFF70FFE0020BEE7CA684968FC
:104010000068FFF7E3FD40212068FFF704FE002061
:10402000B3E70020B1E70120AFE7022070470000AE
:1040300090F83C30012B34D010B4012380F83C3090
:10404000022380F83D3003685A689C6822F0700CA7
:104050000A6842EA0C025A600368134A934212D07B
:1040600002F5006293420ED0B3F1804F0BD0A2F55F
:104070009832934207D002F58062934203D002F552
:104080008062934204D124F080044A6814439C6007
:10409000012380F83D30002380F83C30184610BCE6
:1040A00070470220704700BF002C014070477047E6
:1040B000026802F10C0353E8003F23F490730C32C2
:1040C00042E800310029F3D1026802F1140353E8F9
:1040D000003F23F00103143242E800310029F3D1FC
:1040E000036B012B05D0202380F8423000230363AB
:1040F0007047026802F10C0353E8003F23F01003FD
:104100000C3242E800310029F3D1ECE790F841305D
:10411000DBB2212B01D0022070478368B3F5805FAA
:1041200017D0036A5A1C02621A7803685A60C38C5B
:104130009BB2013B9BB2C3844BB90268D36823F0A6
:104140008003D3600268D36843F04003D36000204B
:1041500070470369002BE4D1036A1B880268C3F32C
:1041600008035360036A02330362E0E710B50446B4
:104170000268136923F44053C1680B4313618368D9
:104180000269134342691A430168CB6823F4B053B0
:1041900023F00C031343CB600268536923F440738C
:1041A00081690B4353610268134B9A4220D0FFF799
:1041B000D7FC024602EB820202EB820263689B009C
:1041C000B2FBF3F20D48A0FB02314909642303FB63
:1041D00011231B013233A0FB03235B0903F0F00220
:1041E00002EB011203F00F03216813448B6010BD32
:1041F000FFF7C6FC0246DDE7003801401F85EB51A2
:104200002DE9F04383B005460E4617469946DDF882
:1042100028802C68246836EA04030CBF4FF0010C98
:104220004FF0000CBC4528D1B8F1FF3FF1D0FEF7AC
:10423000A1FDA0EB0900404523D8B8F1000F22D022
:104240002B68DA6812F0040FE3D0802EE1D0402E04
:10425000DFD01A6812F0080FDBD0002401941A682E
:1042600001925B680193019B2846FFF721FF082319
:104270006B6485F84040012000E0002003B0BDE8F9
:10428000F0830320FAE70320F8E760B310B5044693
:1042900090F8413013B3242384F841302268D36866
:1042A00023F40053D3602046FFF760FF22681369B0
:1042B00023F4904313612268536923F02A03536166
:1042C0002268D36843F40053D36000206064202345
:1042D00084F8413084F84230606310BD80F840308B
:1042E000FEF73EFBD7E7012070472DE9F04182B091
:1042F0001E4690F84130DBB2202B56D104460D46C5
:104300009046002955D00AB901204FE000234364AC
:10431000212380F84130FEF72DFD0746A4F82480C4
:10432000A4F82680A368B3F5805F02D04FF00008A0
:1043300014E023692BB34FF000080FE0202384F82A
:104340004130032032E038F8023B2268C3F308030F
:104350005360E28C92B2013A92B2E284E38C9BB257
:1043600093B100963B46002280212046FFF748FF8C
:104370000028E3D1002DE6D015F8012B23685A6000
:10438000E7E7A8460025E9E700963B4600224021E2
:104390002046FFF735FF18B9202384F8413005E0A7
:1043A000202384F84130032000E0022002B0BDE861
:1043B000F0810120FAE72DE9F04182B01E4690F825
:1043C0004230DBB2202B59D104460D4690460029DD
:1043D00058D00AB9012052E000234364222280F819
:1043E00042200363FEF7C6FC0746A4F82C80A4F81D
:1043F0002E80A368B3F5805F02D04FF000081CE068
:10440000236913B14FF0000817E0A846002514E017
:10441000202384F84230032031E023685B68C3F333
:10442000080328F8023B03E023685B682B70013522
:10443000E28D92B2013A92B2E285E38D9BB2C3B1B2
:1044400000963B46002220212046FFF7D9FE002897
:10445000DED1002DE1D0A368B3F5805FE4D013B9BD
:104460002369002BE0D023685B6803F07F032B7087
:10447000DDE7202384F84230002000E0022002B073
:10448000BDE8F0810120FAE7704708B50168CA6805
:1044900022F04002CA60202280F84120FFF7F4FF9A
:1044A000002008BD7047704708B5406A0023C385E7
:1044B000C384FFF7F8FF08BD704790F84230DBB2C5
:1044C000222B69D18368B3F5805F4FD0826AB3F540
:1044D000805F04D0002B56D10369002B53D10368B1
:1044E0005B681370836A01338362C38D9BB2013BA7
:1044F0009BB2C385002B51D100B583B00268D3684D
:1045000023F02003D3600268D36823F48073D36060
:104510000268536923F001035361202380F842307D
:1045200000234363036B012B33D100230363026831
:1045300002F10C0353E8003F23F010030C3242E871
:1045400000310029F3D103681A6812F0100F06D069
:10455000002201921A6801925B680193019B818D90
:10456000FFF7AAFF002003B05DF804FB0269002AF0
:10457000ACD1826A03685B68C3F308031380836A63
:1045800002338362B1E703685B6803F07F03137053
:10459000A8E7FFF787FFE5E7022070470020704794
:1045A00030B583B0044602681368D068516913F0CF
:1045B0000F0505D113F0200F02D010F0200F19D1F4
:1045C0002DB111F0010119D110F4907F16D1216B9A
:1045D00001297DD013F0800F03D010F0800F40F040
:1045E000188113F0400F03D010F0400F40F01581F8
:1045F00003B030BD2046FFF760FFF9E713F0010F6D
:1046000006D010F4807F03D0626C42F00102626435
:1046100013F0040F04D019B1626C42F0020262641C
:1046200013F0020F04D019B1626C42F0040262640C
:1046300013F0080F07D010F0200F00D119B1626CF1
:1046400042F008026264626C002AD1D013F0200F9D
:1046500002D010F0200F29D123685B6903F04003DA
:10466000626C12F0080F00D163B32046FFF720FD03
:1046700023685B6913F0400F20D0226802F1140315
:1046800053E8003F23F04003143242E80031002990
:10469000F3D1E36B73B1634A5A63E06BFEF70CFC32
:1046A0000028A5D0E06B436B9847A1E72046FFF7B1
:1046B00004FFD1E72046FFF7F6FE99E72046FFF713
:1046C000F2FE95E72046FFF7EEFE002363648FE7D6
:1046D00013F0100F3FF47EAF10F0100F3FF47AAFDD
:1046E000002301931368019353680193019B53695D
:1046F00013F0400F51D0E26B13685B689BB2002B44
:104700003FF476AFA18D99427FF672AFE38593694E
:10471000202B37D0226802F10C0353E8003F23F42A
:1047200080730C3242E800310029F3D1226802F193
:10473000140353E8003F23F00103143242E8003130
:104740000029F3D1226802F1140353E8003F23F05B
:104750004003143242E800310029F3D1202384F8C9
:10476000423000232363226802F10C0353E8003F28
:1047700023F010030C3242E800310029F3D1E06B42
:10478000FEF776FB02236363A18DE38D9BB2C91A0A
:1047900089B22046FFF790FE2AE7A18DE38D9BB2F8
:1047A000C91A89B2E38D9BB2002B3FF421AF0029D7
:1047B0003FF41EAF226802F10C0353E8003F23F4DC
:1047C00090730C3242E800300028F3D1226802F1E5
:1047D000140353E8003F23F00103143242E8003091
:1047E0000028F3D1202384F8423000232363226879
:1047F00002F10C0353E8003F23F010030C3242E8AF
:1048000000300028F3D1022363632046FFF754FEF3
:10481000EEE62046FFF77AFCEAE62046FFF735FE93
:10482000E6E600BFA944000808B50A460130014683
:10483000FEF7BAF900B908BD00F0D8F8FBE708B5F3
:104840000B88052B01D0032008BD4378817841EA0D
:104850000321013101231A4689B20330FDF71AFE04
:104860000028F1D000F0C2F8EEE70B88052B22D922
:1048700010B50C464178837843EA0123013399B29D
:10488000C378027942EA032290F805C0531E9BB216
:10489000772B12D85300DBB2634501D0032010BD43
:1048A00001230630FDF7F6FD10B905232380F6E756
:1048B00000F09CF8F3E7032070470320EFE738B5DA
:1048C0000B88052B01D0032038BD0C464378817836
:1048D00041EA0321013189B2C378057945EA03250C
:1048E0006B1E9BB27C2B01D90320EDE700232380B4
:1048F000844603220CF8022B2288013222806A00AF
:1049000042702288013222802A466046FDF7C2FDAD
:1049100020B9238803EB45052580D5E700F066F82C
:10492000D2E7F8B50B88092B45D904460D464378E4
:10493000817841EA032101318EB2C378077947EAD1
:1049400003274379817941EA0321013189B2C3798F
:10495000027A42EA0322407A7B1E9BB27C2B2CD83F
:104960006AB3792A2DD8B0EB420F01D0032023E09F
:10497000012304F10A00FDF78DFD034618B1D8B1FB
:1049800000F034F818E028802046172200F8022BA7
:104990002A8801322A807A0062702A8801322A80AD
:1049A0003A463146FDF776FD0028E8D12B8803EB27
:1049B00047072F80E3E70020F8BD0320FCE7032032
:1049C000FAE70320F8E7000038B50D46054B1C88D0
:1049D000224605490130FBF70BFC01342C800020F6
:1049E00038BD00BFF0100020D0100020012805D0F5
:1049F000072805D008B1042070477047022070478F
:104A00000620704738B50446084601F1FF3C5FFABE
:104A10008CFCBCF1F60F2DD811461A46184B1870B5
:104A20000CB1022527E0174B174D1D60174B184D91
:104A30001D60184B184D1D60184B194D1D60194B0A
:104A400000251D60184B194D1D60194B194D1D6037
:104A5000194B1A4D1D609DF8103000F0E7F805461F
:104A600048B900F043FA40B1154B1C70154B0122B8
:104A70001A7000E00225284638BD0325FBE700BF79
:104A800015110020001100207D4C000804110020A9
:104A90009D4C0008F8100020094D0008F41000207B
:104AA000B54C0008FC100020081100209D4D0008A6
:104AB0000C110020294E000810110020954E00080E
:104AC000F31000200C00002008B5064B1B78012BCA
:104AD00001D0062008BD044B1B6898470020014BFD
:104AE0001870F7E70C0000200011002030B583B0EB
:104AF000364B1C78002C63D10DF1070000F010FA42
:104B0000012802D0204603B030BD9DF80730022BAB
:104B100014D0042BF6D12E4B186801782D4B197048
:104B20002D4B01221A7000230F2B25DC2B4A12F883
:104B300033200AB3914217D00133F5E7284B1B68A5
:104B4000284A23492848984705460028DAD1264BA9
:104B50001B78264A1278934201D0002B32D10420D0
:104B600000F0D0F92C46CDE71C4A02EBC3035B688A
:104B70001C499847184B18701B4B1B7823B3164BD6
:104B80001B789BB1174A00211180124909781048FF
:104B900005684FF0010CA2F800C041F080012970B7
:104BA0000068118801EB0C0515804354104B1B68FD
:104BB0000C4A1288064909680C4800789847A1E712
:104BC00006249FE704469DE71C469BE70C00002057
:104BD0001811002014110020F210002010000020F5
:104BE000F41000201E1100201C11002015110020BF
:104BF000F810002000B5FF2296460AE010F8013BAD
:104C00005340084AD25C82EA0E02074911F803E0D9
:104C100061464B1E1FFA83FC0029EFD142EA0E20A9
:104C20005DF804FBBCDB0008BCDC000870B50D4679
:104C300014461E4600F04AF933460822214628460B
:104C400000F094F9012804D0032400F047F920462D
:104C500070BDB4F5964F0AD864000748B0FBF4F075
:104C600080B200F013FA012803D00324EDE72320DB
:104C7000F6E70024E9E700BFA07F170008B500F0C1
:104C800025F90021044B1970012000F09FF900F074
:104C9000FFF900F023F908BD2011002008B500F04D
:104CA00015F90021084600F091F900F003FA00F030
:104CB00015F908BD70B506460D46144600F006F914
:104CC0000F4B1B889BB2032B04D8052400F006F978
:104CD000204670BD0A4B198889B20A48FFF78AFF3F
:104CE00058B9084A12F8013B3370054B1B889BB238
:104CF000033B23802A600024E8E70524E6E700BFA1
:104D000028120020281100202DE9F04106460C460B
:104D1000154600F0DBF81C4B1B78DBB2012B05D0ED
:104D2000052400F0DBF82046BDE8F081601E174B3B
:104D30001860174F4FF00108A7F8008004F8016CC5
:104D40003A8892B21544ADB23D80398889B2FFF7F6
:104D500051FF3B889BB203EB080292B23A80C2B289
:104D60000C49CA543B889BB203EB080292B23A80CA
:104D7000C0F30720C854084B83F800804146002048
:104D800000F024F90024CCE7201100202411002099
:104D90002A120020281100202111002000B583B024
:104DA0000DF1070000F054F91C4B1B78DBB2032B0C
:104DB00005D8DFE803F0020B1D0800F069F90020B8
:104DC00003B05DF804FB00F063F9F8E7144A002330
:104DD000138013889BB2591C89B211809DF807106B
:104DE000104AD1540D4B02221A7000F051F9E6E737
:104DF0000B4B1B889BB2FF2B0CD809490B889BB22D
:104E00005A1C92B20A809DF80710064AD15400F04D
:104E10003FF9D4E7014B03221A70F8E72011002074
:104E2000281200202811002010B5174B1B7803F022
:104E3000FF0423B1012C07D00024204610BD00211F
:104E4000012000F0C3F8F8E7104B1B889BB27BB140
:104E50000F4C2368187800F0E7F8236801332360CB
:104E60000A4A13889BB2013B9BB213800024E4E7FB
:104E7000082000F047F804460021012000F0A6F8C1
:104E8000014B00221A70D8E7211100202A120020BD
:104E90002411002010B50C4B1B785BB103F0FF020E
:104EA000022A0CD0002400F005F9074B01221A70E9
:104EB000204610BD012000F025F80446F3E702204B
:104EC00000F020F80446EEE72011002008B500F0BD
:104ED0005FF9014B186008BD2C12002008B5024B89
:104EE000186800F07DF908BD2C12002008B50020DC
:104EF00000F048FA024B1860003818BF012008BDC6
:104F00003012002008B50146044B186820B100F0AB
:104F10006DFAC043C00F08BD0020FCE7301200202E
:104F200010B504464FF0FF3300220F210E480068F1
:104F300000F09AFA431E072B14D8DFE803F00407A9
:104F4000130B1313130F012020700CE002232370A6
:104F5000012008E004232370012004E008232370CB
:104F6000012000E0002010BD3012002008B51648D6
:104F70004160082A0CD04FF48051134A91600021FF
:104F8000D160012B12D0022B15D01BB1002008BD1F
:104F90000021F2E711610C480C2343610023836177
:104FA000C361FFF772F958B90120F0E7064B4FF4DF
:104FB000C0621A61EFE7044B4FF480621A61EAE7BE
:104FC000FCF782FC0020E2E71810002010B50C4628
:104FD00090B1002204211248FEF7AFFA114B1A6873
:104FE000D36843F02003D36094B10E4B1A68D368A2
:104FF00043F08003D36010BD012204210848FEF76E
:105000009CFA084B1A68D36823F02003D360EBE7BF
:10501000044B1A68D36823F08003D360EBE700BF2A
:10502000000C01401810002000B583B08DF8070077
:1050300001231A460DF107010448FFF756F918B18C
:10504000002003B05DF804FB0120FAE718100020EF
:1050500008B5014601231A460348FFF7ACF908B129
:10506000002008BD0120FCE71810002008B5024B05
:105070001B68984708BD00BF0C11002008B5024B03
:105080001B68984708BD00BF081100200120704729
:10509000074B1B686FF001021A61DA6842F00102E7
:1050A000DA6000225A621A6842F001021A60704700
:1050B000400F00200D4B1B68196A41F2111211427A
:1050C00008D1196A40F24442114203D11A6822F011
:1050D00001021A60054B1B6800225A62DA6822F04E
:1050E0000102DA606FF001021A617047400F002080
:1050F00008B5024B1B68984708BD00BF101100207F
:10510000EFF3058393B9EFF3108393B90C4B186851
:10511000022804D080B90A4B01221A607047EFF3CD
:105120001183002BF6D06FF0050070476FF005007B
:1051300070476FF0050070474FF0FF30704700BFB9
:10514000C018002008B5EFF30583B3B9EFF310835F
:10515000B3B90E4B1B68022B08D0012B13D10B4B9C
:1051600002221A6001F094FD002008BDEFF31182C5
:10517000002AF2D06FF00500F7E76FF00500F4E7C2
:105180006FF00500F1E74FF0FF30EEE7C0180020A8
:1051900008B5EFF3058393B9EFF3108393B90F4B81
:1051A0001B68022B02D1EFF3118373B902F096F85A
:1051B00070B102280ED101F0C1FD00200CE06FF0AB
:1051C000050009E06FF0050006E06FF0050003E060
:1051D000012001E04FF0FF3008BD00BFC0180020E3
:1051E00010B5EFF3058313BB0446EFF310830BBB3D
:1051F000164B1B68022B02D1EFF31183EBB902F0BF
:105200006DF808B102281BD1012C06D0DCB901F0E1
:105210002FFE012804D1204610BD01F08FFDFAE7D2
:1052200002F05CF80228F6D04FF0FF34F3E76FF09D
:105230000504F0E76FF00504EDE76FF00504EAE719
:105240004FF0FF34E7E74FF0FF34E4E7C0180020E9
:10525000F0B587B000240494EFF30584002C44D10A
:10526000EFF31083002B40D1344B1B68022B16D078
:1052700000283AD000238DF817306AB3156895B12D
:10528000936903B918235C1E372C52D8546814F064
:10529000010F50D156694EB14FEA960C08E0EFF37A
:1052A000118313BBE4E70DF11705E9E74FF0800C1C
:1052B000946834B1D768B7F5916F02D3176907B115
:1052C000B6B914B14FF0FF340CE0D46894B9146946
:1052D0009CB14FF0FF3405E0002418234FF0800C00
:1052E0000DF11705012C0AD0ACB1049807B0F0BD40
:1052F0000124F7E74FF0FF34F4E70024F2E71469E4
:1053000092680292019400930B466246294601F08E
:105310004DFC0490E9E704AA019200930B461FFAA2
:105320008CF2294601F07FFC0128DED00023049393
:10533000DBE70020DAE70020D8E700BFC018002034
:1053400008B5EFF30583A3B9EFF31083A3B90C4BB2
:105350001B68022B02D040B9002008BDEFF3118377
:10536000002BF8D06FF00500F7E701F0FDFD0020FD
:10537000F3E76FF00500F0E76FF00500EDE700BF21
:10538000C018002008B5EFF3058333BBEFF310839B
:105390002BBB154B1B68022B0CD0D0B1836813B10B
:1053A000C2681F2A11D85BB14FF0FF33CBB900F0B0
:1053B000CEF913E0EFF31183002BEED000200DE0C7
:1053C000C36843B14FF0FF33F0E7184600F09AF995
:1053D00004E00023EAE70023E8E7002008BD0020FE
:1053E000FCE70020FAE700BFC018002070B310B53A
:1053F00082B00C46034611F07F4F2AD1EFF30582AD
:105400004AB9EFF3108232B9164A1268022A18D14B
:10541000EFF31182AAB10022019201AA2146184697
:1054200000F072FAC8B9019BD3B14FF0E0234FF0FE
:105430008052C3F8042DBFF34F8FBFF36F8F204608
:1054400009E02146184600F014FA04E06FF003006A
:1054500070476FF0030002B010BD6FF00200FAE772
:105460002046F8E7C0180020B0B370B582B00C46F3
:105470001D46844611F07F4F31D1EFF3058393BB76
:10548000EFF3108393BB1E4B1B68022B13D012F05B
:10549000010617D0012312F0020F15D0002200954B
:1054A0002146604600F061F986B1844219D005B307
:1054B0006FF0010015E0EFF31183002BE7D06FF0E0
:1054C00005000EE00023E6E70122E8E7044208D1E8
:1054D00095B16FF0010004E06FF0030070476FF0CA
:1054E000030002B070BD6FF00500FAE76FF0050031
:1054F000F7E76FF00200F4E76FF00200F1E700BF9A
:10550000C018002070B5EFF30583002B4ED1044680
:10551000EFF310821346002A4BD1284A1268022A60
:1055200023D004B1636813F0010600D0012613F004
:10553000080F40D17CB3A16811B1E3684F2B1FD88D
:10554000C9B14FF0FF337BBB4EB3042000F0F1FE36
:1055500005462DB104B124682146284601F02CF9F6
:105560002DB326B345F0010521E0EFF31182002AA7
:10557000D7D000251BE0E3687BB14FF0FF33E2E7B3
:1055800026B1042000F0E0FE0546E2E7012000F02D
:10559000DBFE0546DDE70023D5E70023D3E7012046
:1055A00000F0C7FE0546D4E70025D9E700252846C8
:1055B00070BD0025FBE70025F9E700BFC0180020FB
:1055C000EFF3058242BB10B503460C4620F0010004
:1055D00003F00103EFF310820ABB194A1268022A92
:1055E0000AD0F8B17BB1214601F0C6F801281CD0E1
:1055F000ECB16FF0010019E0EFF31182002AF0D056
:105600006FF0050012E0214600F0E3FF012811D001
:1056100094B16FF0010009E06FF0050070476FF082
:10562000050003E06FF0030000E0002010BD6FF004
:105630000200FBE70020F9E76FF00200F6E700BF89
:10564000C0180020EFF3058222BB08B5034620F006
:10565000010003F00103EFF31082F2B9154A12685A
:10566000022A07D0E0B163B100F07DFE01281AD113
:10567000002008BDEFF31182002AF3D06FF005007F
:10568000F7E700231A46194600F083FD01280DD1E3
:105690000020EEE76FF0050070476FF00500E8E7C7
:1056A0006FF00300E5E76FF00200E2E76FF0020041
:1056B000DFE700BFC0180020034B0360034B0B6003
:1056C00080231360704700BF38140020341200207C
:1056D000034B0360034B0B604FF480731360704700
:1056E000C81C0020C41800201AB9084206D1104670
:1056F000704731EA000303D0002070470120704753
:105700000120704780B110B582B004462023019378
:10571000019B202B11D04FF0500383F31188BFF36E
:105720006F8FBFF34F8FFEE74FF0500383F3118865
:10573000BFF36F8FBFF34F8FFEE7002340F8043BAA
:1057400000F0ECF801232377204602B010BD38B5F5
:10575000202000F0F9FA044628B1002540F8045B47
:1057600000F0DCF82577204638BD2DE9F84378B104
:105770000C4616461D46074611F07F4811D04FF0E3
:10578000500383F31188BFF36F8FBFF34F8FFEE792
:105790004FF0500383F31188BFF36F8FBFF34F8F28
:1057A000FEE741B94FF0500383F31188BFF36F8FC9
:1057B000BFF34F8FFEE701F091FD50B9089B43B155
:1057C0004FF0500383F31188BFF36F8FBFF34F8FF8
:1057D000FEE701F0B3FAD7F800902A462146484682
:1057E000FFF782FFF0B116B129EA04033B6001F034
:1057F0003FFBB8F1000F12D048B94FF0E0234FF053
:105800008052C3F8042DBFF34F8FBFF36F8F01F0A9
:1058100059FE814610F0007F1AD029F07F49484692
:10582000BDE8F883089B83B166B941460DB141F0EC
:105830008061089A2143381D01F024FCC146DDF83F
:105840002080D4E74FF08071F0E7DDF82080CEE7CC
:1058500000F000F9D7F800902A4621464846FFF7A5
:1058600043FF18B116B129EA04043C6000F014F9B2
:10587000D3E7F8B568B10D46044611F07F4711D063
:105880004FF0500383F31188BFF36F8FBFF34F8F37
:10589000FEE74FF0500383F31188BFF36F8FBFF320
:1058A0004F8FFEE700F10C0601F048FA20692368EB
:1058B0002B4323600AE0216832EA010105D111E09F
:1058C000216841F0007101F06BFC2846B0420ED017
:1058D0004568036823F07F4213F0806FEBD12168A5
:1058E0001142F2D013F0807FEAD01743E8E7236833
:1058F00023EA0703236001F0BBFA2068F8BD08B56E
:10590000FFF7B7FF08BD000008B513460A46014679
:10591000014802F01BF808BDFF58000800F1080319
:1059200043604FF0FF328260C36003610023036075
:10593000704700230361704743684B609A688A6030
:10594000516099600861036801330360704730B4A7
:105950000D68B5F1FF3F11D000F108031C465B68EC
:105960001A68AA42FAD963684B6099608C606160DA
:10597000086103680133036030BC70470469F2E7D3
:105980000369416882688A60416851605A6882424E
:1059900006D0002202611A68013A1A60186870473E
:1059A00082685A60F5E7000082B0002301930D4B36
:1059B0001B68B3F1FF3F08D04FF0500383F3118809
:1059C000BFF36F8FBFF34F8FFEE74FF0500383F3AA
:1059D0001188BFF36F8FBFF34F8F019B002BFCD05B
:1059E00002B070479000002006480068006880F30D
:1059F000088862B661B6BFF34F8FBFF36F8F00DFC9
:105A000000BF000008ED00E04FF0807340F8043C58
:105A100021F0010140F8081C034B40F80C3C40F811
:105A2000202C4038704700BFA95900080000000032
:105A3000074B19680868B0E8F00F80F30988BFF3D6
:105A40006F8F4FF0000080F311884EF00D0E7047FD
:105A5000B89900204FF0500383F31188BFF36F8F84
:105A6000BFF34F8F0B4A136801331360012B00D033
:105A700070474FF0E023D3F8043D13F0FF0FF7D049
:105A80004FF0500383F31188BFF36F8FBFF34F8F35
:105A9000FEE700BF90000020094B1B6843B94FF0A0
:105AA000500383F31188BFF36F8FBFF34F8FFEE76F
:105AB000013B034A13600BB983F31188704700BFA1
:105AC0009000002000000000000000000000000026
:105AD000EFF30980BFF36F8F0D4B1A6820E9F00FC9
:105AE00010602DE908404FF0500080F3118801F05C
:105AF00061FA4FF0000080F31188BDE80840196892
:105B00000868B0E8F00F80F30988BFF36F8F704723
:105B1000B899002008B54FF0500383F31188BFF304
:105B20006F8FBFF34F8F01F017F928B14FF0E023CB
:105B30004FF08052C3F8042D002383F3118808BD71
:105B40004FF0E022002313619361054B1B68054968
:105B5000A1FB03139B09013B5361072313617047AA
:105B600000000020D34D621010B582B02A4B1A7885
:105B7000D2B20192FF221A701B78DBB28DF803308B
:105B80009DF8033003F05003244A1370244B07227E
:105B90001A6009E0224A1368013B13609DF8033044
:105BA0005B00DBB28DF803309DF8033013F0800FFB
:105BB000F0D11B4B1B68032B08D04FF0500383F32D
:105BC0001188BFF36F8FBFF34F8FFEE71B02144A9C
:105BD000136003F4E0631360019BDBB20E4A1370A1
:105BE0004FF0E023D3F8202D42F47002C3F8202DAB
:105BF000D3F8202D42F07042C3F8202DFFF7A0FF0C
:105C00000024084B1C60FFF7EFFE01F0D3F9FFF70B
:105C1000CBFE204602B010BD00E400E05021002081
:105C20005421002090000020EFF305830F2B0FD9A3
:105C3000114A9B5CDBB2114A12789A4208D94FF0A4
:105C4000500383F31188BFF36F8FBFF34F8FFEE7CD
:105C50004FF0E023D3F80C3D03F4E063084A1268E8
:105C6000934208D94FF0500383F31188BFF36F8F2D
:105C7000BFF34F8FFEE77047F0E300E050210020B4
:105C800054210020124A12F0070F1ED0D11D21F01E
:105C90000701C1F5F04313440A460E480260002193
:105CA00041601344083B23F007030B48036059602D
:105CB0001960991A51601360084B1960084B1960FC
:105CC000084B4FF000421A6070474FF4F043E4E78E
:105CD0005C21002070990020582100206499002048
:105CE000609900205C990020154B1A461B6883427E
:105CF000FBD3516802EB010C844509D0416800EBED
:105D0000010C634509D00360904218D010607047C1
:105D10004068014451601046F0E710B4094C246813
:105D2000A3420AD05B681944416013681B68036092
:105D3000904200D0106010BC70470460F8E77047D4
:105D4000709900205821002070B5054600F0F6FF3C
:105D5000364B1B68A3B1364B1B681D424ED135B183
:105D6000083515F0070F02D025F007050835002D7E
:105D700046D0304B1B68AB4251D32F4A146804E025
:105D8000FFF780FFE7E722461C466368AB4202D27A
:105D90002368002BF7D1254B1B68A34241D016681E
:105DA00008362368136063685B1B102B10D96019D9
:105DB00010F0070F08D04FF0500383F31188BFF3A2
:105DC0006F8FBFF34F8FFEE743606560FFF78CFF77
:105DD000626818490B689B1A0B60184909688B4266
:105DE00001D216490B60124B1B68134363600023FA
:105DF0002360134A13680133136002E0002600E0B9
:105E0000002601F035F816F0070F0CD04FF05003C4
:105E100083F31188BFF36F8FBFF34F8FFEE7002628
:105E2000EFE70026EDE7304670BD00BF58210020A7
:105E30005C990020609900207099002064990020EE
:105E400068990020002834D038B50446A0F1080530
:105E500050F8043C174A1268134208D14FF050031F
:105E600083F31188BFF36F8FBFF34F8FFEE750F8B6
:105E7000081C41B14FF0500383F31188BFF36F8FBB
:105E8000BFF34F8FFEE723EA020340F8043C00F023
:105E900055FF54F8041C084A13680B441360284645
:105EA000FFF722FF054A13680133136000F0E0FF9B
:105EB00038BD70475C990020609900206C990020E3
:105EC0000346406A18B11B6B1868C0F13800704770
:105ED00010B50446FFF7BEFDA26BE36B9A4204D0F7
:105EE0000024FFF7D9FD204610BD0124F9E710B5C5
:105EF0000446FFF7AFFDA36B23B90124FFF7CCFDE8
:105F0000204610BD0024F9E770B504461546866B9F
:105F1000026C5AB903681BB100200136A66370BD3C
:105F2000806801F037FA0023A360F6E76DB9406896
:105F3000FAF75EF9226C636813446360A2689342C7
:105F400019D3236863602846E7E7C068FAF750F979
:105F5000226C5142E3689B1AE3602268934202D2AA
:105F6000A3680B44E360022D01D00020D5E726B1E1
:105F7000013E0020D1E72846CFE70020CDE708B555
:105F80000346026C62B10846D9681144D960D3F85F
:105F900008C0614501D31968D960D968FAF728F9B2
:105FA00008BD38B50546FFF755FD95F8454064B284
:105FB00001E0013C64B2002C0ADD6B6A43B105F1DB
:105FC000240001F0A7F80028F3D001F07BF9F0E7F6
:105FD000FF2385F84530FFF75FFDFFF73BFD95F8A0
:105FE000444064B201E0013C64B2002C0ADD2B693C
:105FF00043B105F1100001F08DF80028F3D001F055
:1060000061F9F0E7FF2385F84430FFF745FD38BD1F
:1060100038B5E0B10D460446FFF71CFD2368E26B7E
:10602000216C01FB0230A0600020A0636360013A94
:1060300002FB0133E360FF2384F8443084F84530E9
:10604000FDB9236963B9FFF727FD012038BD4FF083
:10605000500383F31188BFF36F8FBFF34F8FFEE7B9
:1060600004F1100001F056F80028ECD04FF0E023C6
:106070004FF08052C3F8042DBFF34F8FBFF36F8FE3
:10608000E1E704F11000FFF749FC04F12400FFF7F9
:1060900045FCD8E738B51D46049C0B4649B9246039
:1060A000E063236401212046FFF7B2FF84F84C50DF
:1060B00038BD2260F4E740B94FF0500383F31188F4
:1060C000BFF36F8FBFF34F8FFEE710B584B01C4650
:1060D000844653B192B189B94FF0500383F31188CC
:1060E000BFF36F8FBFF34F8FFEE74FF0500383F383
:1060F0001188BFF36F8FBFF34F8FFEE76AB1502354
:106100000393039B502B13D04FF0500383F311885C
:10611000BFF36F8FBFF34F8FFEE70029EFD04FF033
:10612000500383F31188BFF36F8FBFF34F8FFEE7E8
:10613000039B012384F8463000949DF81830604694
:10614000FFF7A8FF204604B010BD40B94FF0500340
:1061500083F31188BFF36F8FBFF34F8FFEE7F0B566
:1061600083B00D461446064601FB00F05030FFF7A1
:10617000EBFD074650B1002380F8463000902346DF
:1061800000F1500229463046FFF784FF384603B03D
:10619000F0BDF0B585B0019288B10F461D460446AA
:1061A000B1B1022D20D1E36B012B1DD04FF0500374
:1061B00083F31188BFF36F8FBFF34F8FFEE74FF06C
:1061C000500383F31188BFF36F8FBFF34F8FFEE748
:1061D000036C002BE5D04FF0500383F31188BFF31D
:1061E0006F8FBFF34F8FFEE701F078F8064658B97E
:1061F000019B002B48D04FF0500383F31188BFF36D
:106200006F8FBFF34F8FFEE700263DE02A463946E9
:106210002046FFF779FE636A7BB948B14FF0E0236F
:106220004FF08052C3F8042DBFF34F8FBFF36F8F31
:10623000FFF732FC012005B0F0BD04F1240000F0AE
:1062400069FF0028F4D04FF0E0234FF08052C3F8EC
:10625000042DBFF34F8FBFF36F8FE9E7FFF71CFCEF
:106260000020E8E702A800F0DFFF012619E0002384
:1062700084F8443021E0002384F8453023E02046B0
:10628000FFF78FFE00F0F4FDFFF7E4FBA26BE36B7A
:106290009A42BBD3022DB9D0019B002BDED0002E39
:1062A000E0D0FFF7F9FB00F049FDFFF7D3FB94F8CE
:1062B000442052B2B2F1FF3FD9D094F8452052B2F7
:1062C000B2F1FF3FD7D0FFF7E7FB01A902A800F02A
:1062D000B7FFD8B92046FFF7FBFD0028CFD00199C2
:1062E00004F1100000F0B6FE2046FFF75AFE00F061
:1062F000BFFD0028C8D14FF0E0234FF08052C3F813
:10630000042DBFF34F8FBFF36F8FBDE72046FFF71C
:1063100048FE00F0ADFD00208DE748B108B5002132
:1063200081600160C1600B460A46FFF732FF08BD7D
:10633000704710B5024600210120FFF706FF044612
:10634000FFF7EBFF204610BD10B582B00B46009062
:10635000002211460120FFF7AEFE0446FFF7DDFFE5
:10636000204602B010BD38B538B10446856800F04B
:10637000AFFF85420AD0002038BD4FF0500383F3B1
:106380001188BFF36F8FBFF34F8FFEE7E368013BC8
:10639000E3600BB10120EFE71A4619462046FFF7EC
:1063A000F8FE0120E8E72DE9F84390B10F461646C4
:1063B0001C460546B1B1022C20D1EB6B012B1DD040
:1063C0004FF0500383F31188BFF36F8FBFF34F8FEC
:1063D000FEE74FF0500383F31188BFF36F8FBFF3D5
:1063E0004F8FFEE7036C002BE5D04FF0500383F393
:1063F0001188BFF36F8FBFF34F8FFEE7FFF714FCD9
:10640000EFF311894FF0500383F31188BFF36F8FBF
:10641000BFF34F8FAA6BEB6B9A4206D3022C04D0CA
:10642000002089F31188BDE8F88395F845804FFA7C
:1064300088F8AB6B224639462846FFF765FDB8F170
:10644000FF3F06D008F101035BB285F8453001201B
:10645000E7E76B6A0BB90120E3E705F1240000F0E0
:1064600059FE18B126B101203060DAE70120D8E7E3
:106470000120D6E7F0B585B0019290B10F460446F1
:10648000C1B100F02BFF064600BB019B002B5ED084
:106490004FF0500383F31188BFF36F8FBFF34F8F1B
:1064A000FEE74FF0500383F31188BFF36F8FBFF304
:1064B0004F8FFEE7036C002BE3D04FF0500383F3C4
:1064C0001188BFF36F8FBFF34F8FFEE700263EE0CA
:1064D00039462046FFF753FD013DA563236923B9E3
:1064E000FFF7DAFA012005B0F0BD04F1100000F06A
:1064F00011FE0028F4D04FF0E0234FF08052C3F893
:10650000042DBFF34F8FBFF36F8FE9E7FFF7C4FA96
:106510000020E8E702A800F087FE012621E0002322
:1065200084F8443029E0002384F845302BE02046ED
:10653000FFF737FD00F09CFC09E02046FFF731FD36
:1065400000F096FC2046FFF7D2FC00283FD1FFF771
:1065500081FAA56B002DBBD1019B002BD6D0002E5C
:10656000D8D0FFF799FA00F0E9FBFFF773FA94F837
:1065700044305BB2B3F1FF3FD1D094F845305BB209
:10658000B3F1FF3FCFD0FFF787FA01A902A800F0CF
:1065900057FE0028D1D12046FFF7A9FC0028C6D01D
:1065A000019904F1240000F055FD2046FFF7F9FCA5
:1065B00000F05EFC0028CAD14FF0E0234FF080527B
:1065C000C3F8042DBFF34F8FBFF36F8FBFE70020D9
:1065D00089E770B584B0019158B10446036C8BB162
:1065E0004FF0500383F31188BFF36F8FBFF34F8FCA
:1065F000FEE74FF0500383F31188BFF36F8FBFF3B3
:106600004F8FFEE700F06AFE054650B9019B5BB173
:106610004FF0500383F31188BFF36F8FBFF34F8F99
:10662000FEE70026354655E0064653E0013BA363EE
:1066300023683BB123694BB9FFF72EFA0126304698
:1066400004B070BD00F04AFFA060F3E704F1100051
:1066500000F060FD0028EFD04FF0E0234FF08052B3
:10666000C3F8042DBFF34F8FBFF36F8FE4E746B13C
:106670004FF0500383F31188BFF36F8FBFF34F8F39
:10668000FEE7FFF709FADAE702A800F0CDFD0125E1
:106690002AE0002384F8443032E0002384F84530B7
:1066A00034E0FFF7D7F9A06800F028FE0646FFF7B0
:1066B000F3F93BE02046FFF774FC00F0D9FB09E05A
:1066C0002046FFF76EFC00F0D3FB2046FFF70FFCDF
:1066D000002842D1FFF7BEF9A36B002BA6D1019B86
:1066E000002BC4D0002DCFD0FFF7D6F900F026FB49
:1066F000FFF7B0F994F844305BB2B3F1FF3FC8D074
:1067000094F845305BB2B3F1FF3FC6D0FFF7C4F950
:1067100001A902A800F094FD0028D1D12046FFF77E
:10672000E6FB0028C6D02368002BBAD0019904F1FB
:10673000240000F08FFC2046FFF733FC00F098FBAC
:106740000028C7D14FF0E0234FF08052C3F8042D4A
:10675000BFF34F8FBFF36F8FBCE70EB900266EE714
:10676000FFF778F92046FFF7ABFB0146A06800F081
:1067700059FEFFF791F9F1E780B170B50C46054677
:10678000866800F0A5FD864211D021462846FFF715
:1067900020FF80B1EB680133EB600CE04FF0500359
:1067A00083F31188BFF36F8FBFF34F8FFEE7EB6862
:1067B0000133EB60012070BD0023072B0CD8074A82
:1067C00052F833200AB10133F7E7044A42F8331094
:1067D00002EBC30358607047704700BF78990020F0
:1067E00070B504460D461646FFF734F994F8443068
:1067F0005BB2B3F1FF3F0DD094F845305BB2B3F11B
:10680000FF3F0BD0FFF748F9A36B5BB12046FFF7C2
:10681000C8FB70BD002384F84430EDE7002384F802
:106820004530EFE73246294604F1240000F056FCDB
:10683000ECE70000084B1B681B6823B9074B4FF0BF
:10684000FF321A607047044B1B68DB68DB685A68CC
:10685000024B1A60704700BFBC990020649E002064
:106860002DE9F04780460D4617469946089EDDF80B
:1068700024A00A9C9200A521206B01F0A5F8236BAF
:1068800007F18042013A03EB820727F00707002D4A
:1068900065D04FF0000CBCF10F0F0BD815F80C2091
:1068A00004EB0C0383F8342015F80C3013B10CF111
:1068B000010CF0E7002384F84330372E00D9372647
:1068C000E662E66400252565201DFFF732F804F135
:1068D0001800FFF72EF82461C6F13806A66164623D
:1068E000C4F8805484F884544FF48562294604F136
:1068F000580001F069F804F55173E36504F56B7312
:10690000236604F21443636601220023C4E9402392
:1069100043F20E33A4F808314AF6CD33A4F80A3115
:1069200041F23423A4F80C314EF26D63A4F80E3119
:106930004DF6EC63A4F810310523A4F812310B23B3
:10694000A4F814314A4641463846FFF75DF8206006
:10695000BAF1000F01D0CAF80040BDE8F08700236B
:1069600084F83430A9E7000038B5002407E004EBD0
:10697000840293000E481844FEF7D0FF0134372CF0
:10698000F5D90C4D2846FEF7C9FF0B4C2046FEF703
:10699000C5FF0A48FEF7C2FF0948FEF7BFFF0948D6
:1069A000FEF7BCFF084B1D60084B1C6038BD00BFE4
:1069B000C4990020389E00204C9E0020709E00202C
:1069C0009C9E0020889E0020BC990020C099002039
:1069D00010B50446FFF73EF8224A136801331360EE
:1069E000214B1B685BB1214B1B686BB91E4B1B68AD
:1069F000DA6AE36A9A4207D81B4B1C6004E01A4B20
:106A00001C601368012B29D0194A136801331360E5
:106A10006364E06A174B1B68984201D9154B1860F4
:106A200000EB8000211D144B03EB8000FEF784FF78
:106A3000FFF732F80D4B1B687BB10B4B1B68DA6A12
:106A4000E36A9A4209D24FF0E0234FF08052C3F834
:106A5000042DBFF34F8FBFF36F8F10BDFFF784FF7F
:106A6000D2E700BF249E0020B8990020849E002019
:106A7000309E0020349E0020C499002010B50446AA
:106A8000583001F081F894F8853463B1012B11D0AE
:106A9000022B0ED04FF0500383F31188BFF36F8F9A
:106AA000BFF34F8FFEE7206BFFF7CCF92046FFF7CF
:106AB000C9F910BD2046FFF7C5F9FAE70F4B1B686F
:106AC000D3B110B5FEF7C6FF0D4BDB68DC68201DA7
:106AD000FEF756FF0B4A1368013B1360074A136821
:106AE000013B1360FEF7D8FF2046FFF7C7FF034BBB
:106AF0001B68002BE6D110BD704700BF289E002008
:106B00009C9E0020249E002008B5FFF7D7FF074B6E
:106B10001B68012BF9D94FF0E0234FF08052C3F8E6
:106B2000042DBFF34F8FBFF36F8FEEE7C4990020A2
:106B300070B504460D46174B1E68174B1868043095
:106B4000FEF71EFFB4F1FF3F0DD03444124B1B681B
:106B50005C60A64210D9114B18680F4B19680431BC
:106B6000FEF7F5FE70BD002DEFD00B4B1968043118
:106B70000B48FEF7E1FEF5E70A4B1868064B19686B
:106B80000431FEF7E4FE084B1B68A342EAD9064B2A
:106B90001C60E7E7B09E0020B8990020C099002053
:106BA000889E0020BC990020649E002030B587B0EC
:106BB0000B9C8CB10C9DC5B14FF491650495049D5F
:106BC000B5F5916F1AD04FF0500383F31188BFF3DE
:106BD0006F8FBFF34F8FFEE74FF0500383F31188A1
:106BE000BFF36F8FBFF34F8FFEE74FF0500383F378
:106BF0001188BFF36F8FBFF34F8FFEE7049D0C9D8D
:106C00002C63022485F8854400240394029505AC86
:106C100001940A9C0094FFF723FE0C98FFF7D8FE1E
:106C2000059807B030BD2DE9F04385B0074688468A
:106C300014461E469000FFF787F808B381464FF4CC
:106C40009160FFF781F80546B0B1C0F83090E5B12A
:106C5000002385F88534039302950D9B01930C9BCB
:106C600000933346224641463846FFF7F9FD284651
:106C7000FFF7AEFE012005E04846FFF7E3F8E6E740
:106C80004FF0FF3005B0BDE8F0834FF0FF30F9E77B
:106C900010B588B000240594069407AA06A905A893
:106CA000FEF70AFD059B0293069B01930094234681
:106CB000079A1A491A48FFF779FF1A4B186040B132
:106CC00000F086FC012806D0B0F1FF3F1DD008B0CF
:106CD00010BD0020F6E74FF0500383F31188BFF397
:106CE0006F8FBFF34F8F104B1B6858330F4A1360E1
:106CF0000F4B4FF0FF321A600E4B01221A600E4B01
:106D000000221A60FEF730FFE1E74FF0500383F3F3
:106D10001188BFF36F8FBFF34F8FFEE7BCDD000814
:106D2000096B0008609E0020B899002094000020A4
:106D3000649E0020849E0020B09E0020024A1368BA
:106D400001331360704700BF2C9E0020014B186870
:106D5000704700BFB09E0020F8B53A4B1B68002B6F
:106D600069D1394B1D6801351D60C5B9374B1B68AA
:106D70001B6843B14FF0500383F31188BFF36F8F4B
:106D8000BFF34F8FFEE7314A1168314B186810602E
:106D90001960304A136801331360FFF74BFD2E4B27
:106DA0001B68AB423DD900272C4B1B68DB6A03EB09
:106DB00083039A002A4B9B58012B00D90127294BAA
:106DC0001B68002B3CD001273AE001271F4B1B68B2
:106DD0001B6843B31D4B1B68DB68DC6863689D421E
:106DE00026D3261D3046FEF7CBFDA36A1BB104F166
:106DF0001800FEF7C5FDE36A1B4A1268934201D9E9
:106E0000194A136003EB83039A0031461448104477
:106E1000FEF792FDE26A114B1B68DB6A9A42D4D2FC
:106E2000D4E70027D2E70C4B4FF0FF321A60BBE7E4
:106E3000094A1360B8E70D4A13680133136000274D
:106E40003846F8BD2C9E0020B09E0020BC99002042
:106E5000C0990020689E0020649E0020B899002000
:106E6000C4990020B49E0020349E00206C9E002017
:106E700038B5354B1B6843B94FF0500383F3118885
:106E8000BFF36F8FBFF34F8FFEE7FEF7E3FD2E4B8F
:106E90001A68013A1A601B68002B4FD12B4B1B68F4
:106EA0000BB900244BE00024294B1B681BB3284B73
:106EB000DB68DC6804F11800FEF762FD251D28463A
:106EC000FEF75EFDE06A234B1B68984201D9214B17
:106ED000186000EB800029461F4B03EB8000FEF793
:106EE0002BFDE26A1D4B1B68DB6A9A42DCD31C4B0C
:106EF00001221A60D8E70CB1FFF79CFC194B1C6803
:106F000084B9174B1C68D4B14FF0E0234FF0805286
:106F1000C3F8042DBFF34F8FBFF36F8F01240EE032
:106F2000013C07D0FFF718FF0028F9D00C4B0122D5
:106F30001A60F5E70B4B00221A60E2E70024FEF727
:106F4000ABFD204638BD00BF2C9E0020249E0020B3
:106F5000709E0020349E0020C4990020B899002023
:106F6000B49E00206C9E002010B5A8B10446104BC2
:106F70001B6843B14FF0500383F31188BFF36F8F49
:106F8000BFF34F8FFEE7FFF7D9FE00212046FFF742
:106F9000CFFDFFF76DFF48B94FF0E0234FF080526F
:106FA000C3F8042DBFF34F8FBFF36F8F10BD00BF29
:106FB0002C9E0020214B1B681BB1214B01221A6023
:106FC00070471F4B00221A601E4B1B6803EB8301A6
:106FD0008A001D498A585AB90BB1013BF6E74FF0B8
:106FE000500383F31188BFF36F8FBFF34F8FFEE71A
:106FF00003EB830082000A4450684068506003EB52
:10700000830C4FEA8C020832114488420FD003EB04
:10701000830291000C4A0A445268D1680B4A1160FD
:1070200008490B6013685833094A13607047406879
:1070300062469100044A0A445060E8E72C9E002012
:10704000B49E0020349E0020C4990020B8990020EE
:107050009400002058B110B50C46094A1168183147
:10706000FEF775FC01212046FFF762FD10BD4FF0D1
:10707000500383F31188BFF36F8FBFF34F8FFEE789
:10708000B899002070B110B514460246114B1B6828
:107090008BB94FF0500383F31188BFF36F8FBFF3A9
:1070A0004F8FFEE74FF0500383F31188BFF36F8FCC
:1070B000BFF34F8FFEE7084B186841F00041816134
:1070C000196818311046FEF737FC01212046FFF7FA
:1070D0002FFD10BD2C9E0020B899002038B570B14E
:1070E0000D4614460A4A11681831FEF725FC0CB10A
:1070F0004FF0FF3521462846FFF71AFD38BD4FF007
:10710000500383F31188BFF36F8FBFF34F8FFEE7F8
:10711000B899002038B5C368DC6824B304F11805B9
:107120002846FEF72DFC184B1B682BBB251D284657
:10713000FEF726FCE06A154B1B68984201D9134BF9
:10714000186000EB80002946114B03EB8000FEF72E
:10715000F3FBE26A0F4B1B68DB6A9A4211D90120EC
:107160000D4B186038BD4FF0500383F31188BFF307
:107170006F8FBFF34F8FFEE729460848FEF7DCFB11
:10718000E7E70020EEE700BF2C9E0020349E0020A1
:10719000C4990020B8990020B49E0020709E002061
:1071A00038B51C4B1B6843B94FF0500383F311886B
:1071B000BFF36F8FBFF34F8FFEE741F000410160D7
:1071C000C468F4B1FEF7DCFB251D2846FEF7D8FBAA
:1071D000E06A114B1B68984201D90F4B186000EB15
:1071E000800029460D4B03EB8000FEF7A5FBE26A09
:1071F0000B4B1B68DB6A9A4202D90A4B01221A60C8
:1072000038BD4FF0500383F31188BFF36F8FBFF386
:107210004F8FFEE72C9E0020349E0020C499002052
:10722000B8990020B49E0020034B1B680360034BF9
:107230001B684360704700BF689E0020B09E00201E
:10724000D8B170B50C46054601B3FEF703FC1B4BE5
:1072500019686B68C81A2268B2F1FF3F27D0184E30
:107260003668D5F800C0B44501D08B4224D982429B
:1072700015D80023236001241AE04FF0500383F354
:107280001188BFF36F8FBFF34F8FFEE74FF05003AE
:1072900083F31188BFF36F8FBFF34F8FFEE75B1A45
:1072A000134423602846FFF7BFFF002400E00024BA
:1072B000FEF7F2FB204670BD0124F9E7B09E0020E6
:1072C000689E0020014B01221A607047B49E002086
:1072D000014B1868704700BFB8990020054B1B6828
:1072E00033B1054B1B680BB100207047022070477B
:1072F00001207047849E00202C9E002000283ED054
:1073000038B50446C36A204A1268D26A93422ED224
:107310008269002A05DB1C4A1268D26AC2F138026F
:107320008261616903EB8303184A02EB830399428C
:1073300005D0154B1B68DB6AE362012038BD251DB3
:107340002846FEF71DFB104B1B68D86AE062104B05
:107350001B68984201D90E4B186000EB800029464B
:107360000A4B03EB8000FEF7E7FA0120E6E7C26C68
:10737000054B1B68DB6A9A4203D30020DEE700203E
:1073800070470120DAE700BFB8990020C4990020B7
:10739000349E002000283BD038B504461E4B1B68A5
:1073A000834208D04FF0500383F31188BFF36F8FEF
:1073B000BFF34F8FFEE7036D43B94FF0500383F3E4
:1073C0001188BFF36F8FBFF34F8FFEE7013B03655B
:1073D000C16AC26C91421DD00BB1002038BD051DA1
:1073E0002846FEF7CDFAE06CE062C0F13803A361F5
:1073F0000A4B1B68984201D9084B186000EB8000CB
:107400002946074B03EB8000FEF796FA0120E5E7DB
:10741000002070470020E1E7B8990020349E00204A
:10742000C4990020002846D038B50446036D43B9FE
:107430004FF0500383F31188BFF36F8FBFF34F8F6B
:10744000FEE7C26C8A4200D20A46E16A914201D04C
:10745000012B00D038BD184B1B68A34222D0E2623A
:10746000A369002B02DBC2F13802A261626901EB61
:107470008101124B03EB81018A42EBD1251D284685
:10748000FEF77EFAE06A0E4B1B68984201D90C4B5E
:10749000186000EB80002946084B03EB8000FEF7E4
:1074A0004BFAD7E74FF0500383F31188BFF36F8F88
:1074B000BFF34F8FFEE77047B8990020C4990020B2
:1074C000349E0020044A136898691368DB6A1268C6
:1074D000C3F1380393617047B8990020054B1B68CE
:1074E00023B1044B1A68136D01331365014B1868FF
:1074F000704700BFB8990020064B1A6813682BB973
:107500000123036023B9D368186870470023F8E7A4
:1075100000207047B89E002008B54160006191428C
:107520000CD8D21A83699A4201D3012008BD011DEB
:10753000094B1868FEF70BFA0020F7E79A4201D2D0
:10754000994206D2011D054B1868FEF700FA00208B
:10755000ECE70120EAE700BFBC9E0020B89E0020B7
:1075600030B583B0FEF776FA114B1B681BB1FEF7FE
:1075700093FA03B030BD0F4D2846FEF7CFF90E4CFD
:107580002046FEF7CBF90D4B1D600D4B1C60002310
:1075900000930C4B0C4A10210A20FEF78CFD044B83
:1075A00018600028E3D00949FFF706F9DFE700BFBC
:1075B000DC9F0020609F0020749F0020B89E002068
:1075C000BC9E00208C9F0020C09E0020C4DD0008CF
:1075D00010B588B0FFF7C4FF124B1B68CBB1002475
:1075E0000594069407AA06A905A8FEF771F8059B5D
:1075F0000293069B0193022300932346079A0A49AC
:107600000A48FFF7D3FA0A4B186010B1012008B0FE
:1076100010BD4FF0500383F31188BFF36F8FBFF39A
:107620004F8FFEE7DC9F0020CCDD00083579000895
:10763000E09F0020B8B19C4603461848006858B344
:1076400000B585B000910192029305291CDCFFF77B
:1076500045FE022810D000231A4669460F480068EC
:10766000FEF797FD15E04FF0500383F31188BFF349
:107670006F8FBFF34F8FFEE70023069A69460748D6
:107680000068FEF786FD04E0002362466946FEF7C7
:107690008AFE05B05DF804FB00207047DC9F0020E7
:1076A00070B582B01B4B1B681A6862B3DB681E683A
:1076B000DC68251D2846FEF763F9236A20469847B3
:1076C00094F8283013F0040FECD0A36933449E42A1
:1076D00007D26360246129460E4B1868FEF737F91C
:1076E000E0E7002100910B4632462046FFF7A2FF5B
:1076F0000028D7D14FF0500383F31188BFF36F8F69
:10770000BFF34F8FFEE7044A106802490860136018
:1077100002B070BDB89E0020BC9E002038B5054662
:10772000FFF714FB0446074B1B68834205D8002370
:107730002B60044B1C60204638BDFFF7B1FF0123CE
:107740002B60F6E7889F002070B582B006460D4694
:1077500017490968C968CC68201DFEF711F994F82B
:1077600028C01CF0040F08D12CF0010C84F828C0AC
:10777000236A2046984702B070BDA16933462A4665
:1077800031442046FFF7C8FE0028F1D000210091C7
:107790000B4632462046FFF74DFF0028E8D14FF058
:1077A000500383F31188BFF36F8FBFF34F8FFEE752
:1077B000B89E002070B582B006460C46FFF7BEFAB0
:1077C00001A8FFF7ABFF019B33BB05460CB9B042E4
:1077D00019D224B1124A12681268DAB90124224679
:1077E000711B104B1868FEF7FBFFFFF741FBA8B9B0
:1077F0004FF0E0234FF08052C3F8042DBFF34F8FBA
:10780000BFF36F8F0AE0FFF733FB29463046FFF7DF
:107810009BFF03E01C46E2E7FFF72AFB02B070BDC6
:10782000BC9E0020DC9F002010B588B002E0049BC5
:10783000002B0FDA002204A93D4B1868FEF71AFE50
:10784000002873D0049B002BF1DA07990698059B5A
:107850009847ECE7069C636913B1201DFEF790F88A
:1078600003A8FFF75BFF049B092BE3D8DFE803F0D5
:107870000505053037500505303794F8283043F0BA
:10788000010384F82830059BA1690246194420466B
:10789000FFF742FE0028CDD0236A2046984794F88F
:1078A000283013F0040FC5D0A269002100910B46C7
:1078B000059802442046FFF7BDFE0028BAD14FF0DC
:1078C000500383F31188BFF36F8FBFF34F8FFEE731
:1078D00094F8283023F0010384F82830AAE794F8BC
:1078E000283043F0010384F828300599A16131B1B3
:1078F0000346024601442046FFF70EFE9AE74FF08A
:10790000500383F31188BFF36F8FBFF34F8FFEE7F0
:1079100094F8283013F0020F04D023F0010384F808
:10792000283087E72046FEF78DFA83E708B010BDC0
:10793000DC9F002000B583B001A8FFF7DDFD0199B1
:10794000FFF738FFFFF770FFF6E7000010B584B0CF
:1079500014461A466FF001030093019002910394BC
:107960000023694602480068FEF71DFD04B010BD03
:10797000DC9F0020014B1868704700BF9400002076
:1079800070B50D4E0D4D761BB61006D0002455F87F
:10799000043B01349847A642F9D1094E094D06F03F
:1079A00063F8761BB61006D0002455F8043B01346A
:1079B0009847A642F9D170BD000000000000000009
:1079C0000000000000000000830730B548D0541EBE
:1079D000002A3FD00346CAB201E0013C3AD303F883
:1079E000012B9D07F9D1032C2DD9CDB245EA0525F0
:1079F0000F2C45EA054536D9A4F1100222F00F0CF0
:107A000003F1200EE6444FEA121C03F1100242E992
:107A1000045542E9025510327245F8D10CF10102C9
:107A200014F00C0F03EB021204F00F0C13D0ACF1A6
:107A3000040323F003030433134442F8045B93422A
:107A4000FBD10CF003042CB1CAB21C4403F8012B87
:107A50009C42FBD130BD64461346002CF4D1F9E7BB
:107A600003461446BFE71A46A446E0E70FB400B544
:107A7000074A83B004AB106853F8042B8168019364
:107A800000F02CF903B05DF804EB04B0704700BFC0
:107A90009400002030B5054689B008460C4600F039
:107AA000BBF801210223214A04940692AA6B04AC7C
:107AB0000590084401940791AC680293039022B3A7
:107AC000636E13F0010FB4F90C309AB201D198052E
:107AD00025D5910406D4626E43F4005322F400527B
:107AE000A3816266284601AA214603F0F3F9636E7A
:107AF000002814BF4FF0FF350A25DA0702D4A38906
:107B00009B0506D5284609B030BD284603F000F88D
:107B1000D6E7A06D03F084FB284609B030BDA06D08
:107B200003F07CFBB4F90C309AB2D2E7A4DB000876
:107B3000024B01461868FFF7ADBF00BF940000205C
:107B40002DE9F0410E680C460546BEB137688FB18D
:107B5000D7F80080B8F1000F08D0D8F8001009B1AC
:107B6000FFF7EEFF4146284603F0B4F839462846B1
:107B700003F0B0F83146284603F0ACF82146284619
:107B8000BDE8F04103F0A6B8224B1B68834240D009
:107B9000C16C70B5054681B100268C593CB12146B7
:107BA0002468284603F096F8002CF8D1E96C0436D6
:107BB000802EF2D1284603F08DF8296C11B12846A9
:107BC00003F088F8D5F8484154B105F5A676B442DB
:107BD00006D021462468284603F07CF8A642F8D156
:107BE000696D11B1284603F075F8AB6B83B1284677
:107BF000EB6B9847D5F8E04254B1216811B12846A3
:107C0000FFF79EFF21462846BDE8704003F062B8AA
:107C100070BD70479400002020F0030110F00300B5
:107C2000C0F1000051F8043B00F1040C4FEACC0C09
:107C30006FF000021CBF22FA0CF213434FF0010C4C
:107C40004CEA0C2C4CEA0C4CA3EB0C0222EA03028B
:107C500012EACC1204BF51F8043B0430F4D0C2F154
:107C6000000102EA0102B2FA82F2C2F11F0200EB45
:107C7000D200704730B540EA0104A30722D1032A9D
:107C800020D90B468446194653F8045BA5F101340C
:107C900024EA050414F0803F15D1043A032A19465A
:107CA0004CF8045BEFD801F1FF3E52B163461EF879
:107CB000011F541E03F8011B41B122469C46002AB5
:107CC000F4D130BD844601F1FF3EEEE76244002C62
:107CD000F7D003F8011B9342FBD130BD2DE9F04FE3
:107CE000D5B01C46914607910546099003F08EFADF
:107CF00002680E9410461792FFF78EFF16901DB182
:107D0000AB6B002B00F01D82079A536EDD0740F12C
:107D10002D81B2F90C2091B28F0409D4079B42F453
:107D200000529A8191B21A465B6E23F40053536657
:107D30000E0740F1C080079B1B69002B00F0BB8041
:107D400001F01A030A2B00F0C48000242BAB22465A
:107D500098464D46CDE929442893129400230024E7
:107D6000CDE914342B78CDE91922CDE91B221892E4
:107D70000B92002B00F08F81AA4604E01AF8013F15
:107D8000002B00F0BB80252BF8D1BAEB050640F0A4
:107D9000B9809AF80030002B00F07D8100234FF06D
:107DA000FF324FF02B0920241F469AF801600892F9
:107DB0000AF1010A8DF883300A930AF1010AA6F14B
:107DC00020035A2B00F2E180DFE813F00503DF0007
:107DD000DF000003DF00DF00DF00DE02DF00DF0086
:107DE0006A006E02DF0055027802DF0073025B005A
:107DF0005B005B005B005B005B005B005B005B00AB
:107E0000DF00DF00DF00DF00DF00DF00DF006C01EC
:107E1000DF00EA01C4016C016C016C01DF00DF00CE
:107E2000DF00DF00D002DF00DF002302DF00DF0021
:107E3000DF00F801DF009202DF00DF008707DF00CC
:107E4000DF00DF00DF00DF00DF00DF00DF006C01AC
:107E5000DF00EA01C6016C016C016C01B602C601CB
:107E6000BF01DF00C302DF005A022502A402BF01E6
:107E7000DF00F80172008407DF00DF006507DF0024
:107E800072000022A6F130031AF8016B02EB8202A5
:107E900003EB4202A6F13003092BF5D90A928EE7D3
:107EA0000E9B53F8042B002A0A920E93C0F2E08135
:107EB0009AF8006081E7079D0998294601F0FCFCCB
:107EC000002841F04D83A98901F01A030A2B7FF4A1
:107ED0003CAF079AB2F90E30002BFFF636AF536E67
:107EE000D80702D4890541F1488123464A460799BB
:107EF000099855B0BDE8F04F01F09CBCBAEB0506FF
:107F000000F0C9802A9BC8E9005633442A93299B74
:107F10000133072B299305DC08F108080B9B334438
:107F20000B9336E70799099828AA04F0C5FB80B996
:107F30000DF1AC08F2E70799099828AA04F0BCFBF8
:107F4000002800F099800D9B1BB11946099802F09A
:107F5000C1FE079A536ED90740F1E88093895B060A
:107F600001F10A830B9855B0BDE8F08F079BB3F978
:107F70000C20900591B23FF5CFAE1D46986D03F0F1
:107F80004DF9B5F90C2091B2C6E6002E00F08380C1
:107F9000012300228DF8EC6006933BAD8DF8832021
:107FA0000C930D9208920F921392109217F0020305
:107FB00002D006990231069117F0840B07D10A9975
:107FC0000698A1EB0009B9F1000F00F390832A9CF9
:107FD00082B10122C8F80420299A013401320DF13E
:107FE0008301072A2A942992C8F8001000F3D88345
:107FF00008F108087BB10223C8F80430299B023439
:10800000013321AA072B2A942993C8F8002000F3F2
:10801000D58308F10808BBF1800F00F08882089B27
:108020000C9AA3EB020BBBF1000F00F3CB82FB0514
:1080300000F11F820C9BC8F800501C44C8F80430A3
:10804000299B2A940133072B299300F3448308F1D9
:108050000808780705D50A9B069A9D1A002D00F39B
:10806000B983DDE90A2306998A42ACBF9B185B18E5
:108070000B93002C7FF45FAF002329930D9B1BB162
:108080000D99099802F026FE55460DF1AC082B78A3
:10809000002B7FF471AE2A9B002B41F0108200234D
:1080A000299356E70E9B073323F00702F2E80234C8
:1080B000CDE91434DDE9143424F00044994618461F
:1080C0000E9221464FF0FF32AB4BF8F75DFD0028D2
:1080D00040F01885484621464FF0FF32A64BF8F78E
:1080E00035FD002840F00E85DDE914010022002353
:1080F000F8F722FD002840F065879DF883200021D5
:1081000003209E4D9E4B27F080070D910690472E31
:10811000C8BF1D4608910C900F9113911091002A31
:108120003FF444AF069B013306933FE7079B9B89CF
:108130009A053FF514AF079CA06D03F071F8A38971
:108140000DE7099802F0E4FCDEE59AF8006047F0DC
:10815000200732E647F01007BA060E9B40F16E8406
:10816000073323F007031A465B6852F8084B994619
:108170000E92002BC0F26F84089B013300F0FB824B
:1081800054EA090327F0800B40F0F682089B002B8D
:1081900040F0F7825F46002354AD08930C933DE115
:1081A000012000220E9B069053F8041B3BAD8DF876
:1081B00083208DF8EC100E930C90F2E64FF000093E
:1081C0000E9C089B54F8045B8DF88390002D00F002
:1081D000A1855A1C00F0A5861A464946284603F098
:1081E0003DFB0D90002801F050810D9B9DF88320F0
:1081F0005B1B0C9323EAE373CDF820900E94069357
:10820000CDF83490CDF83C90CDF84C90CDF840901E
:1082100085E747F0100717F0200900F0F2830E9B66
:10822000073323F00703D3F8049053F8084B0E9359
:10823000002327F4806B00228DF88320089A511CBC
:1082400000F0D48054EA09012BF0800740F0CD8083
:10825000002A40F00486002B9DD11BF001030C93F3
:1082600000F0308430230DF24F158DF84F31D5E0FA
:108270000A9B5B420A939AF8006047F004079CE56A
:10828000BD0600F1FD84FC0600F1EE85780600F1E4
:10829000B286B90540F1E8850E9B0B9953F8042B83
:1082A000554611700E93F2E69AF800608DF88390AF
:1082B00083E59AF8006047F080077EE5524612F8A1
:1082C000016B2A2E01F08D82A6F13003092B924614
:1082D00098BF002201F2E5801AF8016B02EB8202DE
:1082E00003EB4202A6F13003092BF5D9089266E5AB
:1082F00047F0100B1BF0200900F091830E9B073311
:1083000023F007031A4652F8084BD3F804900E9254
:10831000012390E7302278260E9B8DF8842053F8B5
:10832000044B184A0E934FF00009022347F0020B4A
:108330008DF8856018927EE79AF80060682E03BF7A
:108340009AF8016047F400770AF1010A47F0400704
:1083500033E59AF800606C2E03BF9AF8016047F08D
:1083600020070AF1010A47F0100726E59AF8006095
:1083700047F0080721E500BFFFFFEF7FD4DD0008CD
:10838000D8DD0008E4DD0008099E304602F03EFF1B
:10839000436818461B93FFF73FFC034630461C9387
:1083A0001E4602F033FF83681993002E3FF480AD20
:1083B000199B002B3FF47CAD199B1B78002B3FF4DD
:1083C00077AD9AF8006047F48067F6E49AF80060A9
:1083D00047F00107F1E49DF88330002B7FF468AD8E
:1083E0009AF800608DF88340E7E4BB46012B00F06B
:1083F000C381022B54AD1FD1189A04F00F03D35C34
:10840000240944EA09744FEA191905F8013D54EAB0
:108410000903F2D15F4654AB5B1B0C93089A0C998D
:1084200000238A42B8BF0A460D9306920F939DF827
:1084300083201393109372E604F00703E40844EAE0
:1084400049744FEAD909303354EA09012A4605F83C
:10845000013DF1D11BF0010FDCD0302BDAD03023FD
:10846000023A05F8013C54AB9B1A5F4615460C9343
:10847000D4E7652E40F3E980DDE9140100220023F2
:10848000F8F750FB002800F0E1810123C8F8043020
:10849000299BC04A01330134072B2A942993C8F839
:1084A000002000F3BF8408F10808229B129A93422F
:1084B00080F2DC82169B179A1C44C8E90023299B92
:1084C0002A940133072B299300F3178408F1080835
:1084D000129B5D1E002D7FF7BCAD102D41F35D8119
:1084E000DFF8B492224649461026B946299B0F462A
:1084F000DDF824B0079C05E008F10808103D102DB8
:1085000040F39D8401331032072BC8E90076CDE992
:108510002932F1DD2146584628AA04F0CDF800287A
:108520007FF411ADDDE929320DF1AC08E6E70A9BD5
:10853000069AA3EB020BBBF1000F7FF770ADBBF106
:10854000100F41F35280DFF8509241462046A84672
:108550004C461023299A079DDDF8249006E0ABF1E4
:10856000100BBBF1100F01F1080119DD01321030C1
:10857000072AC1E90043CDE92920F0DD2946484614
:1085800028AA04F099F800287FF4DDACDDE9292061
:10859000ABF1100BBBF1100F4FF010032BA9E5DC72
:1085A0004546A1468846044601325C44072ACDE987
:1085B0002924C8F80090C8F804B000F3918308F1AA
:1085C00008082CE5BBF1100F40F3E384DFF8C891F5
:1085D00041462046A8464C461023299A079DDDF8BF
:1085E000249006E0ABF1100BBBF1100F01F1080174
:1085F00019DD01321030072AC1E90043CDE92920F5
:10860000F0DD2946484628AA04F056F800287FF4F1
:108610009AACDDE92920ABF1100BBBF1100F4FF044
:1086200010032BA9E5DC4546A146884604460132E5
:108630005C44072ACDE92924C8F80090C8F804B0A2
:1086400000F3D28108F10808F1E4129B012B40F3FA
:1086500082810123299E01341E44072EC8F8005050
:108660002A94C8F80430299600F36C8308F10808AE
:10867000169B0136179A1C44072EC8E90023CDE942
:10868000296400F36C8308F108080022DDE9140175
:108690000023F8F747FA002840F07A81129B013650
:1086A000013B01351C44072EC8F800502996C8F834
:1086B00004302A9400F35F8108F108081A9B013600
:1086C0001C44C8F80430072E24ABCDE92964C8F84F
:1086D00000307FF7BCAC0799099828AA03F0ECFF9B
:1086E00000287FF430AC2A9C0DF1AC08B1E4B9F15C
:1086F000100F40F3C686DDE929214046CDE91D363D
:10870000B84610244F46079EA946099D04E0103F35
:10871000102F00F1080016DD0132204B1031072A1E
:10872000C0E90034CDE92921F1DD3146284628AAE7
:1087300003F0C2FF00287FF406ACDDE92921103FD9
:10874000102F2BA8E8DC4D46DDE91D36B94647461B
:10875000804609EB010401321049072ACDE929249A
:10876000C8F80490C8F8001000F340839DF88320F7
:1087700008F108082CE4BB460A2C79F1000380F0CC
:10878000FB82012330345F468DF84F410C930DF28C
:108790004F1543E614DE000828DE000818DE000846
:1087A0000799099828AA1D9303F086FF00287FF4F3
:1087B000CAAB2A9C1D9B0DF1AC081BE407990998D4
:1087C00028AA03F079FF00287FF4BDAB2A9C0DF1A5
:1087D000AC0820E4102D40F3BE861026299B099F8B
:1087E000DDF81C9004E0103D102D08F1080817DD9D
:1087F0000133BA4A1034072BC8E90026CDE92934E1
:10880000F1DD4946384628AA03F056FF00287FF4D8
:108810009AABDDE92934103D102D0DF1AC08E7DCF1
:108820000133AE4A2C44072BCDE92934C8F8045053
:10883000C8F800207FF715AC0799099828AA03F01B
:108840003BFF00287FF47FAB2A9C0AE42299002991
:1088500040F31081DDF84090129B9945A8BF9946DE
:10886000B9F1000F0BDD299B4C440133072BC8E9FC
:1088700000592A94299300F3818508F10808109E75
:10888000B9F1000FA8BFA6EB0906002E00F3F58290
:10889000DDF840B07905AB4400F1AC84229B129A1C
:1088A000934202DBFA0740F19283169A1799144417
:1088B000C8E90012299A2A940132072A299200F362
:1088C000A88508F10808129AAE18A6EB0B06D51A6F
:1088D000AE42A8BF2E46002E0DDD299B3444013345
:1088E000072BC8F800B0C8F804602A94299300F355
:1088F000FC8508F10808002EA8BFAD1B002D7FF7EE
:10890000A8AB102D40F34987DFF8D49122464946A1
:108910001026B946299B0F46DDF824B0079C05E0D8
:1089200008F10808103D102D40F389820133103200
:10893000072BC8E90076CDE92932F1DD21465846FA
:1089400028AA03F0B9FE00287FF4FDAADDE9293248
:108950000DF1AC08E6E7FE073FF57BAE0123299E4B
:1089600001341E44072EC8F800502A94C8F8043079
:1089700029967FF7A1AE0799099828AA03F09CFED3
:1089800000287FF4E0AADDE929640DF1AC0895E642
:10899000129B5D1E002D7FF791AE102D40F31987BD
:1089A000224608974FF0100BDFF83491099C079F7F
:1089B00005E008F10808103D102D40F3C78201368C
:1089C0001032072EC8E9009BCDE92962F1DD394656
:1089D000204628AA03F070FE00287FF4B4AADDE93F
:1089E00029620DF1AC08E6E70799099828AA03F077
:1089F00063FE00287FF4A7AA2A9C0DF1AC08FFF7BC
:108A000016BB17F0100377D117F0400200F0AC82CC
:108A10000E9A994652F8044B0E92A4B208E41BF049
:108A200010030E9A54D11BF040014DD052F8044B64
:108A300099460E920123A4B2FFF7FDBB53F8044BF5
:108A40000E93FB0653D47D064ED544F3C0394B46F6
:108A500024B2FFF78EBB2D2364428DF88330BB46D2
:108A60004FF0010369EB4909FFF7E8BBF8077FF511
:108A7000F0AA1FE50123C8F80430299B194A0133E5
:108A80000134072B2A942993C8F8002000F3688446
:108A900008F10808002940F02582129A07F0010326
:108AA00013433FF4D6AA169B1799E218C8E900139E
:108AB000299B2A920133072B299300F3508308F155
:108AC000080820E254ADA9E41BF4007940F0A0822C
:108AD00052F8044B01230E92FFF7ADBB18DE0008DD
:108AE00028DE000814DE0008B80500F179824FEA9C
:108AF000E4794B46FFF73DBB0E9B53F8044B0E93B6
:108B0000FFF796BBDDE9140102460B46F8F73CF887
:108B1000002840F0F785612E00F06C85412E00F0B2
:108B20007F82089B013300F0948526F02003472BB9
:108B3000069300F07B85DDE9141247F480730F93F0
:108B40001346002BC0F2F4850C9300238B461D9333
:108B50000D93069B462B00F02B84452B00F01485CB
:108B600008990C9B01910221009126A9049123A947
:108B7000039122A95A460998029100F09DFF069B95
:108B80000546472B40F0448617F0010FB9460F9F6A
:108B900040F0F784269B5B1B1293069B472B00F04B
:108BA000F182069B462B00F04284229B1093109B7F
:108BB000069A013B412A229300F08A850021F2B2F5
:108BC000002B8DF89020B6BF2D222B22109B8DF804
:108BD0009120B8BFC3F10103092B40F381850DF14A
:108BE0009F0C6246BA4F1C46104687FB0312D917EA
:108BF000C1EBA20101EB8102A3EB42023032632CF4
:108C000000F8012C0B4600F1FF32ECDC3033811E02
:108C1000DBB28C4502F8013C40F2FF850DF1920178
:108C200001E012F8013B944501F8013BF9D10DF147
:108C3000A1030DF192021B1A134424AA9B1A1A9342
:108C4000129B1A9A012B1A440C9240F39E850C9B9E
:108C5000169A13440C9300230C9A29F4806722EA95
:108C6000E27247F480770F930692139310931D9B43
:108C7000002B40F0B0829DF883200893FFF74FBA95
:108C80000E9B0B9853F8041BC2175546C1E900020E
:108C90000E93FFF7FCB98F4B189317F0200949D0BA
:108CA0000E9B073323F00703D3F8049053F8084BC7
:108CB0000E93F80709D554EA090306D030238DF83E
:108CC000856047F002078DF88430022327F4806B1B
:108CD000FFF7B1BABB46FFF70DBB7F4B1893DCE73C
:108CE0000799099828AA03F0E7FC00287FF42BA92C
:108CF0002A9C0DF1AC08FFF792B90799099828AAA8
:108D000003F0DAFC00287FF41EA92A9C0DF1AC08C0
:108D1000FFF7DEBB062B294628BF06232A46089507
:108D20000D9506936D4D0E940C930F911391109128
:108D3000FFF7F5B917F0100369D00E9B53F8044BF9
:108D40000E93B6E70799099828AA03F0B5FC002806
:108D50007FF4F9A8DDE929640DF1AC0888E40799EE
:108D6000099828AA03F0A8FC00287FF4ECA8DDE904
:108D700029640DF1AC0888E400230BF48062CDE98E
:108D80000CA8069692461E46DDF8648054AF0CE0AF
:108D90000023204649460A22F7F734FF0A2C79F1CE
:108DA00000031BD3044689462F4620460A2200238F
:108DB0004946F7F727FF30327D1E013607F8012CB0
:108DC000BAF1000FE4D098F800309E42E0D1FF2EB7
:108DD000DED00A2C79F1000380F0E080CDF86480C9
:108DE0001296DDE90CA8069EFFF714BB07990998B7
:108DF00028AA1D9303F060FC00287FF4A4A89DF826
:108E000083202A9C1D9B0DF1AC08FFF7E1B817F0F9
:108E1000400200F0B4800E9A994652F8044B0E922C
:108E2000A4B246E70799099828AA03F045FC002850
:108E30007FF489A82A9C0DF1AC08FFF736BB1446D5
:108E40003A464F46914601332C44072BC8F8009010
:108E5000C8F80450CDE929347FF7F9A83BE4012B89
:108E6000BB467FF4C6AA8CE40E9B0B9953F8042BE7
:108E7000554611600E93FFF70AB9102E40F3AD84EA
:108E8000DFF85C90424648462146A846B9464FF076
:108E9000100B0746299B099C079D04E00832103EF1
:108EA000102E40F3488201331031072BC2E9007BBA
:108EB000CDE92931F2DD2946204628AA03F0FCFB42
:108EC00000287FF440A8DDE929312BAAE7E700BF9D
:108ED00067666666E4DD0008F8DD00080CDE000861
:108EE00028DE0008169B1798E218C8E90003299BA2
:108EF0002A920133072B299300F3318108F10808E6
:108F00000029C0F20283129901338C18072BCDE996
:108F10002934C8F80050C8F804107FF798A8FFF764
:108F2000DABB2846CDF820900E94FEF775FE20EAB5
:108F3000E073CDE90C099DF88320CDF83C90CDF885
:108F40004C90CDF840900693FFF7E9B81446089F7F
:108F500001362C44072ECDE92964C8F80090C8F8E2
:108F600004507FF7A9AB06E517F400790E9B3DD0BE
:108F700053F8044B91460E93E4B2FFF759B917F436
:108F800000790E9B40D053F8044B91460E93E4B207
:108F90008FE6299ADFF84C92FFF749BB1C9B1B997F
:108FA000ED1A1A462846FEF765FE98F801300BB117
:108FB00008F10108204649460A2200230026F7F757
:108FC00021FEEFE62D228DF88320FFF798B8129A44
:108FD000AE18A6EB0B06D51AAE42A8BF2E468AE401
:108FE00044F3C0194B4664B2FFF7C3B853F8044BBF
:108FF0000E93FFF71DB90E9B0B9953F8042B5546A2
:1090000011800E93FFF743B853F8044B0E9350E6CC
:1090100052F8044B894601230E92E4B2FFF70BB9D4
:1090200030238DF8843058238DF88530089B47F025
:109030000204632B00F3E38200233BAD0D9347F45E
:1090400081730F93DDE914121346002B2746C0F2FB
:1090500040820C9300238B461D9326F02003069339
:10906000612E00F01783412E7FF473AD22AA58467B
:109070000C9903F055FA00224FF07F53F7F7EAFA04
:1090800002460B46CDE9102300220023F7F74AFDE4
:1090900008B101232293544B0C93089BCDE912A6EF
:1090A000CDE91E78DDE91067AB46DDF830A003F1AD
:1090B000FF39109506E00022002309F1FF39F7F788
:1090C00031FDE8B90022494B30463946F7F7C2FA7C
:1090D0000F460646F7F76EFD0446F7F751FA0B46C2
:1090E000024639463046F7F7FDF81AF80430B9F170
:1090F000FF3FD8464D4606460F460BF8013BDAD1F6
:109100003046394600223A4BA946DDF848A0109D6A
:10911000CDF84880CDE91001DDF87C80139E1E9FBC
:10912000F7F728FD002840F04482DDE91001002215
:109130002F4BF7F7F7FC10B1E10700F13A824B46ED
:10914000002B06DB302201335B440BF8012B5B451F
:10915000FBD1ABEB0503B94612930F9F1DE50799B1
:10916000099828AA03F0A8FA00287EF4ECAEDDE9FD
:10917000293222990DF1AC08C2E6906D02F050F848
:10918000FEF7B3BE229BDA1C109302DB089A9342CF
:1091900004DD023E26F02003069308E5109B129A98
:1091A0009342C0F2828119F0010F00F0A882169A52
:1091B00013440C9319F4806F00F09082109B672683
:1091C000002B00F346810C9B23EAE37306930023F4
:1091D0000F9313934BE52D2200238DF883200893E2
:1091E000FEF7A0BF28DE0008F8DD000800003040D0
:1091F0000000E03F129B4246DDF84C80EB185E46D3
:109200000893CDF830A010972146199FDDF8709093
:10921000DDF824A0DDF81CB00F9B1395B8F1000F0A
:109220002ED0002B6CD1013F08F1FF381B9B494425
:10923000C2E90039299B2A910133072B299363DC6A
:109240000832089B38789B1B8342A8BF0346002B3B
:109250001C460ADD2998194401300728C2E9006339
:109260002A9129905BDC38780832002CB4BF05467F
:10927000051B002D15DC06440F9BB8F1000FD0D163
:10928000002B3DD1DDE91235EB189E42B34619970C
:1092900090460C4628BF9B46DDF830A0109FFFF794
:1092A000FDBA102D40F36F821024299804E0103D80
:1092B000102D02F1080216DD0130A84B10310728ED
:1092C000C2E90034CDE92901F1DD5946504628AA0A
:1092D00003F0F2F900287EF436AEDDE92901103DF5
:1092E000102D2BAAE8DC01309C4B29440728CDE93E
:1092F0002901556013604EDC387808320644BBE71C
:109300000F9B013B0F9391E75946504628AA03F063
:10931000D3F900287EF417AE2A992BAA91E7594673
:10932000504628AA03F0C8F900287EF40CAE38781D
:109330002A992BAA99E7454690463A460C464F464D
:10934000914601333444072BCDE92934C8F8009005
:10935000C8F8046000F35D8108F10808FFF798BAC7
:109360000799099828AA03F0A7F900287EF4EBAD25
:1093700022992A9C0DF1AC08FFF78CBB079909983C
:1093800028AA03F099F900287EF4DDAD2A9C0DF19E
:10939000AC08FFF774BA5946504628AA03F08CF976
:1093A00000287EF4D0AD38782A992BAA064463E7CA
:1093B00008990C9B01910321009126A9049123A9EE
:1093C000039122A95A460998029100F075FB03788F
:1093D0000546302B00F0C081229B089AB946134401
:1093E0000F9FEC185846002200230C99F7F79AFBC0
:1093F00010B12346FFF7CFBB269BA342BFF4CBABF4
:1094000030215A1C26921970269B9C42F9D8FFF7EE
:10941000C2BB0799099828AA03F04EF900287EF4E8
:1094200092AD229B2A9C0DF1AC08FFF74CBA229A10
:10943000002A109240F3B981089909F001030B4307
:1094400040F040816626109B0C9319F4806F3FF426
:10945000BAAE19990B78FF2B00F0D6810024109A30
:10946000204604E001300131FF2B00F0648193427B
:1094700080F26181D21A4B78002BF3D10B78013442
:10948000F2E7DDE92921FFF764B9089B9DF8832005
:109490000E9406930C9308900F9013901090FEF783
:1094A0003EBE00230893FEF78ABC129B169A9A18B8
:1094B000109B0C92002B40F35D816726C5E707994E
:1094C000099828AA03F0F8F800283EF4E8ADFEF762
:1094D00040BD26F0200306932D22DDE914349B467F
:1094E00004F100431D920C93BAE50799099828AA44
:1094F00003F0E2F800287EF426AD229D129B2A9C00
:109500000DF1AC085D1BFFF7F6B94E42103180F249
:10951000818141461024A846DFF84090DDF824B050
:10952000079D04E00831103E102E40F3998001336E
:109530001032072BC1E90094CDE92932F2DD29462A
:10954000584628AA03F0B8F800287EF4FCACDDE900
:1095500029322BA9E7E7299BFFF762B928DE00082B
:10956000079B5B6EDD0707D4079B9B899C0503D493
:10957000079B986D01F054FE4FF0FF330B93FEF7FD
:10958000F1BC089BEC182DE70221009108995A467E
:109590004C1C26A9049123A9039122A90C9B09988C
:1095A0000194029100F088FA0546B9462C440F9FB9
:1095B00018E7129B26930C9B1BF8012CD97B5B466A
:1095C0008A4209D1302003F8010C269B5A1E2692AC
:1095D00013F8012C9142F6D0392A0BBF0C9A0132B4
:1095E000927AD2B203F8012CB3E5299ADFF83492CB
:1095F000FEF7DABF30238DF88430782314E509981C
:10960000591C01F07FFE0546002800F0F6800D9001
:1096100015E50799099828AA03F04EF800287EF46A
:1096200092AC2A9C0DF1AC08FFF732B9089B002BD5
:1096300008BF0123089347F480730F93159B002BF9
:10964000C0F2A980DDF850B01D900C930D90FFF78B
:1096500087BA0623089326F020030693FFF76BBA18
:109660004546884601333244072BCDE92932C8F8F4
:109670000090C8F804607FF722AA0799099828AAE1
:1096800003F01AF800287EF45EACDDE929320DF112
:10969000AC0838E422AA58460C9902F041FF002297
:1096A0004FF07F53F6F7D6FF02460B46CDE9102365
:1096B00000220023F7F736FA08B1012322935A4B10
:1096C0000C93EAE4169B6626D31819440C91BCE669
:1096D00006F10F020121D2B2FFF772BA672672E5D6
:1096E00000295FD130228DF892200DF193023033A2
:1096F00002F8013B24ABD31A1A93FFF7A1BA109BCF
:109700000C9357E5159B0320002BB8BF2D224FF07B
:109710000003A8BF9DF8832019460D93434D444B89
:10972000B8BF8DF8832027F080070690FEF7EFBCC6
:1097300000230D93D0E61991109213900F940F9A75
:10974000139B1C9913440C9A01FB03230C9323EAEB
:10975000E3730693FFF78BBA5846002200230C9957
:10976000F7F7E0F900287FF437AE089BC3F1010357
:10977000229332E6C3F101031A4422EAE273672618
:109780000C92069323E52998ADE519F0010F3FF4FB
:1097900062AAFFF75CBA0D909EE6299BDFF88490E1
:1097A000FFF751BB0DF19202A1E7089A09F00109F8
:1097B00059EA020304D10123662606930C9306E5B9
:1097C000169B662601331A4422EAE2730C92069332
:1097D000FDE4DFF85090FFF7BBBB299BDFF8449016
:1097E000AFE50E9B9AF80160924653F8042B0E9356
:1097F00042EAE2730893FEF7E0BA079A938943F0CE
:1098000040039381FEF7A5BB00230F93139396E7C4
:10981000089CCAE6DFF80C9024E702231A93FFF7AE
:109820000FBA00BF28DE0008E4DD0008DCDD000818
:10983000E0DD0008F0B54FF4806C154600240646C4
:109840001F46ADF26C4D1AAB009304938B8916A89A
:1098500023F00203ADF80C304B6E06941993CB89BC
:109860000C46ADF80E30CB69CDF808C007934B6AB3
:10987000CDF814C0099301F0CDFC2A463B46694659
:109880003046FEF72BFA051E07DB6946304601F02D
:109890000BF9002818BF4FF0FF35BDF80C305B0600
:1098A00003D5A38943F04003A381169801F0B4FCCB
:1098B00028460DF26C4DF0BD38B5334B05461B689C
:1098C0000C460BB19A6B12B3B4F90C3018079AB26C
:1098D00025D5216900292DD012F0010007D00025DF
:1098E0006069A5604042A06139B1002038BD95078C
:1098F00058BF6069A0600029F7D1120658BF08461A
:10990000F4D543F040034FF0FF30A38138BD184633
:1099100001F0FEF8B4F90C3018079AB2D9D4D10688
:109920002AD5520714D4216943F00803A3819AB2BF
:109930000029D1D102F42070B0F5007FCCD02146AF
:10994000284601F06FFCB4F90C3021699AB2C3E7E4
:10995000216B51B104F14002914204D0284601F03C
:10996000B9F9B4F90C30002222630022216923F0F6
:109970002403C4E90012D7E7092243F040032A6018
:109980004FF0FF30A38138BD940000202DE9F04F47
:1099900003690C6985B0A342C0F28980013C01F1E2
:1099A0001405A30000F11408019355F8243058F869
:1099B000242001338A469A4208EB84018146B2FB97
:1099C000F3F605EB840702913AD30021AE464046F8
:1099D0000A46A34603955EF8045B0468ABB206FB37
:1099E00003132D0C190C06FB05119BB2D21A1FFA9A
:1099F00084FC94448AB2C2EB144202EB2C421FFA5C
:109A00008CFC4CEA0243774540F8043B4FEA114195
:109A10004FEA2242DFD2019B5C4658F80330039D97
:109A200073B9029B043B984504D307E0984504F1C1
:109A3000FF3403D253F80429002AF7D0C9F81040A4
:109A40005146484602F056FA00282CDB40460023D7
:109A5000013655F8041BD0F800C08AB29A1A1FFAD2
:109A60008CFE0B0C7244C3EB1C4303EB224392B2FB
:109A700042EA0342AF4240F8042B4FEA2343E8D2C4
:109A800058F8242008EB84036AB9043B984504D3B2
:109A900007E0984504F1FF3403D253F80429002A63
:109AA000F7D0C9F81040304605B0BDE8F08F00206F
:109AB00005B0BDE8F08F00BF2DE9F04F9046994604
:109AC000016C99B00446CDE90489259D41B101237B
:109AD000426C93408B604A6001F0B6FF0023236420
:109AE000B9F1000AB4BF012300232B60764BBCBF41
:109AF0002AF0004ACDF814A033EA0A0300F0AA8045
:109B0000DDE904231046194600220023CDE90A01AD
:109B1000F7F708F8074670B10123249A1360269BD3
:109B2000002B00F0E68269481860431E03930398F7
:109B300019B0BDE8F08F16AB019317AB0093204628
:109B4000DDE90A2302F09CFA5FEA1A56054640F066
:109B50009780DDE916763E4406F23240202840F335
:109B6000B783C0F140000AFA00FA06F2124028FA60
:109B700000F04AEA0000F6F7F3FC0123013E0F93E0
:109B8000A1F1F8710022524BF6F7ACFB48A3D3E9E0
:109B90000023F6F75FFD48A3D3E90023F6F7A4FB03
:109BA000804630468946F6F7EBFC45A3D3E900230F
:109BB000F6F750FD02460B4640464946F6F794FB41
:109BC00080468946F6F7F6FF00228346002340468A
:109BD0004946F6F7B1FF002840F07E82BBF1160F30
:109BE00000F26D82DDE90A013A4B03EBCB03D3E9C6
:109BF0000023F6F7A1FF002872D00023BE1B0E93AE
:109C0000731E0BF1FF3B069300F160820023099362
:109C1000BBF1000F6BDA099BCDF81CB0A3EB0B0373
:109C20000993CBF100030D93229B4FF0000B092BFE
:109C300066D8052B40F34A830026043B2293229BDF
:109C4000023B032B00F26C86DFE813F061045E0434
:109C50005504380442F20F73249ACAF3130A1360AE
:109C60005AEA08031AD1269B002B00F068861A4B8B
:109C700003930833269A0398136019B0BDE8F08F58
:109C8000DDE90A12C2F31303084643F07F510F9730
:109C9000A6F2FF36169F41F4401173E7269B002B76
:109CA00040F0EF830D4B039341E700BFAFF300801B
:109CB00061436F63A787D23FB3C8608B288AC63FD2
:109CC000FB799F501344D33F0000F07F15DE00085E
:109CD0000000F83F88DF00083CDE000838DE00089E
:109CE000BE1B731E069300F18A840E900990069B9A
:109CF0005B44CDE9063B00230D93229B092B98D9A9
:109D0000002322934FF0FF330126089300230C9683
:109D100023930021089B61641293204601F06EFE9C
:109D20000390002800F00486039B2364089B0E2BFD
:109D300000F21481002E00F011810799002940F3F0
:109D40006084AF4B01F00F0203EBC2030A46D3E974
:109D500000674FEA2118D10540F11784DDE90A01B7
:109D6000A84B4FF0030AD3E90823F6F79DFDCDE990
:109D7000100108F00F08B8F1000F13D0DFF884923B
:109D800018F0010F09D0D9E9002330463946F6F71B
:109D900061FC06460F460AF1010A5FEA680809F10C
:109DA0000809EDD1DDE9100132463B46F6F77CFDAE
:109DB000804689460E9B43B1002240464946924B5D
:109DC000F6F7BAFE002840F035855046F6F7D8FB86
:109DD00042464B46F6F73EFC8C4B0022F6F784FADF
:109DE000A1F15073CDE910011193089B002B00F0F5
:109DF0009780079B1493089B13930C9B002B00F0F8
:109E0000A984139A7E4B002003EBC20353E902237B
:109E10007F49F6F749FDDDE91023F6F763FACDE94E
:109E2000100149464046F6F7C5FE0746F6F7A8FB7F
:109E300002460B4640464946F6F754FADDE9102340
:109E4000039E303706F8017B80468946F6F774FE9C
:109E5000002840F02E85CDF854B00027DDE910AB86
:109E60001095139D13942AE00137AF4280F22E859E
:109E7000504659460022674BF6F7ECFB0022654B33
:109E800082468B4640464946F6F7E4FB89468046C3
:109E9000F6F790FE0446F6F773FB02460B46404683
:109EA0004946F6F71FFA303452465B4606F8014B36
:109EB00080468946F6F740FE002840F0F884424686
:109EC0004B4600205049F6F70DFA52465B46F6F72E
:109ED00033FE0028C8D0DDE91343109D039A079391
:109EE00002E0964200F0CD84B24616F8013D392BCF
:109EF000F7D00133DBB23370079B01330793C8E11E
:109F00005046F6F73DFB42464B46F6F7A3FB3F4B68
:109F10000022F6F7E9F9A1F15073CDE91001119390
:109F20004046494600223C4BF6F7DCF9DDE9108952
:109F30004B46424606460F46F6F71CFE8146002871
:109F400040F0AF84DDE91001024601F100433046E4
:109F50003946F6F7F1FD002840F04883179B002BA7
:109F6000C0F28C80079A0E2A00F38880244B03EB02
:109F7000C203D3E900AB239B002B1BDA089B002B09
:109F800018DC40F031830022234B50465946F6F747
:109F900061FB02460B46DDE90A01F6F7D7FDDDF865
:109FA00020904E46002800F0CA82239BDDF80C80EA
:109FB000DF43CCE25246DDE90A785B46384641464B
:109FC000F6F772FCF6F7F6FD81460990F6F7D8FA37
:109FD00052465B46F6F73EFB039E0B460246414661
:109FE0003846F6F77FF909F1300306F8013B089B84
:109FF000012B00F05F83069401271C4604952AE09C
:10A0000088DF000860DF00080000F03F00001C400F
:10A010000000E03F000024400000144052465B4630
:10A0200040464946F6F740FCF6F7C4FD0546F6F70C
:10A03000A7FA52465B46F6F70DFB01370B46024680
:10A0400049464046F6F74EF905F13003A74206F8B7
:10A05000013B00F02C830022AB4BF6F7FBFA002209
:10A06000002380468946F6F75DFD0028D6D0049D82
:10A07000069C079BB246013307930AE10C9A002A1B
:10A080003DD0229A012A40F39F82089B03F1FF38BA
:10A090000D9B4345C0F27082A3EB0808089B002B80
:10A0A000C0F24083069A1A440692099A17461A4447
:10A0B00009920121204601F06FFD064623E00123AD
:10A0C000BE1B0E93731E06937FF5A0ADC6F1010370
:10A0D0000993002306939BE55846F6F751FA42464A
:10A0E0004B46F6F71FFD00287FF478AD0BF1FF3BE0
:10A0F00074E5864B0393039819B0BDE8F08FDDF843
:10A100003480099F0C9E002F0CDD069900290B4618
:10A1100008DDB942A8BF3B46099AFF1AD21ACB1AEA
:10A12000099206930D9BE3B10C9B002B00F060821B
:10A13000B8F1000F10DD31464246204601F008FE1E
:10A1400006462A463146204601F054FD034629467C
:10A1500020461D4601F078FC0D9BB3EB080240F051
:10A16000DB820121204601F017FDBBF1000F814683
:10A1700000F3B380229B012B40F388814FF0000A4B
:10A180000120BBF1000F40F0B480069A104410F09B
:10A190001F0000F09280C0F12003042B40F3D38312
:10A1A000099BC0F11C000344024409930744069232
:10A1B000099B002B05DD29461A46204601F024FEA6
:10A1C0000546069B002B05DD49461A46204601F050
:10A1D0001BFE81460E9B002B40F03881089B002B14
:10A1E00040F31E810C9B002B40F09F80079B0133A6
:10A1F00007930127DDF80C80DDF820A007E0294651
:10A2000000230A22204601F029FC05460137494671
:10A210002846FFF7BBFB574500F1300308F8013B28
:10A22000EDDB089A0027002ACCBF93464FF0010BC4
:10A23000039A9344294601222046049301F0E4FD49
:10A240004946054601F056FE002840F3AB811BF855
:10A25000013C039A0BF1FF3B04E05A4500F0AD814D
:10A260001BF8013D392B0BF1010AF6D001338BF8B5
:10A2700000304946204601F0E7FB56B12FB1B74206
:10A2800003D03946204601F0DFFB3146204601F07D
:10A29000DBFB2946204601F0D7FB0023079A8AF80A
:10A2A0000030249B1A60269B002B3FF440AC03989F
:10A2B000C3F800A019B0BDE8F08F1C20099B07442B
:10A2C00003440993069B0344069371E70126B6E411
:10A2D000C0F1200008FA00F04DE401465A4620463D
:10A2E00001F036FD229B8146012B40F3B6814FF0F1
:10A2F000000AD9F8103009EB8303186901F000FC5B
:10A30000C0F1200041E700BF0000244014DE000837
:10A31000314600230A22204601F0A0FB129B06468C
:10A32000002B40F3E982CDE90783002F00F31D8164
:10A33000BAF1000F40F0D981B046049B089903F0B0
:10A340000102039B0A921F46013B1944229B08917C
:10A350001343099349462846FFF718FB31468346C5
:10A36000284601F0C7FD424649468246204601F094
:10A37000E1FDC26801460BF13003002A43D104908D
:10A380002846069301F0B6FD024604992046049241
:10A3900001F05AFB049A069B1AB90999002900F0AA
:10A3A0009B82BAF1000FC0F2648122994AEA010A45
:10A3B0000A9951EA0A0100F05C81002A00F3B68193
:10A3C000089A07F1010A9742D3463B7000F0B48126
:10A3D000294600230A22204601F040FB4645054657
:10A3E00031464FF000034FF00A02204612D001F030
:10A3F00035FB4146064600230A22204601F02EFB8B
:10A4000057468046A6E72046049301F01DFB012233
:10A41000049BC6E701F022FB57460646804699E7B3
:10A42000229B022B7ADC0C9B002B7FF47EAF079BD8
:10A430004946013328460793FFF7A8FADDF80CB028
:10A4400000F1300300270BF8013BF3E649462846AC
:10A4500001F050FD0028BFF6C1AE294600230A22B4
:10A46000204601F0FBFA079B054603F1FF380C9BE1
:10A47000002B7FF44DAF129B002B40F334820893E6
:10A48000B7E6B04B03930333FFF7F4BBDDE90412E7
:10A4900000297FF473AEC2F31303002B7FF46EAE7A
:10A4A000A94B1340002B00F00082099B4FF0010ADA
:10A4B00001330993069B0133069361E601230C9354
:10A4C000239B079A134412930133012B1F46B8BFF5
:10A4D000012708930021172F61647FF71EAC01222A
:10A4E00004235B0003F11400B842114602F101029B
:10A4F000F7D9616411E401230C93239B002B4CDDFD
:10A500001F4612930893E5E700230C93D8E7002336
:10A510000C93F2E7129BCDF81C800893089B002B4C
:10A520007FF443AD49460522204601F097FA814663
:10A530002846494601F0DEFC00287FF736AD31237E
:10A540000398079F804600F8013B01370390494676
:10A55000204601F079FA7B1CDDF80CA00793CDF8BA
:10A560000C80002E7FF491AE93E631463A462046A9
:10A5700001F04AFC0646DBE60D9BCDF83480A8EBE3
:10A5800003039B444FF0000888E5DDE90A234FF000
:10A59000020ACDE91023FFF7EEBB012323930893B2
:10A5A000FFF7B7BB03D1049BD8073FF550AEDA469F
:10A5B0001BF8013D302BFAD05BE6079B039A013371
:10A5C00007933123137054E60F9A002A00F0288174
:10A5D00003F23343069ADDF834801A440692099A4E
:10A5E00017461A44099264E54FF000094E46DCE430
:10A5F000294620460D9A01F0ABFB0546B1E50E90C9
:10A6000064E500F01181DDE90A01079A4F4B5642DB
:10A6100006F00F0203EBC203D3E90023F6F71AF8A2
:10A6200036118046894600F0708100234FF0020AFF
:10A63000474FF20706D5D7E90023F6F70BF80123B9
:10A640000AF1010A761007F10807F2D1002B3FF456
:10A65000B1AB80468946FFF7ADBB049B002B7FF46E
:10A6600046AEDDE90412C2F31303002B3FF418AF2A
:10A670003DE6002A12DD294601222046049301F01E
:10A68000C3FB4946054601F035FC0028049B40F316
:10A690001781392B00F0FB800BF13103BA46079A82
:10A6A00037460132464607920AF8013BE1E5099533
:10A6B000069C049D02460B46F5F716FE52465B4685
:10A6C00080468946F6F756FA60B952465B464046E0
:10A6D0004946F6F727FA00283FF4CBAC099BD90787
:10A6E0007FF5C7AC039AFFF7FFBB2046716801F006
:10A6F00085F90746002800F00C81336906F10C014A
:10A7000002339A000C30F5F773FD394601222046DA
:10A7100001F07AFB804610E62946204601F018FB3E
:10A7200005461EE5DDE908239F1AC2E4392B00F037
:10A73000AE80BA460133B2E7079A37460132464641
:10A74000079277E538DE00080000F07F88DF000818
:10A7500060DF0008DDF84CA08349DDE9102301EB40
:10A76000CA0151E90201F5F775FFCDE9100149462B
:10A770004046F6F71FFA0646F5F702FF0B4602467B
:10A7800049464046F5F7AEFD5346039F3036012B50
:10A790008046894607F8016B00F0AC80139E039B4E
:10A7A0001E440022714B40464946F5F753FF894647
:10A7B0008046F6F7FFF98246F5F7E2FE02460B46C1
:10A7C00040464946F5F78EFD0AF1300A07F801AB1D
:10A7D000B74280468946E4D1DDE910010022644B8E
:10A7E000F5F782FD42464B46F6F7A6F9002862D1FE
:10A7F000DDE9102300205E49F5F774FD42464B4623
:10A80000F6F7B8F900283FF4A9AB16F8013CB246B8
:10A81000302B06F1FF36F8D0149B0133079338E54F
:10A82000169BC3F13603D5E64FF0020ADDE90A892B
:10A83000FFF7C0BA089B002B3FF462AB129B002BC2
:10A840007FF78CAB1393079B0022013B40464946A0
:10A850001493464BF5F7FEFE804689460AF1010047
:10A86000F5F78EFE42464B46F5F7F4FE414B0022CB
:10A87000F5F73AFDA1F15073CDE910011193FFF7FF
:10A88000BCBA079B013307933123FFF734BB079B07
:10A89000BB4601330793392337460BF8013B464645
:10A8A000D7E44FF000094E4649E69A4668E4109D09
:10A8B000139CB246B0E7149B039A0793FFF714BBAF
:10A8C0007FF4ECAEDA077FF5E9AEE2E6DDF854B0EE
:10A8D000109D139CFFF742BB392BD8D0BAF1000F63
:10A8E0003FF7DAAEDAE6229B022B3FF713AECDF844
:10A8F0001C809CE53E466FE7229B022B3FF70AAE89
:10A90000129BCDF81C8008930FE54FF0020AFFF769
:10A9100051BA024640F2EA21174B184802F0FAFDFC
:10A92000002620463146666401F068F8039078B945
:10A9300000224FF4D571104B104802F0EBFD104B84
:10A940000393FFF7F4B83FF433ACC0F13C00B5E437
:10A95000039B012223644FF0FF33239612930C9242
:10A960000893FFF7FBBA00BF88DF0008000024400F
:10A970000000E03F00001C4048DE00085CDE0008EC
:10A980003CDE0008B1F90C20F8B50C46110707466B
:10A9900043D4636842F40062002BA2815BDDA56AA8
:10A9A000002D56D000233E683B6093B212F48052D3
:10A9B00055D101233846E169A847421C65D0A389D7
:10A9C000A56A5B0705D56368C01A236B0BB1E36BFF
:10A9D000C01A0246E16900233846A847411C40D10D
:10A9E0003B68002B3DD01D2B01D0162B54D10022EB
:10A9F000A38923F40063A3812369C4E90032216B96
:10AA00003E6031B304F14003994202D0384600F071
:10AA100061F9002318462363F8BD2669CEB193B2CD
:10AA20009A0718BF0023256808BF63692660AD1B1D
:10AA3000A3600CE02B463246D4F824C03846E169C6
:10AA4000E047B0F1000CA5EB0C05664416DD002DC7
:10AA5000F0DC0020F8BDE36B002BA0DCF9E7206DF3
:10AA6000AFE70022B4F90C30626023F4006322697E
:10AA7000A381DB042260C2D52065C0E7A3894FF023
:10AA8000FF3043F04003A381F8BD3B68002B96D014
:10AA90001D2B06D0162B04D0A38943F04003A381BD
:10AAA000F8BD00203E60F8BD38B505460C4608B13B
:10AAB000836BA3B1B4F90C00B8B1636EDB0701D4AA
:10AAC000810515D528462146FFF75CFF636E0546D4
:10AAD000DA0702D4A3899B050ED5284638BD00F0BD
:10AAE00017F8B4F90C000028E7D10546284638BD10
:10AAF000A06D00F093FBE5E7A06D00F091FB284608
:10AB000038BD00BF014900F05DBB00BFF1D50008B2
:10AB10002DE9F0478246394800F080FBDAF83840EA
:10AB2000002C66D1042303223549DAF80450CAF810
:10AB30003C10DFF8D090DFF8D080344F344E0AF567
:10AB40003B71CAE9B921CAF8E0422146EB6008220C
:10AB5000C5E90044C5E904446C66AC60AC6105F12C
:10AB60005C00FCF731FFC5E90759C5E90987EE62CA
:10AB700005F1580000F04EFBDAF80850254B21464D
:10AB8000EB600822C5E90044C5E904446C66AC608A
:10AB9000AC6105F15C00FCF717FFC5E90759C5E991
:10ABA0000987EE6205F1580000F034FBDAF80C502A
:10ABB000194B2146EB600822C5E90044C5E904446D
:10ABC0006C66AC60AC6105F15C00FCF7FDFE05F164
:10ABD0005800C5E90759C5E90A76C5F8248000F090
:10ABE00019FB01230548CAF83830BDE8F04700F0EA
:10ABF00017BB0248BDE8F04700F012BBF09F0020F1
:10AC000005AB0008B5C50008D9C5000819C600087D
:10AC100039C600080900010012000200014800F0D6
:10AC2000FDBA00BFEC9F0020014800F0F9BA00BF58
:10AC3000EC9F0020F8B50C46234F064600F0D2FEEC
:10AC4000BB685D68C4F57E6325F003050F332B44B4
:10AC500023F47F6323F00F03A3F58054B4F5805FE2
:10AC600007DB0021304601F093FCBB682B4498427F
:10AC700004D0304600F0BCFE0020F8BD30466142F2
:10AC800001F086FC01300DD0104ABB682D1B45F049
:10AC900001055D60136830461B1B136000F0A8FEC1
:10ACA0000120F8BD0021304601F072FCBA68831A19
:10ACB0000F2BDEDD43F001035360054B03491B6896
:10ACC000C01A0860D5E700BFC0040020F49F002030
:10ACD000C808002000295ED0F8B50C46064600F0F2
:10ACE00081FE54F8042C784FA4F1080522F00101EC
:10ACF0006818D7F808C04368844523F0030300F0C0
:10AD00008780D207436034D454F8082C07F1080434
:10AD1000AD1A1144AA68A24268D000EB030CDCF81B
:10AD200004E0D5F80CC01EF0010FC2F80CC0CCF83E
:10AD3000082000F0918041F001036B600160B1F5E3
:10AD4000007F31D24A09CB08012191407A68013352
:10AD50001143796007EBC30257F83310083AC5E98D
:10AD6000021247F83350CD603046BDE8F84000F09D
:10AD70003FBEC2185268D2070ED4194407F1080426
:10AD80008368A34270D0C268DA60936041F0010327
:10AD90006B606950D3E7704741F00103B1F5007F64
:10ADA00044F8043C0160CDD3B1F5206F4FEA512344
:10ADB00047D28B0903F1390003F13802C300F818B8
:10ADC000FB580838984258D05A6822F003028A4249
:10ADD00002D99B689842F7D1D868C5E902308560EE
:10ADE0003046DD60BDE8F84000F002BEC21852688F
:10ADF000D20763D40B44D0E90212CA60916043F0D9
:10AE000001026A603046EB50BDE8F84000F0F0BD4A
:10AE10000B44D10707D454F8082CAD1A1344D5E9D4
:10AE20000212CA60916043F001026A60274ABD6065
:10AE300012689A4298D8264B30461968FFF7FAFEF6
:10AE400092E7142B0AD9542B1FD80B0B03F16F0078
:10AE500003F16E02C300B2E7194491E703F15C000D
:10AE600003F15B02C300AAE741F00103C7E90455FF
:10AE7000C5E902446B60695076E70121921001FA3E
:10AE800002F279680A437A60A7E7B3F5AA7F06D889
:10AE9000CB0B03F1780003F17702C3008FE740F298
:10AEA0005452934206D88B0C03F17D0003F17C02CF
:10AEB000C30084E74FF47E737E2280E741F00103F4
:10AEC0006B60016050E700BFC0040020CC08002088
:10AED00024A000209368002B00F0B7802DE9F04FEC
:10AEE000B1F90C300C4619078046174683B098B26A
:10AEF00025D523691BB310F002033D682DD04FF018
:10AF0000000B5E46DFF8B8A2002E00F08B8056459D
:10AF100033465A4628BF53464046E169D4F824C018
:10AF2000E047002840F38780BB6883441B1A361A29
:10AF3000BB60002BE8D1002003B0BDE8F08F2146B4
:10AF40004046FEF7B9FC002840F03681B4F90C30D9
:10AF50003D6898B210F00203D1D110F0010976D10A
:10AF60004E46002E5AD08205D4F808B040F1B58084
:10AF7000B3455A4600F2CD8010F4906F00F0CB80BC
:10AF800023682169A3EB010B636903EB430A0AEB16
:10AF9000DA7A0BF101034FEA6A0A33445345524609
:10AFA00084BF9A465246430540F1EA801146404626
:10AFB00000F0A8F9002800F0F9805A4621690190B4
:10AFC000F5F716F9A289019B22F4906242F0800203
:10AFD000A28103EB0B0023613246AAEB0B03B346BD
:10AFE000C4F814A0A3602060B2460026494601922E
:10AFF00000F07CFCA3682168019AA3EB0B030A44D0
:10B00000A3602260B868D144A0EB0A00B8600028B1
:10B0100091D0B4F90C0080B2002EA4D1D5E90096ED
:10B0200008359EE7D5E900B608356DE7214640466C
:10B03000FFF73AFD80B3B4F90C304FF0FF3043F026
:10B040004003A38103B0BDE8F08F002070471E4687
:10B05000AA46994618461D4656B3002832D04A469D
:10B0600020682169B24228BF32468842636904D908
:10B07000A16803EB010B5A4574DC934265DC2A4658
:10B080004046E169D4F824C0E047B0F1000BD2DDBE
:10B09000B9EB0B09CAD00120BB685D44A3EB0B03DD
:10B0A000A6EB0B06BB60002B3FF445AF002ED4D1BE
:10B0B0000AF1080353F8046C9A4653F8085C083305
:10B0C000002EF7D032460A21284600F0C7FB0028A0
:10B0D00069D00130A0EB0509C1E7206823699842D7
:10B0E0001BD86369B34218D86FF0004CB44528BF31
:10B0F000B4469CFBF3FC4A4603FB0CF34046E16973
:10B10000D4F824C0E047B0F1000A94DDA6EB0A06AB
:10B1100078E7B3463246206866E7B345DA4628BF8B
:10B12000B2464946524600F0E1FBA3682268A3EB11
:10B130000A035244A3602260002BE7D12146404617
:10B14000FFF7B2FC0028E1D075E72946934601924B
:10B1500000F0CCFBA368019A9B1AA36023681A44F1
:10B16000226095E729465A4600F0C0FB2368214635
:10B170005B4440462360FFF797FC002888D05AE7DD
:10B18000404600F0DFFF034600287FF422AF404630
:10B190002169FFF79FFD0C22B4F90C30C8F800209C
:10B1A00023F0800349E7721C914659E70C22B4F959
:10B1B0000C30C8F8002040E74FF0FF30BCE600BF7D
:10B1C00000FCFF7F2DE9F8434FF000090746884651
:10B1D00000F53876D6E90154013D10D4A389013D2C
:10B1E000012B08D9B4F90E30013304D0214638467A
:10B1F000C04749EA00096B1C04F16804EED13668C7
:10B20000002EE7D14846BDE8F88300BF00487047EC
:10B21000C0090020704700BF704700BF704700BFE3
:10B22000704700BF2DE9F0418B890C46990796B015
:10B2300008D5012204F14303C4E90432236016B0A7
:10B24000BDE8F081B4F90E100646002927DB6A46F6
:10B2500002F0CCFA002821DB019D4FF4806805F450
:10B260007045A5F50055B5FA85F54FF400676D09F1
:10B270004146304600F046F8B4F90C30F0B1204AAF
:10B2800043F08003F263C4F81480A381206020613E
:10B2900035BB3B43A38116B0BDE8F081A38913F011
:10B2A000800519D04FF0400830464146002500F097
:10B2B00029F82F46B4F90C300028E0D19A05BED405
:10B2C000012123F0030304F1430243F00203C4E924
:10B2D0000421A3812260B2E74FF480682F46C7E7BC
:10B2E0003046B4F90E1002F095FA10B9B4F90C30EA
:10B2F000CFE7A38923F0030343F001031BB2C8E7A0
:10B3000005AB00082DE9F04F01F10B05162D06469F
:10B3100083B025D8102900F2B88000F063FB102517
:10B3200018224FF0020CB54F3A445368A2F10801BD
:10B330008B4200F0B7805A68D96822F003021A44A1
:10B340009C683046E1608C60516803F1080441F06C
:10B350000101516000F04CFB204603B0BDE8F08FC6
:10B3600035F0070500F19180A94200F28E8000F0CF
:10B3700039FBB5F5FC7FC0F094816B0A00F08C803E
:10B38000042B00F26A81AB0903F1390C03F1380494
:10B390004FEACC00994F384443680838984206D1A8
:10B3A0000CE0002980F22681DB68984206D05A68BA
:10B3B00022F00302511B0F29F3DDA4463C69DFF89C
:10B3C00040E274457AD0626822F00302531B0F2BCF
:10B3D00000F37681002BC7E904EE80F26781B2F5B5
:10B3E000007F80F019810121D30852090B4491405C
:10B3F0007A6857F833000A4307EBC3010839A060A5
:10B40000E1607A6047F83340C46001214FEAAC0341
:10B410009940914259D8114206D12CF0030C4900B1
:10B4200011420CF1040CFAD007EBCC0948466446F3
:10B43000D0F80C80404508D11CE1002B80F221811E
:10B44000D8F80C80404500F01581D8F8042022F08F
:10B450000302531B0F2BF0DD08EB050145F001053E
:10B46000C8F804503046D8E90264F460A66043F09E
:10B470000104C7E904114C60C1E902EE48F802304A
:10B4800000F0B6FA08F1080402E00C23002433604F
:10B49000204603B0BDE8F08F4FF400704FF0400C31
:10B4A0003F2477E7D3689A4208BF0CF1020C7FF47F
:10B4B00042AF3C69DFF848E1744584D101217A68E4
:10B4C0004FEAAC0399409142A5D9BC68636823F068
:10B4D00003094D4503D8A9EB05030F2B7ADCDFF8F0
:10B4E00024B1494BDBF800201B6801322B4404EBEC
:10B4F000090A00F02F8103F580530F3323F47F688E
:10B5000028F00F084146304601F042F8411C02463F
:10B5100000F0EF80824500F2EA803C4B196841441C
:10B520000846196000F04981DBF8001001930131F1
:10B530001BBFA2EB0A0A5044CBF80020186012F09F
:10B54000070B00F01181CBF108010A44CBF58051C3
:10B5500090440831A1EB0801C1F30B0A5146304673
:10B56000009201F015F8421CDDE9002300F04B8148
:10B57000801A00EB0A08196848F001005144BC42E7
:10B58000BA601960506000F02481B9F10F0F40F2E9
:10B5900022814FF0050E6068A9F10C0C2CF0070C0D
:10B5A00000F0010040EA0C006060BCF10F0F04EBFA
:10B5B0000C00C0E901EE00F22E8114465068144BD5
:10B5C0001A688A4238BF1960124B1A688A4238BF1B
:10B5D000196090E0621943F0010345F001056560D0
:10B5E0003046BA600834536000F002FA204603B0D7
:10B5F000BDE8F08FD9681A44A2E600BFC00400205D
:10B60000C8040020C808002024A00020F49F0020C7
:10B610001CA0002020A00020B2F5206F4FEA52238A
:10B620005FD3142B00F2B18003F15C01C9005B33DE
:10B63000781879580838884200F08F804B6823F0DA
:10B640000303934202D989688842F7D1C8687A68AF
:10B65000C4E902108460CC60D7E6142B59D9542B6E
:10B6600000F29B802B0B03F16F0C03F16E044FEA89
:10B67000CC008FE60134A30700F108007FF4D8AEB8
:10B6800053E0444642445368D8F80C1043F0010399
:10B69000536054F8083F3046D9608B6000F0A8F939
:10B6A000F6E64FEAD50C05F108023CE62244536861
:10B6B000304643F00103536000F09AF90834E7E69E
:10B6C000611945F00105656043F00105C7E9041102
:10B6D0003046C1E902EE4D60A35000F089F908340C
:10B6E000D6E6930903F13901C9003833A0E7BC421B
:10B6F0005ED0BC68606820F003084545A8EB0503F0
:10B7000002D80F2B3FF766AF304600F071F90024E6
:10B71000BEE603F15C0C03F15B044FEACC0039E6B2
:10B7200059F808394B4540F095801CF0030F0CF197
:10B73000FF3CF5D17B6823EA01037B604900994215
:10B740003FF6C3AE11B9C0E6490004341942FBD03C
:10B75000A44669E603F11008D4E601229B109A4042
:10B760007B681A437A6073E702EB08014942C1F330
:10B770000B0A51463046009200F00AFF431CDDE9F7
:10B7800000237FF4F5AEDA46F5E6542B26D8130BEA
:10B7900003F16F01C9006E334AE7B3F5AA7F26D8DB
:10B7A000EB0B03F1780C03F177044FEACC00F1E5E1
:10B7B000294B186840441860B6E6CAF30B0CBCF17C
:10B7C000000F7FF4B1AEBC68C84448F0010060606F
:10B7D000F5E61446F3E60123536095E7B3F5AA7F37
:10B7E00024D8D30B03F17801C900773320E740F266
:10B7F0005452934224D8AB0C03F17D0C03F17C042A
:10B800004FEACC00C6E5ABF1080BD8444FF0000A74
:10B81000A8EB0208AFE604F1080130460093FFF7F9
:10B8200059FABC68009B60681968C8E640F2545138
:10B830008B420BD8930C03F17D01C9007C33F7E6F2
:10B840004FF47E704FF07F0C7E24A3E54FF47E71A1
:10B850007E23EDE67B6871E7F49F00205FFA81FCB0
:10B86000810710D00346511E2AB90AE09A071846EC
:10B870000AD0013905D3184613F8012B6245F5D1DA
:10B88000704700207047114603290CD80029F8D0D2
:10B890000346014401E08B42F3D0184613F8012B14
:10B8A0006245F8D1ECE7024610B54CEA0C2444EAB4
:10B8B00004441046036804326340A3F1013E2EEABB
:10B8C000030313F0803F04D1043903291046F0D854
:10B8D00051B10346014401E08B4205D0184613F8EC
:10B8E000012B6245F8D110BD002010BD88420DD952
:10B8F0008B1883420AD900EB020CBAB1624613F8E6
:10B9000001CD994202F801CDF9D170470F2A0ED826
:10B91000034602F1FF3C4AB10CF1010C013B8C449F
:10B9200011F8012B614503F8012FF9D1704740EA66
:10B9300001039B074FD1A2F1100370B501F1200C58
:10B9400023F00F0501F1100E00F11004AC441B09A7
:10B950005EF8105C0EF1100E44F8105C5EF81C5C92
:10B96000103444F81C5C5EF8185C44F8185C5EF80F
:10B97000145CE64544F8145CEAD1013312F00C0F74
:10B9800001EB031102F00F0400EB031327D08E46E6
:10B99000043C24F003064FEA940C1E441C1F5EF87E
:10B9A000045B44F8045FB442F9D10CF1010402F0E5
:10B9B000030203EB840301EB840102F1FF3C4AB173
:10B9C0000CF1010C013B8C4411F8012B614503F88B
:10B9D000012FF9D170BD034602F1FF3C9CE72246DE
:10B9E000EBE700BF0148FFF719BC00BFE89F00204C
:10B9F0000148FFF715BC00BFE89F002038B5C36CB5
:10BA000005460C464BB153F8240080B1026843F858
:10BA100024200023C0E9033338BD2122042101F092
:10BA200099FD0346E8640028EDD1002038BD0121CE
:10BA3000284601FA04F56A1D920001F08BFD0028EA
:10BA4000F3D0C0E90145E4E731B1C36C4A6853F86B
:10BA50002200086043F82210704700BF2DE9F04132
:10BA60004FF0000E0E461C460D69074601F114000A
:10BA700001680EF1010E8BB202FB0343090C4FEA81
:10BA8000134C02FB01CC9BB203EB0C43754540F811
:10BA9000043B4FEA1C44EBDC3CB1B368AB4207DD2E
:10BAA00006EB850301355C6135613046BDE8F08108
:10BAB000716838460131FFF7A1FF8046A8B13269AD
:10BAC00006F10C01023292000C30F4F791FBFB6C92
:10BAD000726853F82210316043F82260464606EB44
:10BAE000850301355C613561DFE70246B521024B14
:10BAF000024801F00FFD00BF48DE0008DCDE000850
:10BB0000020C12040346CAB91020834013F07F4F81
:10BB100004BF1B02083013F0704F04BF1B01043038
:10BB200013F0404F04BF9B000230002B05DB13F0E5
:10BB3000804F00F1010008BF202070470020E5E79A
:10BB40000368024613F0070009D0D9071FD49807ED
:10BB50004BBF5B089B08012002201360704799B21D
:10BB600009B91020C340D9B209B908301B0A190716
:10BB700004BF1B090430990704BF9B080230D90792
:10BB800003D45B0800F1010003D01360704700206C
:10BB900070472020704700BF38B5C36C04460D467F
:10BBA0004BB15868B0B102685A6000220123456168
:10BBB000C0E9032338BD2122042101F0CBFC034658
:10BBC000E0640028EDD100224FF4A071074B084833
:10BBD00001F0A0FC1C220121204601F0BBFC002842
:10BBE000F1D001220223C0E90123DEE748DE00088C
:10BBF000DCDE00082DE9F04F0E6915698846AE427B
:10BC0000144685B005DB2A46234635460C461646C3
:10BC10009846A3686168AF19BB42B8BF0131FFF70E
:10BC2000EDFE0190002800F08780019B03F11409CC
:10BC300009EB870AD14505D24B46002243F8042B75
:10BC40009A45FBD808F1140808EB860B04F114039D
:10BC5000D8451A4603EB85055FD22B1B153B23F015
:10BC6000030304331534A54238BF0423CDE902A7EA
:10BC7000AC461F46924605E0000C29D1C34509F1A8
:10BC8000040948D958F8040B85B2002DF4D0564663
:10BC90004C46002356F8040B216882B21FFA81FE3D
:10BCA00005FB02EE000C0A0C05FB0022734402EBBC
:10BCB00013429BB243EA0243B44544F8043B4FEAC3
:10BCC0001243E7D849F8073058F8040C000CD5D0D7
:10BCD000D9F80030544619464D4600222688090CF2
:10BCE00000FB06119BB20A4443EA024345F8043BB9
:10BCF00054F8046B2968360C8BB200FB0633A4455C
:10BD000003EB12434FEA1342E8D8C34549F8073022
:10BD100009F10409B6D8DDE902A7002F02DC05E02D
:10BD2000013F03D05AF8043D002BF9D0019B18467F
:10BD30001F6105B0BDE8F08F024640F25D11024B75
:10BD4000024801F0E7FB00BF48DE0008DCDE000827
:10BD500012F003032DE9F041144607462ED10E469A
:10BD6000A4101CD0BD6C95B3E3074FF0000806D4B7
:10BD7000641014D02868A8B10546E307F8D52A4610
:10BD800031463846FFF736FFB6B17168FB6C641078
:10BD900053F82120326043F821600646EAD130464C
:10BDA000BDE8F0812A4629463846FFF723FF286080
:10BDB0000546C0F80080E0E70646D9E70F4A013B98
:10BDC00052F823200023FFF749FE0646C8E7012169
:10BDD0003846FFF713FE054640B140F271230122B9
:10BDE000C0E904230023B8640360BDE702464FF4B2
:10BDF000A071034B034801F08DFB00BF50E0000829
:10BE000048DE0008DCDE00082DE9F0470C46266914
:10BE1000A36806EB6216751C9D429046074649686A
:10BE20004FEA621904DD5B009D4201F10101FADC79
:10BE30003846FFF7E3FD002851D0B9F1000F00F1BB
:10BE400014010FDD0B464FF0000C09F105024FEA1B
:10BE5000820E00EB820243F804CB9342FBD1AEF199
:10BE600014031944226904F1140318F01F0803EBAA
:10BE7000820C2CD08E464FF0000AC8F120091A68B7
:10BE800002FA08F242EA0A024EF8042B53F8042B95
:10BE90009C4522FA09FAF2D8ACEB0403153B23F0D7
:10BEA0000303043304F11502944538BF0423BAF1A7
:10BEB000000F18BF2E4641F803A0FB6C62680661B4
:10BEC00053F82210216043F82240BDE8F08704397E
:10BED00053F8042B9C4541F8042FF9D8EDE70246AE
:10BEE00040F2D911014B024801F014FB48DE000872
:10BEF000DCDE000884460B690069C01A15D10CF11C
:10BF0000140C14310CEB830210B401EB830301E039
:10BF1000944508D252F8044D53F8041D8C42F7D0D2
:10BF200004D24FF0FF3010BC70477047012010BCA6
:10BF3000704700BF2DE9F84F0C6913698946E41A70
:10BF4000002C17467DD101F11406143202EB830256
:10BF500006EB830301E09E4276D253F8045D52F86B
:10BF6000041D8D42F7D067D3D9F80410FFF746FDC2
:10BF7000002873D0D9F81050C46000F1140426468C
:10BF80004FF0000A3B6909F1140807F1140E09F19A
:10BF9000100C08EB85020EEB83095CF804BF5EF819
:10BFA000041B1FFA8BF353441FFA81FA090CA3EB0D
:10BFB0000A03C1EB1B4101EB23419BB243EA01435E
:10BFC000F14546F8043B4FEA214AE6D8A9EB0701C0
:10BFD00015391537B94521F0030606F1040638BFB7
:10BFE000042621F0030138BF0021B0444245264415
:10BFF0000C4418D93746444654F8041B8BB25344BA
:10C000004FEA234A0AEB11419BB243EA0143A242A1
:10C0100047F8043B4FEA214AEED8541EA4EB08042B
:10C0200024F00304344423B954F8043D013D002BAB
:10C03000FAD00561BDE8F88F4B460124B9461F468A
:10C0400092E7F9DB00248FE70021FFF7D7FC60B10E
:10C0500001220023C0E90423BDE8F88F02464FF413
:10C060001071054B054801F055FA024640F23221A5
:10C07000014B024801F04EFA48DE0008DCDE000801
:10C0800070B5012182B016461D46FFF7B7FC044685
:10C0900000284CD02B46C5F30A55C3F313030DB14A
:10C0A00043F48013002E019322D068460096FFF7D8
:10C0B00047FD002837D0019B0099C0F1200203FA08
:10C0C00002F20A43C34001936261002B14BF0221B4
:10C0D0000121A3612161B5B1069BA5F23345054459
:10C0E0001D60079BC0F135001860204602B070BD8E
:10C0F00001A8FFF725FD0123019A1946626120304E
:10C100002361002DE8D104EB8102A0F232431069D3
:10C11000069A1360FFF7F4FCC0EB41112046079B21
:10C12000196002B070BDDDE900236261CDE702460F
:10C1300040F20A31014B024801F0ECF948DE0008F8
:10C14000DCDE00082DE9F84F1646002900F0988043
:10C1500006F10B0580460C46FFF744FC162D5DD812
:10C1600010252A46AE425ED854F8041CA4F10809F2
:10C1700021F00307974262DABC4B09EB0700D3F8C2
:10C1800008C0844500F09780D0F804C02CF001036B
:10C1900003445B68DB0768D42CF0030C07EB0C034B
:10C1A000934247DACB0710D454F8083CA9EB030AB2
:10C1B000DAF8043023F003018C44BC44944580F247
:10C1C00011817B18934280F2E88031464046FFF7A8
:10C1D00099F80646E0B154F8043CA0F1080223F0B7
:10C1E00001034B44934200F0D2803A1F242A00F20C
:10C1F000F580132A00F2AC800346224611681960CC
:10C200005168596092689A6021464046FEF762FD87
:10C210004046FFF7EDFB3046BDE8F88F25F00705F7
:10C22000002D2A469EDA0C230026C8F8003030463E
:10C23000BDE8F88F1F46D0E90223D3609A607B1BCC
:10C240000F2B22D8D9F8043003F001033B43C9F87F
:10C2500004304F447B6843F001037B602646404630
:10C26000FFF7C6FB3046BDE8F88FC907ADD454F8D8
:10C27000083CA9EB030ADAF8041021F00301A0E757
:10C280001146BDE8F84FFFF73DB8D9F8041043F068
:10C29000010301F001012943C9F8041009EB05016C
:10C2A0004B604F447B68404643F0010308317B609C
:10C2B000FEF710FDD2E7DCF8040020F0030B07EBDB
:10C2C0000B0C05F1100084454DDAC9073FF57DAF31
:10C2D00054F8081CA9EB010ADAF8041021F0030154
:10C2E0008B44BB4458453FF76CAF5646DAF80C1008
:10C2F00056F8080F3A1F242AC160886000F2DB80DC
:10C30000132A40F2D68021681B2ACAF808106168F7
:10C31000CAF80C1000F2E08008340AF1100221681B
:10C32000116061685160A1689160ABEB05020AEB96
:10C33000050142F0010299604A60DAF80430404693
:10C3400003F001031D43CAF80450FFF751FB6EE7E9
:10C3500023681B2A03606368436068D804F10802FD
:10C3600000F108034AE709EB0502ACEB050C9A6003
:10C370004CF00103536054F8043C404603F00103C1
:10C380001D4344F8045CFFF733FB26464FE750F8A3
:10C39000043C23F003031F4451E75646DAF80C101F
:10C3A00056F8080F3A1F242AC16088604CD8132A17
:10C3B00048D921681B2ACAF808106168CAF80C100D
:10C3C00056D808340AF110021F462368D14613607C
:10C3D00063685360A3683446936030E72146FFF7F3
:10C3E00085FA11E75646D0E90213CB60996056F8FA
:10C3F000081FDAF80C303A1F242ACB6099602DD838
:10C40000132A29D923681B2ACAF808306368CAF896
:10C410000C3042D808340AF11003226867461A60CB
:10C420006268D1465A60A26834469A6007E7A368FA
:10C43000242A8360E368C36026D004F1100200F16F
:10C440001003DBE63246BFE7214630461F46D146A1
:10C45000FFF74CFA3446F2E63346DEE72146304633
:10C460006746D146FFF742FA3446E8E6C0040020AA
:10C47000A168242ACAF81010E168CAF8141020D064
:10C4800010340AF118029FE7236904F118020361CE
:10C490006369436100F11803B0E6A368242ACAF86F
:10C4A0001030E368CAF8143022D010340AF11803AF
:10C4B000B3E7324633E721463046FFF717FA174B0A
:10C4C00033E722691834CAF8182054F8042CCAF843
:10C4D0001C200AF1200277E7A168242ACAF810106C
:10C4E000E168CAF814100ED010340AF1180216E7E9
:10C4F00023691834CAF8183054F8043CCAF81C30C0
:10C500000AF1200389E722691834CAF8182054F880
:10C51000042CCAF81C200AF1200200E7C004002005
:10C52000F8B50027DFF85CC021F0004363450446FE
:10C530000D46176023DC844653EA0C0C1FD0DFF84D
:10C5400048C0164601EA0C0C0A46BCF1000F09D19E
:10C5500000220E4BF4F77EF86FF0350704460A46CA
:10C5600021F0004322F0FF421B1522F4E002A3F267
:10C57000FE333B4442F07F55336045F400152046BE
:10C580002946F8BDFFFFEF7F0000F07F0000504319
:10C59000002238B5064D044608462A60F6F7DEF854
:10C5A000431C00D038BD2B68002BFBD0236038BD66
:10C5B000E49F002010B50C46B1F90E1001F06EF9A1
:10C5C000002803DB236D0344236510BDA38923F4F6
:10C5D0008053A38110BD00BF2DE9F0410C46B1F995
:10C5E0000C101F46CB05054616460BD421F480518E
:10C5F000A1813B4632462846B4F90E10BDE8F04111
:10C6000000F072BFB4F90E100223002201F01AF9F3
:10C61000B4F90C10EAE700BF10B50C46B1F90E10E2
:10C6200001F010F9A389421C0EBF23F4805343F498
:10C6300080532065A38110BDB1F90E1000F0C6BF74
:10C640002DE9F84F4B6E90469C042DD593681268E7
:10C6500043B38B46064602F1080959E9025A5FEADC
:10C660009A0715D00024043D01E0A7420ED05A4697
:10C67000304655F8041F01F085F8431C04F101040D
:10C68000F3D10023C8E90133BDE8F88FD8F80830AA
:10C690002AF0030AA3EB0A03C8F8083009F10809D5
:10C6A000002BDAD10020ECE7FEF714FC0023C8E9E8
:10C6B0000133BDE8F88F00BF10B4946814B110BC0A
:10C6C000FFF7BEBF2046546010BC70472DE9F04F05
:10C6D000BDB01C461746CDE90530029118B1836BF9
:10C6E000002B00F07782029A536EDE0740F18481BE
:10C6F000B2F90C108AB2900408D441F400520299A5
:10C700004B6E8A8123F4005392B24B66110740F1BD
:10C71000EC80029B1B69002B00F0E78002F01A03FB
:10C720000A2B00F0F08013AB10930023CDE91133F6
:10C73000CDE90933CDE90B330DF14C0904933B7876
:10C74000002B00F046813C4604E014F8013F002B2A
:10C7500000F02181252BF8D1E51B40F01E812378C4
:10C76000002B00F036814FF0000300254FF0FF3B17
:10C770004FF02B088DF83B3063780395671C013729
:10C78000A3F120025A2A00F24681DFE812F0A1024A
:10C79000440144019D024401440144017C024401DE
:10C7A00044016A00530244012902AF024401AB0272
:10C7B0005B005B005B005B005B005B005B005B00A1
:10C7C0005B0044014401440144014401440144012B
:10C7D000440144011302780044014401440144012E
:10C7E000440144014401440144014401D100440195
:10C7F00044014401F701440141024401440121057F
:10C800004401440144014401440144014401440100
:10C810004401440113027A004401440144013702F7
:10C820007A00740044012D0244016902D3005702CA
:10C8300074004401F70172004105440144014305BD
:10C84000440172000021A3F1300217F8013B01EB13
:10C85000810102EB4101A3F13002092AF5D90391CC
:10C860008EE7059B53F8042B002A03920593C0F230
:10C87000B4813B7883E73B7845F020057FE745F0BE
:10C880001005AC06059E40F16B81073626F00706C1
:10C890003246736852F8086B98460592002BC0F236
:10C8A0004984BBF1FF3F00F0318556EA080325F0CB
:10C8B000800A00F025840A2E78F1000380F0E184DC
:10C8C0000123554630368DF8EF6001930DF1EF04EA
:10C8D000DDF804809DF83B30D845B8BFD846002B22
:10C8E00000F0A88008F10108A4E0029D06982946FE
:10C8F000FCF7E2FF002840F09485AA8902F01A03B1
:10C900000A2B7FF410AF0299B1F90E30002BFFF61D
:10C910000AAF4B6EDE0702D4950540F162852346CF
:10C920003A46029906983DB0BDE8F04F00F09ABD36
:10C9300045F0100515F0200800F00381059E07362C
:10C9400026F007063346D6F8048053F8086B0593A3
:10C95000002325F4806A4FF000028DF83B20BBF1E4
:10C96000FF3F00F0DD8156EA08022AF0800540F022
:10C97000D681BBF1000F40F0CC84002B40F0C58382
:10C980001AF00103019300F0EC8330230DF1EF0462
:10C990008DF8EF309CE7E51B1BD0119B129A0133F9
:10C9A0002A44072BC9E900751292119305DC09F19D
:10C9B0000809049B2B440493D1E6002A00F09C83D1
:10C9C0000299069810AAFFF73BFE40B90DF14C09F9
:10C9D000EFE7129B002B40F0158500231193029A7C
:10C9E000536ED90740F1A28093895B0600F125853B
:10C9F00004983DB0BDE8F08F029BB3F90C108D0593
:10CA00008AB23FF578AE1D46986DFEF707FCB5F982
:10CA10000C108AB26FE6002BDBD04FF001088DF8C6
:10CA20008C304FF0000323AC8DF83B30CDF8048000
:10CA30004FF0000B15F00203079318BF08F102082E
:10CA400015F08403089305D1039BA3EB0806002E81
:10CA500000F38A82DDE91112481C9DF83B6076B133
:10CA6000012101320DF13B060728CDE91102C9E988
:10CA7000006100F35882014609F108090130079B63
:10CA8000D3B102230232C9F8043007280FABCDE935
:10CA90001102C9F8003040F36282002A00F02783B7
:10CAA0000299069810AAFFF7CBFD002897D1DDE97F
:10CAB00011120DF14C09481C089B802B00F071816C
:10CAC000019BABEB0306002E00F3CF81019B0728EF
:10CAD0001A44CDE91102C9F80040C9F8043040F306
:10CAE0005D81002A00F093820299069810AAFFF750
:10CAF000A7FD00287FF473AF129A0DF14C09680767
:10CB000005D5039BA3EB0804002C00F38A82DDE922
:10CB100003134145ACBF5B1843440493002A40F023
:10CB2000F38100230DF14C09119308E6029B9B89C8
:10CB30009A053FF55AAF029CA06DFEF771FBA389E1
:10CB400053E715F0100340F0188315F0400200F091
:10CB50001083059E984656F8043B05969EB2F7E66C
:10CB600056F8043BE806059600F11083690640F18B
:10CB70000A8343F3C0381EB243468FE64FF00003EA
:10CB8000059E8DF83B3056F8044B002C00F0CF8307
:10CB9000BBF1FF3F00F041835A4600212046FEF7DB
:10CBA0005DFE002800F02284031B4FF0000B059669
:10CBB00001938DE64FF000034FF00108059E8DF8BC
:10CBC0003B3056F8043B23AC8DF88C300596CDF8FD
:10CBD00004802DE7FDF79CFF85E5039B5B420393F3
:10CBE0003B7845F00405CAE53B786C2B03BF7B78A6
:10CBF00045F02005013745F01005C0E53B78682B6E
:10CC000003BF7B7845F40075013745F04005B6E574
:10CC100045F0100A1AF0200800F07E82059E0123DC
:10CC2000073626F007063246D6F8048052F8086B1D
:10CC3000059290E63B788DF83B80A0E530228DF898
:10CC40003C207822059B8DF83D2053F8046BBE4AAA
:10CC500005934FF00008022345F0020A09927AE694
:10CC6000AE0600F1A482EC0600F15983680600F1DB
:10CC7000B083A90540F15383059E049A56F8043BFE
:10CC80001A7005965BE5069C2046FEF7BFFA4368DE
:10CC900018460B93FAF7C0FF034620460C931C4638
:10CCA000FEF7B4FA83680A93002C3FF4E2AD0A9BC6
:10CCB000002B3FF4DEAD0A9B1B78002B3FF4D9AD6F
:10CCC0003B7845F480655AE53B7845F0010556E52B
:10CCD0009DF83B30002B7FF4CCAD20238DF83B300A
:10CCE0003B784CE53B7845F0800548E5394611F83E
:10CCF000013B2A2B00F0A683A3F13002092A0F463C
:10CD00004FF0000B3FF63CAD17F8013B0BEB8B0BE4
:10CD100002EB4B0BA3F13002092AF5D930E5AA4604
:10CD2000012B3FF4C8AD022B3CAC12D1099A06F09E
:10CD30000F03D35C360946EA08764FEA181804F860
:10CD4000013D56EA0803F2D13CAB1B1B554601934B
:10CD5000BEE506F00703F60846EA48764FEAD8082B
:10CD6000303356EA0801224604F8013DF1D11AF0A9
:10CD7000010FE9D0302BE7D03023023A04F8013C10
:10CD80003CAB9B1A554614460193A1E50123019A39
:10CD900013941193149212920DF14C0909F10809A0
:10CDA000ADE6039BA3EB0806002E7FF789AE102E9D
:10CDB000DFF898A138DD5346CC46BA46C146079401
:10CDC000A8461F46069C029D07E001F1020E01469F
:10CDD0000CF1080C103E102E1EDD1023481C1032E2
:10CDE0000728CDE91102CCF80070CCF80430ECDD56
:10CDF000002A00F092802946204610AAFFF720FC66
:10CE000000287FF4ECADDDE91112103E102E0DF17B
:10CE10004C0C01F1010EE0DC3B4645465746C84646
:10CE20007046E1469A46079C32440728CDE9110234
:10CE3000C9F800A0C9F8046040F39681002A00F008
:10CE40009A820299069810AAFFF7FAFB00287FF44D
:10CE5000C6ADDDE91112019B0DF14C09ABEB0306E8
:10CE6000002E01F101007FF731AE102E40F36B82EE
:10CE7000DFF8D8A0CC465346C146BA46A846079428
:10CE80004FF0100B1F46069C029D07E001F1020EB9
:10CE900001460CF1080C103E102E19DD481C103212
:10CEA0000728CCE9007BCDE91102EFDD32B329463A
:10CEB000204610AAFFF7C4FB00287FF490ADDDE9FF
:10CEC0001112103E102E0DF14C0C01F1010EE5DC9B
:10CED0003B4645465746C8467046E1469A46079C3B
:10CEE00032440728CDE91102C9F800A0C9F804604E
:10CEF00000F3E98009F108090130E7E54FF0010E80
:10CF000011460DF14C0CC6E70299069810AAFFF7DE
:10CF100097FB00283FF405AE61E54FF0010E114686
:10CF20000DF14C0C56E7002A00F0DE8002990698BD
:10CF300010AAFFF785FB00287FF451ADDDE911123F
:10CF40000DF14C09481C9AE5E4DD00086CE000088E
:10CF5000022201200FAB13930DF14C0914920146EC
:10CF600009F10809481CA7E5102E40F34582DDE9C8
:10CF70001132DFF8F0A219465346CC46BA46C146F4
:10CF80000D94A8461F46069C029D07E001F1020E83
:10CF900001460CF1080C103E102E1CDD1023481C1D
:10CFA00010320728CDE91102CCF80070CCF804301B
:10CFB000ECDD32B32946204610AAFFF741FB0028DA
:10CFC0007FF40DADDDE91112103E102E0DF14C0C69
:10CFD00001F1010EE2DC3B4645465746C846714624
:10CFE000E1469A460D9C32440729CDE91112C9F851
:10CFF00000A0C9F8046000F3A78009F10809481CE3
:10D000002BE511464FF0010E0DF14C0CC3E76C07F8
:10D01000119250D5039BA3EB0804002C4BDD0DF1BE
:10D020004C09102C40F3F881DFF838A21025534644
:10D030001199BA46069E1F46DDF808B006E0881C26
:10D04000194609F10809103C102C19DD4B1C10324F
:10D05000072BC9E90075CDE91132F0DD32B359462D
:10D06000304610AAFFF7ECFA00287FF4B8ACDDE9EF
:10D070001112103C102C0DF14C0901F10100E5DCFE
:10D080003B4657469A4622440728C9E900A4CDE901
:10D0900011027FF73CAD72B10299069810AAFFF712
:10D0A000CFFA00287FF49BAC129A30E5012011469C
:10D0B0000DF14C09C7E7DDE903234245ACBF9B18DE
:10D0C000434404932DE5002A3FF460AE029906988C
:10D0D00010AAFFF7B5FA00287FF481AC1198129AD4
:10D0E0000DF14C090130F1E4079B002B69D10120BF
:10D0F00011460DF14C09DFE411920DF14C0958E491
:10D10000BBF1000F7FF4DCAB55464FF0000B3CAC9D
:10D11000CDF804B0FFF7DCBB1AF0100340D11AF0D1
:10D12000400239D0059E984656F8042B01230596F7
:10D1300096B210E42D2376428DF83B30AA464FF08C
:10D14000010368EB48080AE4002A6FD002990698A8
:10D1500010AAFFF775FA00287FF441AC0DF14C09D5
:10D1600078E43CACFFF7B4BB014609F10809013093
:10D17000A6E415F4007840F01D81059B53F8046B7C
:10D180000593FFF7E5BBAA0500F10E814FEAE378AE
:10D190001E464346FFF782BB1AF4007840F0FB803E
:10D1A000059A012352F8046B0592FFF7D4BBDDE921
:10D1B000041656F8042BCB17C2E900130596FFF7A7
:10D1C000BEBA02220FAB13930DF14C091492C7E6BD
:10D1D000254A099215F0200836D0059E073626F01C
:10D1E00007063246D6F8048052F8086B0592EA0723
:10D1F00009D556EA080206D08DF83D30302345F0B7
:10D2000002058DF83C30022325F4806AFFF7A3BBAA
:10D21000AA46FFE4154A0992DCE720460596FAF78C
:10D22000FBFC4FF0000B0190FFF752BB9DF83B1049
:10D23000002900F0A68001200DF13B0213920DF1B0
:10D240004C090246149016E415F0100214D115F0A2
:10D2500040010DD0059E904656F8042B059696B2D7
:10D26000C5E700BF5CE00008F8DD0008E4DD000869
:10D2700015F4007840F0A680059A52F8046B0592E8
:10D28000B5E700230AF48062CDF804B0CDF81CA005
:10D29000BB46CDF820909A461746DDF828903CAD65
:10D2A0000CE00023304641460A22F3F7ABFC0A2E7D
:10D2B00078F100031BD30646884625463046414692
:10D2C0000A220023F3F79EFC30326C1E0AF1010A99
:10D2D00005F8012C002FE4D099F800305345E0D137
:10D2E000BAF1FF0FDDD00A2E78F100032ED2DDF85F
:10D2F0001CA03CAB1B1B5F46CDF82890DDF804B0AA
:10D300005546DDF820900193FFF7E2BAAA46FFF7F1
:10D31000D2BA012BAA467FF406ADFFF7D1BA059E1B
:10D32000049A56F8043B1A600596FFF708BABBF159
:10D33000060FD84628BF4FF00608474CCDF80480AA
:10D340000596FFF775BBDFF814A1C9E50C9B0B9997
:10D35000E41A1A462046FAF78DFC99F801300BB111
:10D3600009F10109304641460A2200234FF0000A24
:10D37000F3F748FC9FE7012011460DF14C09FFF738
:10D380009FBB079B002B7FF4E3AD114601200DF1FD
:10D390004C09FFF795BB059E904656F8042B0123D8
:10D3A0000596D6B2FFF7D7BA43F3C0185EB243462C
:10D3B000FFF774BA059E904656F8043B0596DEB218
:10D3C000FFF7C6BA059E884656F8042B0596D6B2D6
:10D3D0000DE7059E049A56F8043B1A800596FFF760
:10D3E000AEB9886DFDF71CFFFFF799BACDF804B010
:10D3F00005968346FFF76CBA1199129ADFF860A080
:10D400000131F0E50299069810AAFFF719F90028F2
:10D410003FF4E3AAFFF7E3BA1198DFF844A0013024
:10D4200031E6029B5B6EDB0707D4029B9B899F055D
:10D4300003D4029B986DFDF7F3FE4FF0FF33049386
:10D44000FFF7D6BA059A7B780F4652F8041B05926F
:10D4500041EAE17BFFF793B90CDE00086CE00008BD
:10D460005CE00008F0B54FF4806C154600240646D9
:10D470001F46ADF26C4D1AAB009304938B8916A82E
:10D4800023F00203ADF80C304B6E06941993CB8950
:10D490000C46ADF80E30CB69CDF808C007934B6A47
:10D4A000CDF814C00993FDF7B5FE2A463B46694600
:10D4B0003046FFF70BF9051E07DB69463046FDF7DE
:10D4C000F3FA002818BF4FF0FF35BDF80C305B06AB
:10D4D00003D5A38943F04003A3811698FDF79CFE72
:10D4E00028460DF26C4DF0BD38B50C4611460022B1
:10D4F0008446074D20462A601A466446F5F7C0F96F
:10D50000431C00D038BD2B68002BFBD0236038BDF6
:10D51000E49F0020144600B51A460A4B0D461B68CE
:10D5200085B0DE6803464CB1074901913046074992
:10D530000294009500F0C2F800F04AFA04490C4643
:10D54000F3E700BF940000207CE000088CE00008B6
:10D5500088E0000838B5A1FB021484BBFDF7D2FEB9
:10D560000546D8B150F8042C22F00302043A242ACC
:10D5700016D8132A19D91B2AC0E900441CD9002344
:10D58000242A14BF00F1100200F11802C0E902447D
:10D5900004BF04614461C2E900339360284638BD8A
:10D5A0002146FAF711FA284638BD024600232846DC
:10D5B000C2E90033936038BD00F10802F6E7FAF7DC
:10D5C000D9F90C2300250360E8E700BF002238B535
:10D5D000064D044608462A60F5F7B4F8431C00D00F
:10D5E00038BD2B68002BFBD0236038BDE49F0020A2
:10D5F00070B500294BD006460C4610B1836B002B4A
:10D6000048D0636ED80734D5B4F90C30002B3ED027
:10D6100021463046FDF7B6F9E36A054633B1304698
:10D62000E16998470028B8BF4FF0FF35A3891A0673
:10D630003BD4216B41B104F14003994202D0304602
:10D64000FDF748FB00232363616C21B13046FDF7F1
:10D6500041FB00236364FDF7E1FA0022636EA281BF
:10D66000DB0727D5A06DFDF7D7FDFDF7DDFA2846CE
:10D6700070BDA3899905CBD4A06DFDF7CFFDB4F99A
:10D680000C30002BC4D1656E15F0010508D00025C3
:10D69000284670BDFDF73CFA636ED807B4D4E8E7BE
:10D6A000A06DFDF7BDFD284670BD30462169FDF730
:10D6B00011FBBEE7A06DFDF7B3FDD3E70EB400B5D7
:10D6C000074A82B003AB0146106853F8042B01935C
:10D6D000FEF7FCFF02B05DF804EB03B0704700BF3B
:10D6E000940000202DE9F04383B007468846144695
:10D6F00000F0A2F8012803D108F1FF33FE2B33D943
:10D700004246384604F15C0301A900F035F9421C99
:10D7100006462FD018B39DF8041000250DF1050919
:10D7200008E023685A1C226019700135B54216D2F0
:10D7300019F8011BA368013B002BA360F1DAA26971
:10D74000934201DB0A29ECD12246384600F0BCF8AE
:10D75000431CEAD10646304603B0BDE8F083464696
:10D76000304603B0BDE8F0835FFA88F106468DF8D5
:10D770000410D2E73046A38943F04003A38103B0ED
:10D78000BDE8F08330B5536E144613F0010FB2F9C3
:10D790000C30054683B09AB201D198051CD590048F
:10D7A00006D4626E43F4005342F40052A3816266D1
:10D7B00022462846FFF796FF636E0546DA0702D435
:10D7C000A3899B0502D5284603B030BDA06DFDF7A7
:10D7D00027FD284603B030BDA06D0191FDF71EFD69
:10D7E000B4F90C3001999AB2D9E700BF70B50026A0
:10D7F000074D0446084611462E60F4F7A6FF431C69
:10D8000000D070BD2B68002BFBD0236070BD00BF23
:10D81000E49F0020002238B5064D044608462A60E1
:10D82000F4F798FF431C00D038BD2B68002BFBD0C9
:10D83000236038BDE49F0020014B93F82801704716
:10D84000D008002038B50C46114600228446074D0A
:10D8500020462A601A466446F4F77EFF431C00D037
:10D8600038BD2B68002BFBD0236038BDE49F00201F
:10D8700082B049B15AB16BB113780B601278101EA7
:10D8800018BF012002B0704701A9002AF3D1104649
:10D8900002B070476FF00100F4E700BF38B50C46E6
:10D8A000114600228446074D20462A601A466446E7
:10D8B000F4F7CEFF431C00D038BD2B68002BFBD003
:10D8C000236038BDE49F0020F8B506460D46144697
:10D8D00010B1836B002B43D0B4F90C20A36910075F
:10D8E000A36091B21BD52369CBB1EDB289042F4659
:10D8F00022D522686169D31A994229DD0133A168D2
:10D900000139A160511C2160157062699A422AD0C8
:10D91000A389DB0701D50A2D25D03846F8BD21465D
:10D920003046FBF7C9FF20BBB4F90C20EDB291B231
:10D9300089042F462369DCD442F40052A281626E2E
:10D94000616922F4005262662268D31A9942D5DCDA
:10D9500021463046FDF7A8F858B901232268CEE7E2
:10D96000FDF7D6F8B8E721463046FDF79DF80028C8
:10D97000D3D04FF0FF37D0E770B505461C4684B0D2
:10D9800039B10B4ED6F8E060B047431C09D004B063
:10D9900070BD0A460649D1F8E06001A9B047431CB2
:10D9A000F5D100228A2322602B6004B070BD00BF35
:10D9B000D0080020034649B1FF2A02D801200A708E
:10D9C00070478A224FF0FF301A6070470846704750
:10D9D000062008B500F004F80120F4F7ADFE00BF02
:10D9E00038B5154B1F281D6820D8D5F8DC22044611
:10D9F00062B152F820304BB1012B15D0591C0FD019
:10DA0000002542F820509847284638BD284600F0A7
:10DA100029F8224601462846BDE8384000F00EB8F5
:10DA2000162301202B6038BD002038BD16234FF08F
:10DA3000FF302B6038BD00BF9400002070B5002679
:10DA4000074D0446084611462E60F4F76DFE431C50
:10DA500000D070BD2B68002BFBD0236070BD00BFD1
:10DA6000E49F0020F4F75EBEF8B500BFF8BC08BC28
:10DA70009E467047F8B500BFF8BC08BC9E4670478C
:10DA800044454255473A205468652073797374655C
:10DA90006D207374617274732072756E6E696E6737
:10DAA0002E0D000064656661756C745461736B00C3
:10DAB000A4DA0008000000000000000000000000E0
:10DAC0000000000000020000300000000000000024
:10DAD0000000000044454255473A20576169746987
:10DAE0006E6720666F722067617465776179207454
:10DAF0006F2073746172742E0D000000736C617678
:10DB0000655F3438355F7461736B0000FCDA0008C0
:10DB10000000000000000000000000000000000005
:10DB200000020000280000000000000000000000CB
:10DB300000000000000000000102030406070809BD
:10DB4000000000000102030444454255473A2066A4
:10DB50006C6173685F65726173650D004445425581
:10DB6000473A20436F64655F53746F726167655F06
:10DB7000446F6E650D00000044454255473A2066EB
:10DB80006C6173685F77726974653A25640D0A0089
:10DB900044454255473A20637263206572726F7242
:10DBA0003A25640D0A00000002030405060708096F
:10DBB0000A0B0C0D0E0F10100102000000C1814075
:10DBC00001C0804101C0804100C1814001C080414D
:10DBD00000C1814000C1814001C0804101C080413D
:10DBE00000C1814000C1814001C0804100C181402D
:10DBF00001C0804101C0804100C1814001C080411D
:10DC000000C1814000C1814001C0804100C181400C
:10DC100001C0804101C0804100C1814000C18140FC
:10DC200001C0804101C0804100C1814001C08041EC
:10DC300000C1814000C1814001C0804101C08041DC
:10DC400000C1814000C1814001C0804100C18140CC
:10DC500001C0804101C0804100C1814000C18140BC
:10DC600001C0804101C0804100C1814001C08041AC
:10DC700000C1814000C1814001C0804100C181409C
:10DC800001C0804101C0804100C1814001C080418C
:10DC900000C1814000C1814001C0804101C080417C
:10DCA00000C1814000C1814001C0804100C181406C
:10DCB00001C0804101C0804100C1814000C0C1015C
:10DCC000C30302C2C60607C705C5C404CC0C0DCDEC
:10DCD0000FCFCE0E0ACACB0BC90908C8D81819D95C
:10DCE0001BDBDA1A1EDEDF1FDD1D1CDC14D4D5158C
:10DCF000D71716D6D21213D311D1D010F03031F17C
:10DD000033F3F23236F6F737F53534F43CFCFD3DAB
:10DD1000FF3F3EFEFA3A3BFB39F9F83828E8E9299B
:10DD2000EB2B2AEAEE2E2FEF2DEDEC2CE42425E54B
:10DD300027E7E62622E2E323E12120E0A06061A1BB
:10DD400063A3A26266A6A767A56564A46CACAD6D6B
:10DD5000AF6F6EAEAA6A6BAB69A9A86878B8B979DB
:10DD6000BB7B7ABABE7E7FBF7DBDBC7CB47475B50B
:10DD700077B7B67672B2B373B17170B050909151FB
:10DD80009353529296565797559594549C5C5D9D2B
:10DD90005F9F9E5E5A9A9B5B99595898884849891B
:10DDA0004B8B8A4A4E8E8F4F8D4D4C8C44848545CB
:10DDB00087474686824243834181804049444C459F
:10DDC00000000000546D725100000000546D72207C
:10DDD00053766300494E4600696E66004E414E0020
:10DDE0006E616E0030313233343536373839616226
:10DDF00063646566000000003031323334353637F5
:10DE0000383941424344454600000000286E756C95
:10DE10006C2900003000000020202020202020203D
:10DE20002020202020202020303030303030303072
:10DE300030303030303030304E614E00496E6669DF
:10DE40006E6974790000000042616C6C6F6320732E
:10DE50007563636565646564000000002F6D6E7412
:10DE60002F776F726B73706163652F776F726B734F
:10DE7000706163652F4743432D31302D70697065A4
:10DE80006C696E652F6A656E6B696E732D474343CF
:10DE90002D31302D706970656C696E652D333338A6
:10DEA0005F32303231313031385F313633343531F1
:10DEB000363230332F7372632F6E65776C69622F41
:10DEC0006E65776C69622F6C6962632F7374646C22
:10DED00069622F64746F612E630000002F6D6E7491
:10DEE0002F776F726B73706163652F776F726B73CF
:10DEF000706163652F4743432D31302D7069706524
:10DF00006C696E652F6A656E6B696E732D4743434E
:10DF10002D31302D706970656C696E652D33333825
:10DF20005F32303231313031385F31363334353170
:10DF3000363230332F7372632F6E65776C69622FC0
:10DF40006E65776C69622F6C6962632F7374646CA1
:10DF500069622F6D707265632E630000000000001F
:10DF60000080E03779C34143176E05B5B5B89346D5
:10DF7000F5F93FE9034F384D321D30F94877825AA1
:10DF80003CBF737FDD4F1575000000000000F03FBF
:10DF90000000000000002440000000000000594084
:10DFA0000000000000408F40000000000088C340D7
:10DFB00000000000006AF8400000000080842E414C
:10DFC00000000000D01263410000000084D7974198
:10DFD0000000000065CDCD41000000205FA002429E
:10DFE000000000E876483742000000A2941A6D4213
:10DFF000000040E59C30A2420000901EC4BCD64206
:10E0000000003426F56B0C430080E03779C34143B0
:10E0100000A0D8855734764300C84E676DC1AB4326
:10E02000003D9160E458E143408CB5781DAF154444
:10E0300050EFE2D6E41A4B4492D54D06CFF080441F
:10E04000F64AE1C7022DB544B49DD9794378EA4434
:10E0500005000000190000007D00000020202020A5
:10E060002020202020202020202020203030303070
:10E070003030303030303030303030302C20667539
:10E080006E6374696F6E3A200000000061737365FF
:10E090007274696F6E2022257322206661696C6537
:10E0A000643A2066696C6520222573222C206C69F5
:10E0B0006E65202564257325730A00004300000067
:10E0C000504F5349580000002E000000002020202F
:10E0D0002020202020202828282828202020202018
:10E0E00020202020202020202020202020881010E8
:10E0F0001010101010101010101010101004040444
:10E100000404040404040410101010101010414101
:10E1100041414141010101010101010101010101EF
:10E120000101010101010101101010101010424203
:10E1300042424242020202020202020202020202BF
:10E14000020202020202020210101010200000005F
:10E1500000000000000000000000000000000000BF
:10E1600000000000000000000000000000000000AF
:10E17000000000000000000000000000000000009F
:10E18000000000000000000000000000000000008F
:10E19000000000000000000000000000000000007F
:10E1A000000000000000000000000000000000006F
:10E1B000000000000000000000000000000000005F
:10E1C000000000000000000000000000000000004F
:08E1D000642AFF7F010000003A
:10E1D80000127A0001010000100000000200000097
:10E1E80011000000C949000803000000BF480008EA
:10E1F800100000006B480008060000003F480008B7
:10E2080017000000234900081500000029480008ED
:10E2180000000000000000000000000000000000F6
:10E2280000000000000000000000000000000000E6
:10E2380000000000000000000000000000000000D6
:10E2480000000000000000000000000000000000C6
:10E2580000000000000000000000000000000000B6
:10E26800AAAAAAAA9800002000000000840300209F
:10E27800EC0300205404002000000000000000000F
:10E288000000000000000000000000000000000086
:10E298000000000000000000000000000000000076
:10E2A8000000000000000000000000000000000066
:10E2B8000000000000000000000000000000000056
:10E2C8000000000000000000000000000000000046
:10E2D8000000000000000000000000000000000036
:10E2E8000000000000000000000000000000000026
:10E2F8000000000000000000000000000000000016
:10E308000000000000000000000000000000000005
:10E3180001000000000000000E33CDAB34126DE6A2
:10E32800ECDE05000B00000000000000000000000B
:10E3380000000000000000000000000000000000D5
:10E3480000000000000000000000000000000000C5
:10E3580000000000000000000000000000000000B5
:10E3680000000000000000000000000000000000A5
:10E698000000000000000000C0040020C0040020AA
:10E6A800C8040020C8040020D0040020D0040020A2
:10E6B800D8040020D8040020E0040020E004002052
:10E6C800E8040020E8040020F0040020F004002002
:10E6D800F8040020F80400200005002000050020B0
:10E6E800080500200805002010050020100500205E
:10E6F800180500201805002020050020200500200E
:10E7080028050020280500203005002030050020BD
:10E71800380500203805002040050020400500206D
:10E72800480500204805002050050020500500201D
:10E7380058050020580500206005002060050020CD
:10E74800680500206805002070050020700500207D
:10E75800780500207805002080050020800500202D
:10E7680088050020880500209005002090050020DD
:10E778009805002098050020A0050020A00500208D
:10E78800A8050020A8050020B0050020B00500203D
:10E79800B8050020B8050020C0050020C0050020ED
:10E7A800C8050020C8050020D0050020D00500209D
:10E7B800D8050020D8050020E0050020E00500204D
:10E7C800E8050020E8050020F0050020F0050020FD
:10E7D800F8050020F80500200006002000060020AB
:10E7E8000806002008060020100600201006002059
:10E7F8001806002018060020200600202006002009
:10E8080028060020280600203006002030060020B8
:10E818003806002038060020400600204006002068
:10E828004806002048060020500600205006002018
:10E8380058060020580600206006002060060020C8
:10E848006806002068060020700600207006002078
:10E858007806002078060020800600208006002028
:10E8680088060020880600209006002090060020D8
:10E878009806002098060020A0060020A006002088
:10E88800A8060020A8060020B0060020B006002038
:10E89800B8060020B8060020C0060020C0060020E8
:10E8A800C8060020C8060020D0060020D006002098
:10E8B800D8060020D8060020E0060020E006002048
:10E8C800E8060020E8060020F0060020F0060020F8
:10E8D800F8060020F80600200007002000070020A6
:10E8E8000807002008070020100700201007002054
:10E8F8001807002018070020200700202007002004
:10E9080028070020280700203007002030070020B3
:10E918003807002038070020400700204007002063
:10E928004807002048070020500700205007002013
:10E9380058070020580700206007002060070020C3
:10E948006807002068070020700700207007002073
:10E958007807002078070020800700208007002023
:10E9680088070020880700209007002090070020D3
:10E978009807002098070020A0070020A007002083
:10E98800A8070020A8070020B0070020B007002033
:10E99800B8070020B8070020C0070020C0070020E3
:10E9A800C8070020C8070020D0070020D007002093
:10E9B800D8070020D8070020E0070020E007002043
:10E9C800E8070020E8070020F0070020F0070020F3
:10E9D800F8070020F80700200008002000080020A1
:10E9E800080800200808002010080020100800204F
:10E9F80018080020180800202008002020080020FF
:10EA080028080020280800203008002030080020AE
:10EA1800380800203808002040080020400800205E
:10EA2800480800204808002050080020500800200E
:10EA380058080020580800206008002060080020BE
:10EA4800680800206808002070080020700800206E
:10EA5800780800207808002080080020800800201E
:10EA680088080020880800209008002090080020CE
:10EA78009808002098080020A0080020A00800207E
:10EA8800A8080020A8080020B0080020B00800202E
:10EA9800B8080020B8080020FFFFFFFF00000200B0
:10EAA800430000000000000000000000000000001B
:10EAB800000000000000000000000000000000004E
:10EAC80043000000000000000000000000000000FB
:10EAD800000000000000000000000000000000002E
:10EAE80043000000000000000000000000000000DB
:10EAF800000000000000000000000000000000000E
:10EB080043000000000000000000000000000000BA
:10EB180000000000000000000000000000000000ED
:10EB2800430000000000000000000000000000009A
:10EB380000000000000000000000000000000000CD
:10EB4800430000000000000000000000000000007A
:10EB580000000000000000000000000000000000AD
:10EB6800430000000000000000000000000000005A
:10EB7800000000000000000000000000000000008D
:10EB8800B5D9000871D8000800000000CCE00008E2
:10EB9800C8E0000888E0000888E0000888E000086D
:10EBA80088E0000888E0000888E0000888E000089D
:10EBB80088E0000888E00008FFFFFFFFFFFFFFFF75
:10EBC800FFFFFFFFFFFF00000100415343494900D9
:10EBD800000000000000000000000000000000002D
:10EBE80000000000000000000000415343494900B4
:10EBF800000000000000000000000000000000000D
:0CEC080000000000000000000000000000
:0400000508002CEDD6
:00000001FF
